:100000000C946B090C948A090C948A090C941C0AB0
:100010000C94520A0C948A090C948A090C948A094B
:100020000C948A090C948A090C948A090C948A0904
:100030000C948A090C948A090C948A090C947D0DFD
:100040000C948A090C948A090C948A090C948A09E4
:100050000C94106E0C94C3650C948A090C948A0954
:100060000C948A090C9498660C948A090C948C66FA
:100070000C948A090C948A090C948A090C948A09B4
:100080000C9443790C948A090C948A090C948A097B
:100090000C94D6660C948A090C94CA660C948A094E
:1000A0000C948A090C948A090C948A090C948A0984
:1000B0000C948A090C948A090C948A090C948A0974
:1000C0000C948A090C948A090C948A090C948A0964
:1000D0000C948A090C948A090C948A090C948A0954
:1000E0000C948A090C94C96D0C94D36D0C94BF6D5B
:1000F0000C947F6D0C94046E0C94F56D0C94E96D6A
:100100000C94DD6D0C948A090C948A090C948A096C
:100110000C948A090C948A090C948A090C948A0913
:100120007A82998218830784278447844F84FC83CA
:10013000084AD73B3BCE016E84BCBFFDC12F3D6C4E
:1001400074319ABD56833DDA3D00C77F11BED9E4B4
:10015000BB4C3E916BAAAABE000000803F076342E1
:1001600036B79BD8A71A39685618AEBAAB558C1D4E
:100170003CB7CC5763BD6DEDFD753EF6177231BFD0
:10018000000000803F08000000BE922449123EABF0
:10019000AAAA2ABECDCCCC4C3E00000080BEABAAA1
:1001A000AAAA3E00000000BF000000803F0000003F
:1001B0000000084178D3BB4387D1133D190E3CC3DF
:1001C000BD4282AD2B3E68EC8276BED98FE1A93E5E
:1001D0004C80EFFFBE01C4FF7F3F00000000000025
:1001E00025730A005854414C5F5452494D3D2564D3
:1001F0000025730A0025730A0054657374203620A5
:1002000025730A005465737420352025730A005441
:1002100065737420342025730A0054657374203389
:100220002025730A005465737420322025730A0058
:100230005465737420312025730A006368616E3D34
:1002400025640A0074787077723D25640A003530A1
:10025000306B0A003235306B0A003131356B0A00E1
:1002600035366B0A0033386B0A0025730A00765F57
:100270006C6F773D252D332E32660A0025730A00F8
:1002800073656E743D252D75206475703D252D7543
:100290002069676E6F7265643D252D752074746CDE
:1002A0005F7A65726F3D252D750A0025372E3366FE
:1002B0002025372E33660025352E32662000457204
:1002C000726F72203020566F6C74004E6F74207302
:1002D0007570706F727465640A004572726F722077
:1002E0003020566F6C74004572726F722030205649
:1002F0006F6C74007062323D25730A00256C7500C6
:10030000416C6C6F77656420737065656420312F74
:1003100031302F3130302F343030206B6269742F00
:10032000730025630074746C3D252D642000747483
:100330006C3D252D6420004E65772074746C3D253E
:100340002D6420002563004D533536313120503D5A
:10035000252D372E326620252D372E32666D0A0068
:10036000424D5030383520256C64205061202025C6
:100370002D372E32666D00256300545F4845415489
:100380005F4944583D252D352E32662000545F4488
:1003900045573D252D352E3266200041483D252DFF
:1003A000352E32662000545F53485432583D252D77
:1003B000352E3266200052485F53485432583D254E
:1003C0002D352E32662000545F52483D252D342EA7
:1003D0003166200052483D252D342E3166200025FF
:1003E00063002563002563002563002563007265B3
:1003F000706F72745F616C6C3D007265706F7274C7
:100400003D00256300256300256300256300204F20
:10041000534343414C3D2564200020467573653AA3
:100420002065653D253032782068663D253032787C
:10043000206C663D25303278206C623D2530327864
:10044000004D43553D2530366C78002563007478A7
:100450005F6C656E3D252D6C752C765F6C6F773DFE
:10046000252D6C752C73687432783D252D6C750ABA
:10047000002563004F4B0A002563002563002563B8
:1004800000256300256300256300256300256300C4
:1004900064656275675F616C6C3D00646562756779
:1004A0003D0064656275673D0025730A00646565FB
:1004B000700A006E6F6E650A00707772733D00708F
:1004C00062323D25730A007062313D25730A00696E
:1004D0006E74725F7365635F70313D252D372E3307
:1004E000660A00696E74725F70313D252D6C640A76
:1004F00000696E74725F7365635F70303D252D37E0
:100500002E33660A00696E74725F70303D252D6C63
:10051000640A00765F6D63753D252D352E32660ABF
:1005200000745F6D63753D252D352E32660A0070AF
:100530007077723D25730A0064656275673D0072CD
:10054000636D643D25730A0025730A006175746F3D
:100550000A006C6F675F6D6F64653D007573625F65
:100560007077723D25730A0072656C61793D257361
:100570000A0074746C3D252D640A0052494D455F94
:10058000616464723D252D642E252D640A006E651C
:10059000696768626F725F7461626C655F73697AC4
:1005A000653D25640A00765F6C6F773D252D332EFF
:1005B00032660A00747870773D25640A00636861CA
:1005C0006E3D25640A0069643D006932635F6275AF
:1005D000733D006932635F73706565643D252D6C02
:1005E000750A007478743D25730A00537973746535
:1005F0006D2053756D6D6172790A002530366C7807
:100600000041744D656761323536524652320041C1
:10061000744D656761313238524652320041744D33
:100620006567613634524652320041744D656761E8
:1006300031323852464131004D43553D006D6173B2
:100640006B3D002C00696E74657276616C3D252DE2
:10065000750023252D642C00745F686561745F69E3
:10066000647800745F64657700616800705F6D7323
:10067000353631310072685F736874327800745FA8
:1006800073687432780070610070006164340061D6
:1006900064330061643200616431006133006132AF
:1006A00000613100765F696E0072680065727200E9
:1006B000757074696D650070315F6C7374007031B2
:1006C0005F740070310070305F6C73740070305F65
:1006D0007400703000765F6D637500745F6D6375D4
:1006E00000743100740069640065363400747874F5
:1006F000002D002B006175746F006E6F6E650070C9
:100700006F7765725F736176655F6C65647279009F
:1007100072656C61795F6C65647900636F6D70619F
:10072000737300616363656C007072657300705F62
:10073000707772006165730070315F6C6564790079
:1007400070305F6C656472006576656E74006C6510
:1007500064006F7700706B740074785F6C65647907
:100760000072785F6C656472006F706572006E6F06
:100770006E65002530327800765F6164343D252D4A
:10078000382E3666002000765F6164333D252D38B3
:100790002E3666002000765F6164323D252D382EAE
:1007A0003666002000765F6164313D252D382E3697
:1007B00066002000765F6C696768743D252D382ED1
:1007C0003666002000765F61323D252D372E336678
:1007D000002000765F61313D252D372E33660020E5
:1007E00000765F696E3D252D352E326600204E6500
:1007F0007665722D7573656420737461636B203E3A
:100800002025642062797465730A00757074696DBF
:10081000653D252D642D646179732D253032643A50
:10082000253032643A253032642D686F7572730A50
:100830000074657374205B6F66667C317C327C3338
:100840007C347C355D20202020202020202D207429
:10085000657374206D6F6465730A0D007478205B96
:10086000706B74207061796C6F61645D2020202052
:1008700020202020202020202D2073656E642072EF
:100880006164696F20706B74206B6579626F61724F
:10089000640A0D00776474205B6F6E7C6F66667C03
:1008A000746573745D2020202020202020202020CB
:1008B0002D207761746368646F670A0D00765F6C42
:1008C0006F77205B765F6C6F775D20202020202083
:1008D0002020202020202020202D206C6F77657381
:1008E00074207265706F727420766F6C74616765C6
:1008F0000A0D007570677220202020202020202003
:100900002020202020202020202020202020202DDA
:10091000207265626F6F742076696120626F6F74F8
:100920006C6F616465720A0D0075617274205B33CF
:10093000386B7C35366B7C3131356B7C3235306BC6
:100940007C3530306B5D202D2073657420746572AA
:100950006D2F756172742073706565640A0D006295
:100960006F6F742020202020202020202020202095
:1009700020202020202020202020202D2072656291
:100980006F6F740A0D0070777273205B6465657019
:100990007C6E6F6E655D202020202020202020208E
:1009A00020202D206D637520736C656570206D6F40
:1009B00064650A0D007265737420656570726F6DF1
:1009C0002020202020202020202020202020202027
:1009D000202D20726573746F726520656570726F6B
:1009E0006D0A0D0070707772205B6F6E7C6F6666AB
:1009F0005D202020202020202020202020202020BA
:100A00002D2070726F6772616D6D61626C65207010
:100A100077720A0D0070623220205B6F6E7C6F6609
:100A2000665D202020202020202020202020202043
:100A3000202D2070726F6772616D6D61626C652030
:100A400070696E2062320A0D00747874205B7374D2
:100A500072696E675D202020202020202020202029
:100A600020202020202D20536574207265706F7225
:100A700074207465787420737472696E670A0D004F
:100A800074787077205B31352D305D202020202058
:100A90002020202020202020202020202D205458DD
:100AA000205077722E204869676865737420302063
:100AB000283364426D290A0D0074746C205B302D5C
:100AC00031355D20202020202020202020202020C3
:100AD00020202020202D2074696D652D746F2D6CD1
:100AE00069766520666F72207061636B6574730A46
:100AF0000D00737320202020202020202020202083
:100B000020202020202020202020202020202D20D8
:100B100073797374656D2073756D6D6172790A0DEB
:100B20000072732020202020202020202020202040
:100B3000202020202020202020202020202D207256
:100B40006164696F2073746174730A0D00726920A7
:100B50005B236E5D205B696E745D20202020202069
:100B60002020202020202020202D207265706F72F0
:100B70007420696E74657276616C0A0D0072636D23
:100B800064205B6F6E7C6F66665D202020202020D5
:100B90002020202020202020202D20616C6C6F77C9
:100BA00020636D642066726F6D206E65746F726B6A
:100BB0000A0D007265205B236E5D205B2B7C2D5D32
:100BC000205B6D61736B7C6175746F2C6D61736BF1
:100BD0005D202D206D6F7465207265706F727420BA
:100BE0007365742F6D6F646966790A0D006F7720E5
:100BF00020202020202020202020202020202020F5
:100C00002020202020202020202D206F6E652D7791
:100C10006972652073656E736F72730A0D006C6F75
:100C200067205B6175746F7C6F6E7C6F66665D209C
:100C3000202020202020202020202D206D6F746572
:100C4000732064617461206F6E205553420A0D0059
:100C50006E65205B666C7573685D20202020202007
:100C60002020202020202020202020202D206E65E4
:100C7000696768626F72207461626C650A0D006555
:100C800072722020202020202020202020202020C0
:100C900020202020202020202020202D206572725E
:100CA0006F722073746174730A0D006D6375202078
:100CB0002020202020202020202020202020202034
:100CC000202020202020202D206D637520696E6655
:100CD0006F0A0D00693263205B70726F62657C730E
:100CE0007065656420236E5D202020202020202058
:100CF0002D206932632070726F6265206275737C8B
:100D0000736574206275732073706565640A0D00E5
:100D10006964205B72657365745D2020202020204B
:100D20002020202020202020202020202D20696429
:100D30002068616E646C696E670A0D0068756D20CD
:100D400020202020202020202020202020202020A3
:100D500020202020202020202D2068756D696469C6
:100D600074792073656E736F720A0D0072656C6121
:100D700079205B6F6E7C6F66667C73746174735DE3
:100D800020202020202020202D2072656C617920D9
:100D90006E6574776F726B207265706F7274730A10
:100DA0000D006465205B6D61736B5D202020202049
:100DB00020202020202020202020202020202D2026
:100DC00064656275670A0D006368616E205B31318E
:100DD0002D32365D202020202020202020202020A1
:100DE000202020202D206368616E2031312D323685
:100DF0002028322E3430352D32343830204D687A68
:100E0000290A0D0063616C69205B5B765F696E7C0B
:100E100061317C61325D20766F6C747C72657365C4
:100E2000747C6E6F6E655D202D2063616C696272EB
:100E30006174650A0D006164632020202020202059
:100E400020202020202020202020202020202020A2
:100E500020202D2073686F7720765F696E2C2061CB
:100E6000312C20613220766F6C74616765730A0DD6
:100E7000007520202020202020202020202020203D
:100E8000202020202020202020202020202D207500
:100E90007074696D650A0D007620202020202020C6
:100EA0002020202020202020202020202020202042
:100EB000202020202D2076657273696F6E0A0D0048
:100EC00068202020202020202020202020202020DA
:100ED0002020202020202020202020202D20686578
:100EE0006C700A0D00256300756E6B6E6F776E2057
:100EF000636D640A00484D4335383833002573006C
:100F0000257300202573002025362E32662000250B
:100F10003032780074656D705F65787465726E3D0F
:100F2000252D362E326600202573002025362E32E0
:100F300066204F6E2D426F6172640025303278005A
:100F400074656D705F626F6172643D252D362E325F
:100F500066000A00503A20256C642050612020254C
:100F60002D372E3266206D0A002563002563004967
:100F700032433A2000452025642E256420636C6F9F
:100F8000636B20256C752063707520256C75206C53
:100F9000706D20256C752069727120256C75206735
:100FA0006C656420256C7520796C656420256C75F2
:100FB00020726C656420256C7520747820256C7512
:100FC000206C697374656E20256C752073656E7373
:100FD0006F727320256C752073657269616C2025B2
:100FE0006C750A00532025642E256420636C6F63A2
:100FF0006B20256C7520747820256C752072782004
:10100000256C752072747820256C7520727278209A
:10101000256C75207265786D697420256C7520616A
:10102000636B747820256C75206E6F61636B7478C8
:1010300020256C752061636B727820256C75207497
:10104000696D65646F757420256C752062616461DB
:10105000636B727820256C7520746F6F6C6F6E6790
:1010600020256C7520746F6F73686F727420256C07
:10107000752062616473796E636820256C752062E7
:10108000616463726320256C7520636F6E74656E96
:1010900074696F6E64726F7020256C752073656E55
:1010A00064696E6764726F7020256C75206C6C7457
:1010B0007820256C75206C6C727820256C750A0080
:1010C000257325730A004F6E6C696E650A000A006D
:1010D0002C20636865636B20726174652025752020
:1010E000487A0025732025732C206368616E6E6535
:1010F0006C20257520706F776572202575000A00B9
:1011000025783A004D414320616464726573732011
:101110000052616E646F6D2045554936342061641C
:1011200064726573732067656E6572617465640AC5
:10113000000A2A2A2A2A2A2A2A426F6F74696E67AD
:101140002025732A2A2A2A2A2A2A0A00454550528B
:101150004F4D20697320636F72727570742C20720A
:101160006577726974696E67207769746820646551
:101170006661756C74732E0A006C6F63616C686FC6
:1011800073740041544D45474131323872666131C4
:1011900000020000FFFE0000016E616E00696E66D5
:1011A0000000407A10F35A00A0724E18090010A5F2
:1011B000D4E80000E87648170000E40B5402000071
:1011C000CA9A3B000000E1F50500008096980000F7
:1011D0000040420F000000A0860100000010270020
:1011E000000000E803000000006400000000000AA6
:1011F00000000000000100000000002C76D888DC10
:10120000674F0823DFC1DFAE59E1B1B796E5E3E4EC
:1012100053C63AE651997696E8E6C28426EB898C65
:101220009B62ED407C6FFCEFBC9C9F40F2BAA56FC7
:10123000A5F490055A2AF75C936B6CF9676DC11B96
:10124000FCE0E40D47FEF520E6B500D0ED902E035E
:1012500000943577050080841E080000204E0A00A7
:101260000000C80C333333330F986E12831141EFF3
:101270008D2114893BE65516CFFEE6DB18D1844B51
:10128000381BF77C1D901DA4BBE424203284725EC1
:10129000228100C9F124ECA1E53D274E414E494E83
:1012A000495459494E46CDCCCC3D0AD7233C17B7BB
:1012B000D13877CC2B329595E6241FB14F0A000028
:1012C00020410000C84200401C4620BCBE4CCA1B46
:1012D0000E5AAEC59D7411241FBECFEFD1E4DEBF00
:1012E000CDBF19E0A0E0B2E0ECE6FEE201E00BBF0A
:1012F00002C007900D92AE3BB107D9F721E3AEEBE8
:10130000B9E001C01D92A33DB207E1F70E941E851E
:101310000C9434970C9400008115910511F00197FD
:10132000F1F7089589EB94E09F938F930E941994AD
:101330008091580290915902A0915A02B0915B029B
:101340000F900F9093FF03C083EB94E002C08DEAEF
:1013500094E09F938F930E9419940F900F9008959B
:10136000E091771BEF73F0E0E853F44E80838091B7
:10137000771B8F5F8093771B80910D298860809306
:101380000D294EE352E061E1CA010E94A35580E0BD
:1013900090E00895CF93DF93EC018091C50990917F
:1013A000C60986FF1DC08E811F928F938D811F926B
:1013B0008F938C811F928F938B811F928F938A8141
:1013C0001F928F9385E693E09F938F930E940794DB
:1013D0008DB79EB70C960FB6F8949EBF0FBE8DBF0B
:1013E000BE018CEF99E00E94D556BE0184E092E0E8
:1013F000DF91CF910C944A568823B9F052985A98AD
:101400001DBA80916900806280936900EA9A5398BE
:101410005B98EB9A80916900806880936900809165
:1014200068008160809368000895109269005A9A5C
:10143000EA985B9AEB9808951F920F920FB60F925D
:1014400011248F939F93AF93BF938091680080FF87
:1014500020C08091E8289091E928A091EA28B091D5
:10146000EB280196A11DB11D8093E8289093E928EF
:10147000A093EA28B093EB288091C5099091C60902
:1014800087FF07C0749882E090E090938502809374
:101490008402BF91AF919F918F910F900FBE0F90DB
:1014A0001F9018951F920F920FB60F9211248F93D1
:1014B0009F93AF93BF938091680080FF20C080917D
:1014C000EC289091ED28A091EE28B091EF2801969C
:1014D000A11DB11D8093EC289093ED28A093EE28D8
:1014E000B093EF288091C5099091C60990FF07C07D
:1014F000739882E090E09093850280938402BF917C
:10150000AF919F918F910F900FBE0F901F901895E4
:1015100080937C0080917B00877F80937B0080910B
:101520007C00806C80937C0085E080937A008091C1
:101530007A00806880937A0080917B0087FFFCCFDF
:1015400080917B0085FFFCCF80917A00806480933E
:101550007A0080917A0086FDFCCF1092790010927B
:10156000780084E090E060E070E020917A002064F0
:1015700020937A0020917A0026FDFCCF20917800FC
:1015800030917900620F731F0197009771F71092E5
:101590007C0080917A008F7780937A0076956795AA
:1015A0007695679580E090E00E94748A089580E0C7
:1015B0000E94880A20917C0230917D0240917E0237
:1015C00050917F020E94588C21EE3AE744E95EE395
:1015D0000E940D8908950F931F93CF93DF93CFE15E
:1015E000D0E00BE51EE0C093510187EC90E00E9433
:1015F0008C098091510185FD0DC0C031D10521F0CC
:101600002CF00B54110904C004EC19E00253110929
:101610002197E9CFB80180E090E00E94748A20E031
:1016200030E04AE754E40E94D789DF91CF911F91BF
:101630000F910895CF93DF93EC01888199810097F2
:1016400099F0873B904121F01982188283E011C004
:10165000623171F40E94EB0A60933F24709340243E
:10166000809341249093422487EB90E1998388836F
:1016700081E0DF91CF91089580917B008860809315
:101680007B0089EC80937C0085E080937A008091D8
:101690007A00806880937A0080917B0087FFFCCF7E
:1016A00080917B0085FFFCCF80917A0080648093DD
:1016B0007A0080917A0086FDFCCF80917A00806468
:1016C00080937A0080917A0086FDFCCF609178004B
:1016D0007091790080917A008F7780937A0080E012
:1016E00090E00E94748A27ED33EA40E95FE30E94AC
:1016F000588C26E636E648E853E40E940C890895A3
:10170000BF92CF92DF92EF92FF920F931F93CF93EE
:10171000DF93CDB7DEB729970FB6F894DEBF0FBEC3
:10172000CDBF6C011092BE098FEF898708E81BE1DD
:10173000B12C7E0189E0E80EF11C89858823E9F14E
:10174000E8E0BE16E1F1BE016F5F7F4FC7010E9466
:101750003E5F89858F3F11F08E3F19F48093BE095B
:101760002CC0CE010196C114D10471F40E94575FC0
:1017700080930A29FE013196A2E0B9E281918D930E
:10178000EE15FF05D9F71DC00E94575FF801808351
:10179000FE01319620E030E0A801485051098191C6
:1017A000DA01A20FB31F8C932F5F3F4F2830310512
:1017B000B1F7B394075F1F4FC0CF8B2D03C088E0F4
:1017C00001C081E029960FB6F894DEBF0FBECDBFF1
:1017D000DF91CF911F910F91FF90EF90DF90CF900D
:1017E000BF90089582E59FE09F938F930E94199484
:1017F0000F900F9008952F923F924F925F926F92A9
:101800007F928F929F92AF92BF92CF92DF92EF9290
:10181000FF920F931F93CF93DF93EC014B0100973F
:1018200011F427E004C08130910549F426E04AE232
:1018300050E06BE270E089E290E00E941E5ECE0113
:101840000E94800B9E012154364F5901D9018C937F
:10185000CD2B69F098E8C92E9BE1D92EC0E8DBE1D9
:10186000E12CF12C23E0222E2FE0322EA6C082E0C4
:1018700099E20E948C60BC01882777FD8095982FA3
:101880000E94768A6B017C01892869F020E030E0B3
:1018900048EC52E40E94D7899F938F937F936F9374
:1018A00080E49FE0ACC0C2E0D9E20BE31FE0899185
:1018B0001F928F931F930F930E9419940F900F9074
:1018C0000F900F90B9E2CA30DB0789F720E030E0D3
:1018D00048EC52E4C701B6010E94D7899F938F93C9
:1018E0007F936F938BE29FE09F938F930E94199455
:1018F0000F900F900F900F900F900F9080910A29EA
:10190000882319F084E993E002C088E094E09F9373
:101910008F9387E29FE09F938F930E9419940F907B
:101920000F900F900F9075C000E010E0FE01E00FE7
:10193000F11F80811F928F93AFE0BFE0BF93AF9301
:101940000E9419940F5F1F4F0F900F900F900F90F0
:101950000830110559F720E030E048EC52E4C301AB
:10196000B2010E94D7899F938F937F936F93A7E0D3
:10197000BFE0BF93AF930E9419940F900F900F9008
:101980000F900F900F90D6018C91882309F455C0C9
:1019900084E993E09F938F933F922F920E94199432
:1019A0000E94F20BBFEFEB1AFB0AE9E0CE0ED11C4E
:1019B00029960F900F900F900F90D5018C9190E089
:1019C000E816F906ECF5CE010E948C60BC01882770
:1019D00077FD8095982F0E94768A2B013C01811417
:1019E000910409F4A1CF20E030E048EC52E40E94D9
:1019F000D7899F938F937F936F9384E19FE09F9309
:101A00008F930E9419940F900F900F900F900F904A
:101A10000F90DF91CF911F910F91FF90EF90DF908A
:101A2000CF90BF90AF909F908F907F906F905F907E
:101A30004F903F902F900C94F20B88E094E0AACF47
:101A4000DF91CF911F910F91FF90EF90DF90CF909A
:101A5000BF90AF909F908F907F906F905F904F90CE
:101A60003F902F900895CF93DF9300D0CDB7DEB78E
:101A7000809103298983809109298A83CE01019667
:101A80000E9497530F900F90DF91CF910895CF93BD
:101A9000DF93EC0120910229309103294091042920
:101AA0005091052960910629709107298091082994
:101AB00090910929AFEF0E94888FE1F427E04AE274
:101AC00050E06BE270E089E290E00E941E5E80E0F0
:101AD00090E00E94800BC154D64F888349E050E0CB
:101AE0006AE070E082E099E20E948B95DF91CF91ED
:101AF0000C94330DDF91CF9108951F920F920FB682
:101B00000F9211240BB60F92DF92EF92FF920F9378
:101B10001F932F933F934F935F936F937F938F9375
:101B20009F93AF93BF93CF93DF93EF93FF938091F6
:101B30000D29826080930D298091580286FD2B9A91
:101B40008091580287FD2B9A8091840290918502A2
:101B50001816190614F4749A739A8091C509909115
:101B6000C60985FF02C07498739880910202909113
:101B7000030201979093030280930202892B09F0DC
:101B800037C18091D3099091D40901969093D409DB
:101B90008093D3098091432490914424A0914524BB
:101BA000B09146240196A11DB11D809343249093CA
:101BB0004424A0934524B093462480E190E0909380
:101BC0000302809302028091580280FD02C01D9B97
:101BD00005C01092C3091092C20906C081E090E0CE
:101BE0009093C3098093C2098091C5099091C60959
:101BF00097FF08C08091C2099091C309892B61F0B9
:101C0000749A739807E21BE1C4E5D4E234E0E32E52
:101C1000F12CDD24D3941FC0739A7498F3CF809174
:101C2000D3099091D40901960E94288D892BD1F077
:101C3000F801608571856115710509F5F801608508
:101C400071856115710569F5065F1F4F2596FBE1EA
:101C50000F341F07D1F1F801608571856115710599
:101C600039F3DDCF77988091C5099091C60992FF2D
:101C7000DFCF7498F0928502E0928402D9CF8091F0
:101C8000D3099091D40901960E94288D892BB1F631
:101C90001C821B82AE0162E186E192E00E94A355A4
:101CA000CDCF8091D3099091D4090E94288D892BA2
:101CB00059F6D8821A8309831C821B82AE0162E125
:101CC00084E392E00E94A355BFCF60915E027091C1
:101CD0005F0261157105A1F18091D3099091D4093A
:101CE0000E94288D892B61F58091E8289091E92840
:101CF000A091EA28B091EB284091351C5091361CF8
:101D00006091371C7091381C841B950BA60BB70B88
:101D100080934F1B9093501BA093511BB093521B69
:101D20008091E8289091E928A091EA28B091EB28C9
:101D30008093351C9093361CA093371CB093381CAD
:101D400060915C0270915D0261157105A1F1809155
:101D5000D3099091D4090E94288D892B61F5809137
:101D6000EC289091ED28A091EE28B091EF284091B9
:101D7000391C50913A1C60913B1C70913C1C841B97
:101D8000950BA60BB70B8093531B9093541BA093FA
:101D9000551BB093561B8091EC289091ED28A09193
:101DA000EE28B091EF288093391C90933A1CA093B1
:101DB0003B1CB0933C1C8091580286FD2B9880916F
:101DC000580290915902A0915A02B0915B0291FF82
:101DD0000FC00E943D6A8A3119F0C1E0C80F01C0EE
:101DE000CBE00E94F9688C2F0E94556A0E944169DD
:101DF00040E050E060E086E892E00E94A355FF9149
:101E0000EF91DF91CF91BF91AF919F918F917F9192
:101E10006F915F914F913F912F911F910F91FF9083
:101E2000EF90DF900F900BBE0F900FBE0F901F90A2
:101E300018958091771B90915324891B08950E94D7
:101E4000190F882371F0E0915324EF73F0E0E85309
:101E5000F44E808190E0209153242F5F20935324EF
:101E600008958FEF9FEF0895CF93DF93EC011092C9
:101E7000F0091092EF09888199810097B1F08638B6
:101E8000934021F01982188283E0B6C0613109F0D5
:101E9000B2C00E941F0F99279093EB098093EA0923
:101EA0008D3009F443C08F3F49F40E94190F81110E
:101EB000F0CF86E893E0998388839DC082319105B5
:101EC00009F45AC08F37910509F052C08091E80992
:101ED0009091E909181619060CF56091CD317091B1
:101EE000CE3188E090E00E94D5936091CD31709121
:101EF000CE3180E290E00E94D5936091CD31709117
:101F0000CE3188E090E00E94D5938091E8099091CD
:101F1000E90901979093E9098093E8098091E8091C
:101F20009091E9098F37910509F0BFCF10925324A2
:101F30001092771B8091E8099091E909FC01E8591A
:101F4000FB4D10829093F0098093EF091092E909FC
:101F50001092E80980910B2990910C29009709F4BF
:101F6000A4CF40E050E06091FE110E94A3559DCFA8
:101F70008830910571F5AACF6091CD317091CE3145
:101F80008DE090E00E94D5931092E7091092E60947
:101F90008091E6099091E7092091E8093091E909DB
:101FA000821793070CF0BACFFC01E859FB4D8081F2
:101FB0006091CD317091CE3190E00E94D5938091A7
:101FC000E6099091E70901969093E7098093E60965
:101FD000DFCF6091CD317091CE310E94D593809149
:101FE000E8099091E9092091EA09FC01E859FB4DC3
:101FF000208301968FCF81E0DF91CF91089580916A
:10200000C2099091C309892BD1F080915802909117
:102010005902A0915A02B0915B0293FD10C00E9438
:10202000F96883B7817F866083BFF89483B7816046
:1020300083BF7894889583B78E7F83BF7894089503
:10204000CF93DF93EC0188819981009719F08A3E44
:10205000904199F40E94B6670E94FF0F40E050E063
:1020600065E880910212909103120E94A3558AEEB6
:1020700090E19983888381E003C01982188283E00C
:10208000DF91CF910895CF93DF9300D0CDB7DEB726
:10209000892B81F05F934F9380E09FE09F938F9314
:1020A00069837A830E9419940F900F900F900F907C
:1020B0007A8169817F936F938DEF9EE09F938F93D9
:1020C0000E9419940F900F900F900F900F900F9007
:1020D000DF91CF910895FF920F931F93CF93DF93DA
:1020E0000E94B66780EB0E94196181111CC00E949A
:1020F0007D6180913D2090913E20816090933E20B3
:1021000080933D208DE993E09F938F938DEF9EE028
:102110009F938F930E9419940F900F900F900F90A0
:10212000C1E0D0E002C0C0E0D0E0FEB08F2D8470EE
:10213000F82E729A0E94B6678EE40E94196181118E
:1021400016C00E947D6180913D2090913E2082606A
:1021500090933E2080933D208E010F5F1F4F43E2FE
:1021600059E065EA73E0CE010E944310E801F110E6
:1021700001C072980E94B6678EEE0E9419618111AB
:1021800016C00E947D6180913D2090913E20846028
:1021900090933E2080933D208E010F5F1F4F43E2BE
:1021A00059E06DEA73E0CE010E944310E8010E94FD
:1021B000B66786EA0E941961811116C00E947D618E
:1021C00080913D2090913E20886090933E208093A6
:1021D0003D208E010F5F1F4F43E259E064EB73E037
:1021E000CE010E944310E8010E94B6678CE30E9472
:1021F000196181111EC00E947D6180913D209091E6
:102200003E20806190933E2080933D208E010F5FA1
:102210001F4F43E259E06CEB73E0CE010E94431084
:1022200085EF9EE09F938F930E9419940F900F90DB
:10223000E8010E94B66782ED0E941961811116C003
:102240000E947D6180913D2090913E20806290931C
:102250003E2080933D208E010F5F1F4F43E259E0E7
:1022600064EC73E0CE010E944310E8010E94B6675F
:1022700080E80E941961811116C00E947D618091E1
:102280003D2090913E20916090933E2080933D2090
:102290008E010F5F1F4F43E259E06DEC73E0CE01FA
:1022A0000E944310E8010E94B66780ED0E94196108
:1022B000811116C00E947D6180913D2090913E2049
:1022C000806890933E2080933D208E010F5F1F4FCA
:1022D00043E259E063ED73E0CE010E944310E80150
:1022E0000E94B6678CEE0E941961811116C00E948F
:1022F0007D6180913D2090913E20926090933E20A0
:1023000080933D208E010F5F1F4F43E259E06BED3C
:1023100073E0CE010E944310E80107E010E00E9444
:10232000B6678CE70E941961811113C00E947D611C
:1023300080913D2090913E20806490933E20809338
:102340003D2043E259E062EE73E0CE010E9443106B
:1023500005C0015011090115110509F70E947D61A1
:10236000DF91CF911F910F91FF900C94F20BCF93BF
:10237000DF9300D0CDB7DEB74A8369830E945461F2
:102380006981862F0E9485614A81842F0E94856120
:102390000F900F90DF91CF910C947D61AF92BF921F
:1023A000DF92EF92FF920F931F93CF93DF9300D0B2
:1023B0001F92CDB7DEB7182FD22E4A835B83698375
:1023C0000E9454616981862F0E948561812F8160FE
:1023D0000E947B614A81A42E5B81B52E00E010E053
:1023E000ED2CF12C81E0E81AF1080D1580F40E15A2
:1023F0001F0519F40E94A06102C00E949661F501B8
:1024000080830F5F1F4FFFEFAF1ABF0AEECF0F9011
:102410000F900F90DF91CF911F910F91FF90EF9050
:10242000DF90BF90AF900C947D61AF92BF92CF923E
:10243000DF92EF92FF920F931F93CF93DF93CDB76D
:10244000DEB760970FB6F894DEBF0FBECDBFB82ED3
:10245000A42E6623E9F18E010F5F1F4F80E1F80182
:1024600011928A95E9F728E0A80168E980EB0E94BB
:10247000CE11BB2041F02BEE33E03F932F930E940F
:1024800007940F900F906E01F8E0CF0ED11C52EF21
:10249000E52E53E0F52EF80181918F011F928F9365
:1024A000FF92EF920E9407940F900F900F900F9061
:1024B0000C151D0581F788851F928F9327E434E062
:1024C0003F932F930E9407940F900F900F900F90BF
:1024D000AA20E9F18E010F5F1F4F80E1F8011192F0
:1024E0008A95E9F728E0A80160E880EB0E94CE1108
:1024F000BB2041F087EF93E09F938F930E94079456
:102500000F900F906E01F0E1CF0ED11C42EFE42E40
:1025100043E0F42EF80181918F011F928F93FF9277
:10252000EF920E9407940F900F900F900F900C1550
:102530001D0581F788851F928F9387E494E09F9310
:102540008F930E9407940F900F900F900F906096BA
:102550000FB6F894DEBF0FBECDBFDF91CF911F91B4
:102560000F91FF90EF90DF90CF90BF90AF900895C4
:10257000CF93DF9300D0CDB7DEB71A82198222E065
:10258000AE014F5F5F4F6AEA8EEE0E94CE118981E5
:1025900090E0982F88272A81822B9093091C8093A2
:1025A000081C22E0AE014F5F5F4F6CEA8EEE0E9486
:1025B000CE11898190E0982F88272A81822B9093D1
:1025C0000B1C80930A1C22E0AE014F5F5F4F6EEA46
:1025D0008EEE0E94CE11898190E0982F88272A8163
:1025E000822B90930D1C80930C1C22E0AE014F5F58
:1025F0005F4F60EB8EEE0E94CE11898190E0982FA4
:1026000088272A81822B90931B1C80931A1C22E01E
:10261000AE014F5F5F4F62EB8EEE0E94CE1189815B
:1026200090E0982F88272A81822B90931D1C8093FD
:102630001C1C22E0AE014F5F5F4F64EB8EEE0E94E8
:10264000CE11898190E0982F88272A81822B909340
:102650001F1C80931E1C22E0AE014F5F5F4F66EB94
:102660008EEE0E94CE11898190E0982F88272A81D2
:10267000822B90930F1C80930E1C22E0AE014F5FC3
:102680005F4F68EB8EEE0E94CE11898190E0982F0B
:1026900088272A81822B9093111C8093101C22E0A2
:1026A000AE014F5F5F4F6AEB8EEE0E94CE118981C3
:1026B00090E0982F88272A81822B9093151C809375
:1026C000141C22E0AE014F5F5F4F6CEB8EEE0E9458
:1026D000CE11898190E0982F88272A81822B9093B0
:1026E000171C8093161C22E0AE014F5F5F4F6EEB0C
:1026F0008EEE0E94CE11898190E0982F88272A8142
:10270000822B9093191C8093181C0F900F90DF91CF
:10271000CF9108952F923F924F925F926F927F9246
:102720008F929F92AF92BF92CF92DF92EF92FF92E1
:102730000F931F93CF93DF93CDB7DEB76A970FB692
:10274000F894DEBF0FBECDBF182F488F298F198296
:102750001A821B8280912C1C811107C06A8F0E94F3
:10276000B81281E080932C1C6A8D662309F46CC03A
:102770004EE264EF8EEE0E94B71169E07AE180E0EC
:1027800090E00E94F76022E0AE014F5F5F4F66EF7E
:102790008EEE0E94CE112981822F90E0A0E0B0E061
:1027A0002227382F492F5A2F8A81282B80911E1CCF
:1027B00090911F1C281B390B41095109A0911C1C29
:1027C000B0911D1C0E94BC8D6B017C018FE0F594C3
:1027D000E794D794C7948A95D1F76091161C7091AD
:1027E000171C882777FD8095982F2BE0660F771FA1
:1027F000881F991F2A95D1F72091181C3091191C18
:10280000442737FD4095542F2C0D3D1D4E1D5F1D57
:102810000E94728DC20ED31ED092131CC092121C45
:1028200088E0C80ED11C34E0D594C7943A95E1F7FE
:10283000EE24D7FCE094FE2CC092201CD092211CE8
:10284000E092221CF092231C012F0295000F000F32
:10285000007C0C5CA12FB0E0BD8BAC8BA3E0B0E0A2
:10286000012E02C0AA0FBB1F0A94E2F725E335E050
:102870000E94B58DDC01CB010296A11DB11D8C8794
:102880009D87AE87BF8780E593ECA0E0B0E004C0F1
:10289000B595A795979587951A95D2F7888B998BBB
:1028A000AA8BBB8B10E0188619861A861B86A8E0B7
:1028B0002A2E312CAC89BD892A1A3B0A988D19170A
:1028C00009F436C1402F64EF8EEE0E94B7116C857B
:1028D0007D858E859F850E94F76023E0AE014F5F66
:1028E0005F4F66EF8EEE0E94CE11E091121CF091C8
:1028F000131CE05AFF409F01DF010E949E8D6B0177
:102900007C0180910A1C90910B1C9F8B8E8BA09058
:10291000081CB090091C20910C1C30910D1C0E94C9
:102920009E8D2B013C013DE075946794579447942C
:102930003A95D1F7A0910E1CB0910F1CA7019601FA
:102940006CE055954795379527956A95D1F70E9484
:10295000C78DBB2797FDB095AB2F480E591E6A1E39
:102960007B1E92E0490E511C611C711CB2E07594F3
:10297000679457944794BA95D1F7A0E85A0E611C12
:10298000711CA0911A1CB0911B1CA30192010E9402
:10299000BC8DDC01CB012FE0B695A7959795879567
:1029A0002A95D1F78C839D83AE83BF8329818A8149
:1029B00090E0A0E0B0E04424582E692E7A2E622ADE
:1029C0008B81482A022C04C07594679457944794CD
:1029D0000A94D2F74501AA2497FCA094BA2C42E0AD
:1029E000880C991CAA1CBB1C4A95D1F7A091101CFD
:1029F000B091111CA70196010E94C78D6B017C014B
:102A000057E1F594E794D794C7945A95D1F72E8956
:102A10003F89DF010E949E8DEBE095958795779524
:102A20006795EA95D1F7C60ED71EE81EF91E8C0CE5
:102A30009D1CAE1CBF1C0C8804C0880C991CAA1CD1
:102A4000BB1C0A94D2F792E0890E911CA11CB11C08
:102A5000F2E0B594A79497948794FA95D1F7481823
:102A600059086A087B08A3019201688979898A89D3
:102A70009B890E94188D97FD0DC0660F771F881FD8
:102A8000991F2C813D814E815F810E94508D4901AB
:102A90005A010CC02C813D814E815F810E94508D76
:102AA00049015A01880C991CAA1CBB1C9927B7FC28
:102AB0009A958B2D7A2D692D9B01AC010E94188D62
:102AC0009B01AC01AEEDBBE00E94BC8D6C01FF240C
:102AD000D7FCF094EF2CA3E4B3EEA50194010E947F
:102AE000CA8DBB2797FDB095AB2FC80ED91EEA1E25
:102AF000FB1EAFECCA0EAEE0DA1EE11CF11CA4E036
:102B0000F594E794D794C794AA95D1F7C80CD91C2B
:102B1000EA1CFB1C88859985AA85BB858C0D9D1DAB
:102B2000AE1DBF1D88879987AA87BB871F5FC6CE4A
:102B3000112391F0212F30E040E050E06885798545
:102B40008A859B850E94508D2093241C3093251CE0
:102B50004093261C5093271CA98DAA2389F16091CC
:102B6000241C7091251C8091261C9091271C6115B6
:102B700071058105910521F10E94768A20E836EEE3
:102B800045EC57E40E94D78921E03EED42E45EE344
:102B90000E94BB8C9B01AC0160E070E080E89FE389
:102BA0000E940C892BE43AE34DEB57E30E94D7894E
:102BB0006093281C7093291C80932A1C90932B1CD3
:102BC0006A960FB6F894DEBF0FBECDBFDF91CF91EE
:102BD0001F910F91FF90EF90DF90CF90BF90AF903B
:102BE0009F908F907F906F905F904F903F902F902D
:102BF00008950F931F93CF93DF9300D000D000D0A0
:102C0000CDB7DEB78E010F5F1F4F86E0F80111923E
:102C10008A95E9F780911E1B811113C040E061E3A2
:102C200086EA0E94B7114AE06CE286EA0E94B71178
:102C300081E080931E1B6CE77EE380E090E00E94C1
:102C4000F76048E06DE286EA0E94B7116CE77EE328
:102C500080E090E00E94F76026E0A80162E386EA47
:102C60000E94CE1147E06DE286EA0E94B7118A8188
:102C700090E0982F88272981822B9093191B8093AD
:102C8000181B2C8130E0322F22274B81242B3093CC
:102C90001B1B20931A1B4E8150E0542F44276D813B
:102CA000462B50931D1B40931C1B5F934F933F93E8
:102CB0002F939F938F938BEF93E09F938F930E941B
:102CC00007940FB6F894DEBF0FBECDBF26960FB6A1
:102CD000F894DEBF0FBECDBFDF91CF911F910F9152
:102CE0000895CF92DF92EF92FF920F931F93CF93AD
:102CF000DF93CDB7DEB72A970FB6F894DEBF0FBECD
:102D0000CDBF8E010F5F1F4F86E0F80111928A95AB
:102D1000E9F741E062E08CE30E94B71148E560E02A
:102D20008CE30E94B71162E174E380E090E00E94BE
:102D3000F76026E0A80163E08CE30E94CE1143E037
:102D400062E08CE30E94B711098110E0102F002788
:102D50008A81082B1093F91A0093F81AEB80F12C52
:102D6000FE2CEE248C81E82AF092FB1AE092FA1AEB
:102D7000CD80D12CDC2CCC248E81C82AD092FD1A97
:102D8000C092FC1AB801882777FD8095982F0E9481
:102D9000768A9B01AC01B701882777FD8095982F33
:102DA0002F83388749875A870E94768A2F813885F2
:102DB00049855A850E94808920EE3EE245E652E42C
:102DC0000E94588C20E030E044E353E40E940D89D7
:102DD0009F938F937F936F93DF92CF92FF92EF92A7
:102DE0001F930F9389E094E09F938F930E94079421
:102DF0000FB6F894DEBF0FBECDBF2A960FB6F8947B
:102E0000DEBF0FBECDBFDF91CF911F910F91FF901D
:102E1000EF90DF90CF900895CF93DF93EC018881FE
:102E200099810097F9F0833D904121F01982188231
:102E300083E063C085ED99E00E944958892BE1F059
:102E40008091C5099091C60993FD18C08091C5096C
:102E50009091C60994FD43C08091C5099091C6091F
:102E600095FD44C060E870E085ED99E00E9422582D
:102E700083ED90E19983888381E03FC080913D207C
:102E800082FFE4CF21E048E061E083E00E948A1302
:102E900080912B1C8F9380912A1C8F938091291CE9
:102EA0008F938091281C8F938091271C8F93809102
:102EB000261C8F938091251C8F938091241C8F93C7
:102EC00084E59FE09F938F930E9419948DB79EB7DE
:102ED0000A960FB6F8949EBF0FBE8DBFB7CF8091F4
:102EE0003D2083FFB9CF0E94F915B6CF80913D20D8
:102EF00084FFB8CF0E947116B5CFDF91CF910895AE
:102F0000CF93C82F8CEE0E947B618C2F0E9485612D
:102F100065E375E080E090E00E94F7608DEE0E942E
:102F20007B610E949661C82F0E94A0612C2F30E027
:102F3000322F2227A901482BCA01CF910895CF93A0
:102F4000DF93C82F8CEE0E947B618C2F0E948561DD
:102F500062E174E380E090E00E94F7608CEE0E94F2
:102F60007B6180E00E94856165E375E080E090E030
:102F70000E94F7608DEE0E947B610E949661C82FCF
:102F80000E949661D82F0E94A0614D2F50E060E012
:102F900070E0762F652F542F44276C2B482BCB01E4
:102FA000BA01DF91CF9108952F923F924F925F9295
:102FB0006F927F928F929F92AF92BF92CF92DF9249
:102FC000EF92FF920F931F93CF93DF93CDB7DEB7AE
:102FD000CD54D1090FB6F894DEBF0FBECDBF80919E
:102FE000000290910102892BD1F1109201021092FE
:102FF00000028CEE0E947B618EE10E9485616BE194
:103000007EE480E090E00E94F76082EA0E948017F0
:103010009093D2098093D10984EA0E9480179093FB
:10302000D0098093CF0986EA0E9480179093CE0939
:103030008093CD0988EA0E9480179093CC098093F1
:10304000CB098AEA0E9480179093CA098093C90924
:103050008CEA0E9480179093C8098093C70988E47E
:103060000E949F176FAB78AF89AF9AAF88E50E9437
:103070009F174B015C018091C9099091CA0920E01A
:1030800030E040E050E0BA0126962FAF2697279611
:103090003FAF279728964FAF289729965FAF29977C
:1030A0002A966FAF2A972B967FAF2B979C0140E013
:1030B00050E060E070E080E090E008E00E942A8F3D
:1030C0000E94E38E3901B42FA52FF62FE72F8C0134
:1030D0009401A50160E070E080E090E05301CB2E08
:1030E000DA2EEF2EFE2E0E94618F29833A832A0169
:1030F0001B014C01B101C401315041095F4F6F4FB9
:103100007F4F8F4F9F4FA1E0B0E02596BFAFAEAF8E
:10311000259721153F4F4F4F51406105710581059E
:10312000910509F020F425961FAE1EAE2597259631
:103130006EAC7FAC25978091C7099091C8095C015E
:10314000C12CD12CE12CF12C00E010E029813A8136
:10315000A201B101C4010E94CF8DD22EE32EF42E24
:10316000052F162FB72FF82FE92FA0E00E94888F88
:1031700084F42150310940485F4F6F4F7F4F8F4F8C
:103180009F4FD22EE32EF42E052F162FB72FF82F98
:10319000E92F2D2D3E2D4F2D502F612F7B2F8F2F5F
:1031A0009E2F07E10E94438F2B8F3C8F4D8F5E8FA8
:1031B0006F8F78A389A39AA32053384F4F4F5F4F47
:1031C0006F4F7F4F8F4F9F4F2B8B3C8B4D8B5E8B69
:1031D0006F8B788F898F9A8F2056304F4F4F5F4F6C
:1031E0006F4F7F4F8F4F9F4F243D30434105510517
:1031F000610571058105910541F038F025966EACA9
:103200007FAC2597FFEF6F1A7F0A8091CF099091CD
:10321000D0099C0140E050E060E070E080E090E088
:1032200000E10E942A8F2B833C834D835E836A8753
:1032300079878F8398874091CB095091CC09A980D9
:10324000BA806201710184019A0140E050E060E0BF
:1032500070E080E090E00E94CF8DD22EE32EF42E1D
:10326000052F162FB72FF82FE92FA0E00E94888F87
:103270005CF4AFE70E946A8FD22EE32EF42E052F66
:10328000162FB72FF82FE92F2D2D3E2D4F2D502F14
:10329000612F7B2F8F2F9E2F07E00E94438F5901B4
:1032A0006A017B018C012B813C814D815E816A85A5
:1032B00079858F8198850E94618F2B833C834D8314
:1032C0005E836F8378878F87988B2E5F3F4F434055
:1032D00051096E4F7F4F8F4F9F4F22303105494F1D
:1032E0005F4F644071058105910521F018F01FEFD3
:1032F000611A710A8091D1099091D209BC0180E0D4
:1033000090E020E030E840E050E00E94288E2987DD
:103310003A874B875C876A8B798B8D879E87409134
:10332000CD095091CE09A980BA8062017101840152
:103330009A0140E050E060E070E080E090E00E94A0
:10334000CF8DD22EE32EF42E052F162FB72FF82F68
:10335000E92FA0E00E94888F84F421503F4F4F4F07
:103360005F4F6F4F7F4F8F4F9F4FD22EE32EF42E24
:10337000052F162FB72FF82FE92F2D2D3E2D4F2D6E
:10338000502F612F7B2F8F2F9E2F08E00E94438F9D
:1033900059016A017B018C0129853A854B855C8541
:1033A0006A8979898D859E850E94618F29873A87F0
:1033B0004B875C876D877E87898B9A8B2F5F3F4F0A
:1033C0004140510961097109810991092130304851
:1033D0004C4F5F47614071058105910521F018F060
:1033E000BFEF6B1A7B0A2B893C894D895E896F89F7
:1033F000788D898D9A8D2F3C3740410551056105A7
:1034000071058105910511F00CF0A5C1A980BA8064
:103410006201710184019501A201B101C4010E9400
:10342000CF8DA12CB12CC12C10E8D12EE12CF12C88
:1034300000E010E00E94558E2BAF3CAF4DAF5EAF69
:103440006FAF21967FAF219722968FAF2297239659
:103450009FAF2397AB8CBC8CCD8CDE8CEF8CF8A00F
:1034600009A11AA19501A601B701C8010E94CF8D3B
:1034700059016A017B01E82F192F02E00E942A8F6F
:103480000E2F0E94618F69017A01162F272EF82FC7
:10349000E92F322E8D2C942EAF2CB62E072F582EBE
:1034A000B92FA0E00E94888F5CF4A1E00E946A8F8F
:1034B000322E832E942EA52EB62E072F582EB92FDE
:1034C000232D382D492D5A2D6B2D702F852D9B2F97
:1034D00001E00E94438F2E962FAF2E972D963FAF7F
:1034E0002D9749A75AA76BA77CA78DA79EA7522EF9
:1034F000432E4BA35CA36DA37EA38FA398A7B22DED
:103500009601A701612F722D8F2F9E2FA0E00E94A0
:10351000888F4CF4A3E00E946A8F69017A01162F0C
:10352000B72FF82FE92F9601A701612F7B2F8F2F3F
:103530009E2F02E00E94438F2FA738AB49AB5AABB6
:103540006BAB7CAB8DAB9EAB19014A01B62FA72F9D
:1035500024968FAF2497F92F2B893C894D895E895A
:103560006F89788D898D9A8D24323A4F4F4F5F4FF6
:103570006F4F7F4F8F4F9F4F0CF08CC02B8D3C8D2A
:103580004D8D5E8D6F8D78A189A19AA12455324F02
:103590004F4F5F4F6F4F7F4F8F4F9F4F59016A01C2
:1035A0007B018C010E94CF8D19014A01B62FA72FF4
:1035B000FC0103E00E942A8F51016401EB2EFA2ED8
:1035C0008F010E94768F59016A017B018C012E9632
:1035D0002FAD2E972D963FAD2D9749A55AA56BA5DA
:1035E0007CA58DA59EA50E94618F522E432E4BA3D4
:1035F0005CA36DA37EA38FA398A79101A4016B2F59
:103600007A2FCF0102E00E942A8F51016401EB2E34
:10361000FA2E8F010E94768F02E00E942A8F0E2FD1
:103620000E94768FF22E032F142FD52EE62EB72F61
:10363000F82FE92FA0E00E94888F5CF4A1E00E949F
:103640006A8FF22E032F142FD52EE62EB72FF82FC8
:10365000E92F2F2D302F412F5D2D6E2D7B2F8F2F9A
:103660009E2F01E00E94438F59016A017B018C016A
:103670002FA538A949A95AA96BA97CA98DA99EA9EA
:103680000E94618F19014A01B62FA72F24968FAF90
:103690002497F92F2B813C814D815E816F81788544
:1036A0008F859889A52CB42CCBA0DCA0EDA0FEA022
:1036B0000FA118A50E94768F2B833C834D835E83D8
:1036C0006F8378878F87988B29853A854B855C85B2
:1036D0006D857E8589899A8951016401EB2EFA2EC8
:1036E00024960FAD24971F2F0E94768F29873A8743
:1036F0004B875C876D877E87898B9A8B2B893C896A
:103700004D895E896F89788D898D9A8DABACBCAC03
:10371000CDACDEACEFAC2196FFAC219722960FAD7D
:10372000229723961FAD23970E94768F2056304F05
:103730004F4F5F4F6F4F7F4F8F4F9F4F243D304311
:1037400041055105610571058105910521F018F0CC
:103750002FEF621A720A6FA978AD89AD9AADAB01ED
:10376000BC0180E090E0DC0124964FAF24972596C1
:103770005FAF259726966FAF269727967FAF27973F
:1037800028968FAF289729969FAF29972A96AFAF93
:103790002A972B96BFAF2B97A984BA84CB84DC845D
:1037A000ED84FE8409891A899A01AB0160E070E01A
:1037B00080E090E00E94CF8DF22E032F142FD52EA3
:1037C000E62EB72FF82FE92FA0E00E94888F84F40F
:1037D00021503109404E5F4F6F4F7F4F8F4F9F4FAA
:1037E000F22E032F142FD52EE62EB72FF82FE92F08
:1037F0002F2D302F412F5D2D6E2D7B2F8F2F9E2F44
:1038000005E10E94438FAB80BC80CD80DE80EF80DD
:10381000F8840F8518890E94768FF22E032F142FBB
:10382000D52EE62EB72FF82FE92FA0E00E94888F23
:1038300084F4215030484F4F5F4F6F4F7F4F8F4F71
:103840009F4FF22E032F142FD52EE62EB72FF82FD1
:10385000E92F2F2D302F412F5D2D6E2D7B2F8F2F98
:103860009E2F0FE00E94438F69017A018B018A83AA
:10387000998329011A014B015C01285E33404109FB
:1038800051096109710981099109283D304D414073
:103890005105610571058105910521F018F0BFEF13
:1038A0006B1A7B0A0E947D61672859F09601A70177
:1038B000B8018A8199810E94E38E29011A014B0186
:1038C0005C019201A101B401C5010E94708A20E04F
:1038D00030E048EC52E40E94D789C35BDF4F0FB65B
:1038E000F894DEBF0FBECDBFDF91CF911F910F9136
:1038F000FF90EF90DF90CF90BF90AF909F908F9010
:103900007F906F905F904F903F902F9008954F92CF
:103910005F926F927F928F929F92AF92BF92CF925F
:10392000DF92EF92FF922B013C0169017A0123ECB7
:1039300035EF4CE851E4C701B6010E94588C4B01A9
:103940005C0128EB3EE143E753E4C701B6010E9466
:103950000D899B01AC01C501B4010E94D7890E9469
:10396000448A4B015C0120E030E048EC52E4C301A2
:10397000B2010E94D78921E835E943EC50E40E9466
:10398000588CA50194010E94588C4B015C0123E3E3
:1039900033E948E853E4C701B6010E940D899B0151
:1039A000AC01C501B4010E94D78923E333EB48E59C
:1039B00053E40E94588CFF90EF90DF90CF90BF901F
:1039C000AF909F908F907F906F905F904F900895F1
:1039D0004F925F926F927F928F929F92AF92BF921F
:1039E000CF92DF92EF92FF9269017A010E94DA8B07
:1039F00020E030E040E050E40E940C8922E93CE500
:103A00004EED5EE30E94D7894B015C0123EC35EF5C
:103A10004CE851E4C701B6010E94588C2B013C01CF
:103A200028EB3EE143E753E4C701B6010E940D894C
:103A30009B01AC01C301B2010E94D7899B01AC017B
:103A4000C501B4010E940D896B017C0128EB3EE1A8
:103A500043E753E40E94588C4B015C01A701960197
:103A600063EC75EF8CE891E40E940C899B01AC013A
:103A7000C501B4010E94D789FF90EF90DF90CF90ED
:103A8000BF90AF909F908F907F906F905F904F907E
:103A900008954F925F926F927F928F929F92AF9212
:103AA000BF92CF92DF92EF92FF922B013C0169010E
:103AB0007A0123EC35EF4CE851E4C701B6010E94CE
:103AC000588C4B015C0128EB3EE143E753E4C7010E
:103AD000B6010E940D899B01AC01C501B4010E9491
:103AE000D7890E94448A4B015C0120E030E048EC19
:103AF00052E4C301B2010E94D789A50194010E943A
:103B0000588C20E030E040E251E40E940C8924EE21
:103B100038E34EE05FE30E94588C9B01AC01C70183
:103B2000B6010E940D89FF90EF90DF90CF90BF907B
:103B3000AF909F908F907F906F905F904F9008957F
:103B400080E80E947B6181110DC08EEF0E9485612B
:103B5000811108C06BE17EE480E090E00E94F76094
:103B60000C947D610E947D6180914F24909150243E
:103B7000A0915124B09152240196A11DB11D8093B2
:103B80004F2490935024A0935124B093522408952D
:103B9000FC01DC0182E020E041E39D91292798E0CF
:103BA000322F330F27FF03C0232F242701C0232FD9
:103BB0009150B1F7815089F781E090E0328123176D
:103BC00011F080E090E00895DF92EF92FF920F9362
:103BD0001F93CF93DF930E94A01D80E80E947B611A
:103BE00081116DC08AEF0E948561811168C08FE0EC
:103BF0000E948561811163C065E375E080E090E01B
:103C00000E94F76081E80E947B61811158C00E9488
:103C10009661C82F0E9496610E949661D82F0E94DB
:103C200096610E949661182F0E9496610E94A06181
:103C3000082F80E80E947B61811141C08CEF0E94B7
:103C4000856181113CC089EC0E948561811137C07A
:103C500065E375E080E090E00E94F76081E80E94F3
:103C60007B610E949661E82E0E949661D82E0E9488
:103C700096610E949661F82E0E94A0611F92DF92C9
:103C80001F92EF921F920F931F921F931F92DF9329
:103C90001F92CF931F928F931F92FF928EE194E019
:103CA0009F938F930E9407940E947D618DB79EB76A
:103CB00042960FB6F8949EBF0FBE8DBF17C00E94EC
:103CC0007D6180914F2490915024A0915124B09116
:103CD00052240196A11DB11D80934F24909350242E
:103CE000A0935124B09352240E94A01D20E030E004
:103CF00040E050E060E070E080E090E0DF91CF9144
:103D00001F910F91FF90EF90DF900895EF92FF9237
:103D10000F931F93CF93DF9300D01F92CDB7DEB7E1
:103D20008C0180E80E947B61811154C0011511054E
:103D300051F085EE0E94856181114CC061E077E908
:103D400080E090E009C083EE0E948561811142C04D
:103D500069E97AEB81E090E00E94F76081E80E94D7
:103D60007B61811137C00E949661F82E89830E9481
:103D70009661E82E8A830E94A0618B830E947D61F8
:103D8000CE0101960E94C81D892B21F16E2D70E095
:103D90007F296C7F80E090E0012B69F00E94748A9B
:103DA00020E030E04AEF5AE30E94588C20E030E0F7
:103DB00040EC50E40CC00E94748A22E538EB4FE2DC
:103DC0005BE30E94588C26E636E64BE352E40E9401
:103DD0000C891BC00E947D6180914F2490915024DA
:103DE000A0915124B09152240196A11DB11D809340
:103DF0004F2490935024A0935124B09352240E94B6
:103E0000A01D60EF7FEF89E794E40F900F900F9073
:103E1000DF91CF911F910F91FF90EF9008950F9335
:103E20001F93CF93DF93729A8091580283FF08C04B
:103E30008EE40E941961811167C0C0E5D0E00AC01C
:103E4000C0E5D0E087EE93E00E948C09219720978F
:103E5000C9F7EECF87EE93E00E948C092197209757
:103E6000C9F78FE40E9419610E949661082F0F73B1
:103E70000E949661182F0E949661D82F0E94A0611F
:103E8000C82F0E947D618091580283FF7298602F35
:103E900070E0762F6627610F711D80E090E00E9430
:103EA000748A20E134E048EC5BE30E94588C609314
:103EB000311C7093321C8093331C9093341C6D2FF3
:103EC00070E0762F66276C0F711D76956795769555
:103ED000679580E090E00E94748A24EA3CEF44E217
:103EE0005CE30E94588C20E030E040E252E40E9403
:103EF0000C8960930E2970930F2980931029909359
:103F0000112980E090E002C081E090E0DF91CF9144
:103F10001F910F9108957298729A8EE40E94196110
:103F200080EA0E94856180E00E94856180E00E94B5
:103F300085618FE40E9419610E9496618EE40E945F
:103F4000196180E80E94856180E00E94856180E0BF
:103F50000E9485610E947D6180E090E0089588EE76
:103F60009EE09F938F930E941994809173020F900B
:103F70000F90882361F01F928F9385EE9EE09F93B0
:103F80008F930E9419940F900F900F900F900895A7
:103F900080EC9EE09F938F930E94199488E99EE0A5
:103FA0009F938F930E94199481E79EE09F938F9334
:103FB0000E94199486E39EE09F938F930E94199428
:103FC00084E09EE09F938F930E94199488EC9DE07B
:103FD0009F938F930E94199482EA9DE09F938F9301
:103FE0000E9419948CE69DE09F938F930E941994F0
:103FF00080913D2090913E20827091702DB73EB708
:10400000205F3F4F0FB6F8943EBF0FBE2DBF892BE8
:1040100041F08CE39DE09F938F930E9419940F9041
:104020000F9080E19DE09F938F930E94199484EDFF
:104030009CE09F938F930E9419948BEA9CE09F933E
:104040008F930E9419948FE79CE09F938F930E9417
:10405000199480E59CE09F938F930E9419948EE1C0
:104060009CE09F938F930E9419948DEE9BE09F9309
:104070008F930E94199483EB9BE09F938F930E94F0
:1040800019948DE79BE09F938F930E9419948DE480
:104090009BE09F938F930E94199481E29BE09F93F2
:1040A0008F930E94199482EF9AE09F938F930E94BE
:1040B000199489EB9AE09F938F930E94199480E85A
:1040C0009AE09F938F930E94199489E49AE09F93BA
:1040D0008F930E94199485E19AE09F938F930E9499
:1040E00019948DB79EB780960FB6F8949EBF0FBEF9
:1040F0008DBF84EE99E09F938F930E94199485EB76
:1041000099E09F938F930E94199486E899E09F937A
:104110008F930E9419948FE599E09F938F930E944B
:10412000199489E299E09F938F930E94199483EFE9
:1041300098E09F938F930E9419948DEB98E09F9342
:104140008F930E94199484E998E09F938F930E9423
:1041500019948CE598E09F938F930E94199481E3C2
:1041600098E09F938F930E9419942DB73EB72C5ED1
:104170003F4F0FB6F8943EBF0FBE2DBF08958DE49C
:1041800094E00C943D944F925F926F927F928F9245
:104190009F92AF92BF92CF92DF92EF92FF92CF9316
:1041A000DF93CDB7DEB728970FB6F894DEBF0FBE0A
:1041B000CDBF8091432490914424A0914524B09197
:1041C000462489839A83AB83BC83409043245090D8
:1041D000442460904524709046248091432490911B
:1041E0004424A0914524B09146248D839E83AF83BF
:1041F000B887609143247091442480914524909124
:1042000046242CE3822E912CA12CB12CA5019401E3
:104210000E94508D7F936F9330E1C32E3EE0D32EEA
:10422000E12CF12C6D817E818F819885A70196010B
:104230000E94508DA50194010E94508D3F932F93B1
:1042400040E8842E41E5942EAA24A394B12CC30106
:10425000B201A50194010E94508DA70196010E9410
:10426000508D3F932F9369817A818B819C81A50129
:1042700094010E94508D3F932F938BE098E09F9381
:104280008F930E9419940FB6F894DEBF0FBECDBF76
:1042900028960FB6F894DEBF0FBECDBFDF91CF9149
:1042A000FF90EF90DF90CF90BF90AF909F908F9056
:1042B0007F906F905F904F900895E3EDF1E38081E0
:1042C00091818234924479F0E35DF143FF93EF935F
:1042D0008DEE97E09F938F930E9419940F900F900B
:1042E0000F900F9008953A96E53F81E4F80738F370
:1042F0000895CF93DF93EC018C9A0E94D70A9F9385
:104300008F937F936F9381EE97E09F938F930E949B
:1043100019940F900F900F900F900F900F9020977F
:1043200019F00E94F20B08C08FED97E09F938F93D6
:104330000E9419940F900F9081E00E94880A2091AA
:1043400078023091790240917A0250917B020E946A
:10435000588C9F938F937F936F9383ED97E09F93F8
:104360008F930E9419940F900F900F900F900F90C1
:104370000F90209719F00E94F20B08C081ED97E092
:104380009F938F930E9419940F900F9082E00E9448
:10439000880A209174023091750240917602509102
:1043A00077020E94588C9F938F937F936F9385EC35
:1043B00097E09F938F930E9419940F900F900F9006
:1043C0000F900F900F90209719F00E94F20B08C0E9
:1043D00083EC97E09F938F930E9419940F900F9016
:1043E00083E00E94880A9F938F937F936F9384EB5F
:1043F00097E09F938F930E9419948C980F900F9041
:104400000F900F900F900F90209719F00E94F20BD1
:1044100008C082EB97E09F938F930E9419940F90AE
:104420000F9080913D2087FF83C021E042E161E051
:1044300080ED0E94DD629F938F937F936F9385EA57
:1044400097E09F938F930E9419940F900F900F9075
:104450000F900F900F90209719F00E94F20B08C058
:1044600083EA97E09F938F930E9419940F900F9087
:1044700021E042E162E080ED0E94DD629F938F9334
:104480007F936F9386E997E09F938F930E9419948F
:104490000F900F900F900F900F900F90209719F0A2
:1044A0000E94F20B08C084E997E09F938F930E94CB
:1044B00019940F900F9021E042E163E080ED0E949B
:1044C000DD629F938F937F936F9387E897E09F932D
:1044D0008F930E9419940F900F900F900F900F9050
:1044E0000F90CD2B19F00E94F20B08C085E897E0E1
:1044F0009F938F930E9419940F900F9021E042E1B7
:1045000064E080ED0E94DD629F938F937F936F93B1
:1045100088E797E09F938F930E9419940F900F90D4
:104520000F900F900F900F90DF91CF910C94F20BA2
:10453000CD2BD1F3DF91CF9108950F931F93CF939C
:10454000DF93882389F049E050E06FEF70E082E06C
:1045500099E20E945B9349E050E06AE070E082E0FB
:1045600099E20E948B9513C0C2E0D9E203E717E0FD
:1045700089911F928F931F930F930E9419940F900C
:104580000F900F900F9089E2CA30D80789F7DF911A
:10459000CF911F910F910C94F20B882311F02A9A5E
:1045A00008952A980895882311F02B9A08952B983E
:1045B0000895CF92DF92EF92FF92CF93DF936B013A
:1045C0007C0160FF11C08AE894E09F938F938DEF88
:1045D0009EE09F938F930E9419940F900F900F90DD
:1045E0000F9081E090E002C080E090E0C1FE09C041
:1045F000EC01219643E259E06FE874E00E94431019
:10460000CE01C2FE09C0EC01219643E259E067E900
:1046100074E00E944310CE01C3FE09C0EC01219654
:1046200043E259E06FE974E00E944310CE01C4FEFA
:1046300009C0EC01219643E259E063EA74E00E946C
:104640004310CE01C5FE09C0EC01219643E259E0BA
:1046500066EA74E00E944310CE01C6FE09C0EC0178
:10466000219643E259E06AEA74E00E944310CE01C9
:10467000C7FE09C0EC01219643E259E060EB74E00B
:104680000E944310CE01D0FE09C0EC01219643E206
:1046900059E068EB74E00E944310CE01D1FE09C0DE
:1046A000EC01219643E259E060EC74E00E94431073
:1046B000CE01D2FE09C0EC01219643E259E064EC40
:1046C00074E00E944310CE0120913D2030913E20A5
:1046D00024703270232B59F0D3FE09C0EC012196CF
:1046E00043E259E06AEC74E00E944310CE0120914D
:1046F0003D2023FF0BC0D4FE09C0EC01219643E20C
:1047000059E06FEC74E00E944310CE0120913D20EF
:1047100024FF0BC0D5FE09C0EC01219643E259E00D
:1047200065ED74E00E944310CE01D6FE09C0EC0195
:10473000219643E259E06DED74E00E944310CE01F2
:10474000B701A60144275078452B462B472B61F033
:1047500043E259E068EE74E0DF91CF91FF90EF9073
:10476000DF90CF900C944310CD28CE28CF2841F471
:104770008EE697E09F938F930E9419940F900F906D
:10478000DF91CF91FF90EF90DF90CF9008950F933E
:104790001F93CF93DF938C01C0E0D0E0011511058A
:1047A00009F48AC069E677E0C8010E943A93892B30
:1047B00009F4C16061E677E0C8010E943A93892B51
:1047C00009F4C26069E577E0C8010E943A93892B39
:1047D00009F4C46065E577E0C8010E943A93892B2B
:1047E00009F4C86062E577E0C8010E943A93892B1A
:1047F00009F4C0616EE477E0C8010E943A93892B06
:1048000009F4C06268E477E0C8010E943A93892BFA
:1048100009F4C06460E477E0C8010E943A93892BF0
:1048200009F4C06868E377E0C8010E943A93892BD5
:1048300009F4D16064E377E0C8010E943A93892BC0
:1048400009F4D2606EE277E0C8010E943A93892BA6
:1048500009F4D46069E277E0C8010E943A93892B99
:1048600009F4D86063E277E0C8010E943A93892B8B
:1048700009F4D0616BE177E0C8010E943A93892B7B
:1048800009F4D06260E177E0C8010E943A93892B75
:1048900009F4D0646FEF76E0C8010E943A93892B47
:1048A00009F4D068609171027091720280E090E02A
:1048B0000E944E938C0172CFCE01DF91CF911F9158
:1048C0000F910895AF92BF92CF92DF92EF92FF9235
:1048D0000F931F93CF93DF93F22E032F142FE52E08
:1048E000D62EA72EB82EC92E217030E040E050E021
:1048F00060E070E080E090E0A0E00E94888F89F0A6
:10490000E9EFF4E0FF93EF93EDEFFEE0FF93EF9319
:104910000E9419940F900F900F900F90E1E0F0E03B
:1049200002C0E0E0F0E080913D2080FF17C02F2D15
:10493000247030E040E050E060E070E080E090E023
:10494000A0E00E94888F51F0EF01219643E259E0E8
:104950006DEF74E0CF010E944310FE012F2D2270F5
:1049600030E040E050E060E070E080E090E0A0E007
:104970000E94888F51F0EF01219643E259E061E0F7
:1049800075E0CF010E944310FE012F2D287030E00A
:1049900040E050E060E070E080E090E0A0E00E9445
:1049A000888F51F0EF01219643E259E069E175E00B
:1049B000CF010E944310FE012F2D207130E040E016
:1049C00050E060E070E080E090E0A0E00E94888F1E
:1049D00051F0EF01219643E259E064E075E0CF0128
:1049E0000E944310FE012F2D207230E040E050E085
:1049F00060E070E080E090E0A0E00E94888F51F0DD
:104A0000EF01219643E259E067E075E0CF010E9493
:104A10004310FE012F2D207430E040E050E060E0B4
:104A200070E080E090E0A0E00E94888F51F0EF01FC
:104A3000219643E259E06DE075E0CF010E944310FA
:104A4000FE012F2D207830E040E050E060E070E083
:104A500080E090E0A0E00E94888F51F0EF01219665
:104A600043E259E063E175E0CF010E944310FE018B
:104A700020E0302F317040E050E060E070E080E0F6
:104A800090E0A0E00E94888F51F0EF01219643E270
:104A900059E066E175E0CF010E944310FE0120E07D
:104AA000302F327040E050E060E070E080E090E055
:104AB000A0E00E94888F51F0EF01219643E259E077
:104AC0006BE175E0CF010E944310FE0120E0302F22
:104AD000347040E050E060E070E080E090E0A0E002
:104AE0000E94888F51F0EF01219643E259E062E283
:104AF00075E0CF010E944310FE0120E0302F387096
:104B000040E050E060E070E080E090E0A0E00E94D3
:104B1000888F51F0EF01219643E259E065E275E09C
:104B2000CF010E944310FE0120E0302F307140E0A1
:104B300050E060E070E080E090E0A0E00E94888FAC
:104B400051F0EF01219643E259E06AE275E0CF01AE
:104B50000E944310FE0120E0302F307240E050E010
:104B600060E070E080E090E0A0E00E94888F51F06B
:104B7000EF01219643E259E061E375E0CF010E9425
:104B80004310FE0120E030E040E050E06D2D647005
:104B900070E080E090E0A0E00E94888F51F0EF018B
:104BA000219643E259E068E375E0CF010E9443108B
:104BB000FE0180913D2081FF17C020E0302F30742E
:104BC00040E050E060E070E080E090E0A0E00E9413
:104BD000888F51F0EF01219643E259E06CE375E0D4
:104BE000CF010E944310FE0180913D2090913E2014
:104BF00090FF17C020E030E040E05E2D507160E093
:104C000070E080E090E0A0E00E94888F51F0EF011A
:104C1000219643E259E06FE375E0CF010E94431013
:104C2000FE0180913D2090913E2090FF17C020E032
:104C300030E040E05E2D507260E070E080E090E097
:104C4000A0E00E94888F51F0EF01219643E259E0E5
:104C500062E475E0CF010E944310FE0180913D2087
:104C600090913E2090FF17C020E030E040E05E2DA4
:104C7000507460E070E080E090E0A0E00E94888FD7
:104C800051F0EF01219643E259E068E475E0CF016D
:104C90000E944310FE0120E0302F307840E050E0C9
:104CA00060E070E080E090E0A0E00E94888F51F02A
:104CB000EF01219643E259E063E575E0CF010E94E0
:104CC0004310FE0120E030E0412F417050E060E0F1
:104CD00070E080E090E0A0E00E94888F51F0EF014A
:104CE000219643E259E068E575E0CF010E94431048
:104CF000FE0120E030E0412F427050E060E070E0C3
:104D000080E090E0A0E00E94888F51F0EF012196B2
:104D100043E259E06BE575E0CF010E944310FE01CC
:104D200020E030E0412F447050E060E070E080E02F
:104D300090E0A0E00E94888F51F0EF01219643E2BD
:104D400059E06EE575E0CF010E944310FE018091AD
:104D50003D2087FF17C020E030E0412F487050E031
:104D600060E070E080E090E0A0E00E94888F51F069
:104D7000EF01219643E259E061E675E0CF010E9420
:104D80004310FE0180913D2087FF17C020E030E0F6
:104D9000412F407150E060E070E080E090E0A0E0E2
:104DA0000E94888F51F0EF01219643E259E065E6B9
:104DB00075E0CF010E944310FE0180913D2087FFE6
:104DC00017C020E030E0412F407250E060E070E01A
:104DD00080E090E0A0E00E94888F51F0EF012196E2
:104DE00043E259E069E675E0CF010E944310FE01FD
:104DF00080913D2087FF17C020E030E0412F4074B4
:104E000050E060E070E080E090E0A0E00E94888FD9
:104E100051F0EF01219643E259E06DE675E0CF01D4
:104E20000E944310FE0180913D2082FF17C020E0C8
:104E300030E0412F407850E060E070E080E090E0AA
:104E4000A0E00E94888F51F0EF01219643E259E0E3
:104E50006DE376E0CF010E944310FE0180913D207A
:104E600082FF17C020E030E040E05E2D517060E02E
:104E700070E080E090E0A0E00E94888F51F0EF01A8
:104E8000219643E259E061E775E0CF010E944310AB
:104E9000FE0180913D2090913E2090FF17C020E0C0
:104EA00030E040E05E2D527060E070E080E090E025
:104EB000A0E00E94888F51F0EF01219643E259E073
:104EC00064E775E0CF010E944310FE0180913D2010
:104ED00090913E2090FF17C020E030E040E05E2D32
:104EE000547060E070E080E090E0A0E00E94888F65
:104EF00051F0EF01219643E259E06CE775E0CF01F4
:104F00000E944310FE0180913D2090913E2091FF30
:104F10001EC020E030E040E05E2D587060E070E0A0
:104F200080E090E0A0E00E94888F89F043E259E0A1
:104F300065E875E0CF01DF91CF911F910F91FF9050
:104F4000EF90DF90CF90BF90AF900C9443102F2D37
:104F5000302F412F5E2D6D2D7A2D8B2D9C2DA0E0B5
:104F60000E94888F41F48AEF96E09F938F930E946E
:104F700019940F900F90DF91CF911F910F91FF9097
:104F8000EF90DF90CF90BF90AF9008958F929F9257
:104F9000BF92DF92EF920F931F93CF93DF93EC01B9
:104FA0004B01FB01108265EF76E00E943A93892B5A
:104FB00061F580913D207DE4D72EE0E8EE2E82FD64
:104FC00002C004E001C004E810E0B12C81FF02C07F
:104FD00060ECE62E26E04AE250E06BE270E089E207
:104FE00090E00E941E5E81E090E00E94800B88238A
:104FF00011F05DE5D52E80913D2090913E2090FDF1
:1050000016E091FF07C0186005C0D12CE12C00E02C
:1050100010E0B12C63EF76E0CE010E943A93892B29
:1050200061F481E0F40180836091710270917202F9
:1050300080E090E00E944E93EC0161EF76E0CE01BB
:105040000E943A93892B61F48FEFF4018083609181
:1050500071027091720280E090E00E944E93EC0128
:10506000209709F424C16DEE76E0CE010E943A93B8
:10507000892B19F4FD2DF160DF2E69EE76E0CE016B
:105080000E943A93892B19F48D2D8460D82E66EEF8
:1050900076E0CE010E943A93892B19F4ED2DE2605F
:1050A000DE2E64EE76E0CE010E943A93892B19F44D
:1050B000FD2DF860DF2E61EE76E0CE010E943A937E
:1050C000892B19F48D2D8061D82E6BED76E0CE0101
:1050D0000E943A93892B19F4ED2DE062DE2E65EDE6
:1050E00076E0CE010E943A93892B19F4FD2DF064ED
:1050F000DF2E62ED76E0CE010E943A93892B19F4FF
:105100008D2D8068D82E6DEC76E0CE010E943A930A
:10511000892B19F4EE2DE160EE2E66EC76E0CE01DF
:105120000E943A93892B19F4FE2DF260EF2E63EC66
:1051300076E0CE010E943A93892B19F48E2D84607B
:10514000E82E6EEB76E0CE010E943A93892B19F49B
:10515000EE2DE860EE2E67EB76E0CE010E943A93EA
:10516000892B19F4FE2DF061EF2E60EB76E0CE0175
:105170000E943A93892B19F48E2D8062E82E6CEAF6
:1051800076E0CE010E943A93892B19F4EB2DE4606E
:10519000BE2E69EA76E0CE010E943A93892B19F47B
:1051A000FE2DF064EF2E64EA76E0CE010E943A9381
:1051B000892B19F48E2D8068E82E61EA76E0CE0105
:1051C0000E943A93892B09F401606EE976E0CE01E2
:1051D0000E943A93892B09F402606BE976E0CE01D4
:1051E0000E943A93892B09F4046067E976E0CE01C6
:1051F0000E943A93892B09F4086063E976E0CE01B6
:105200000E943A93892B09F400616FE876E0CE01A1
:105210000E943A93892B09F400626BE876E0CE0194
:105220000E943A93892B09F4006469E876E0CE0184
:105230000E943A93892B09F4006866E876E0CE0173
:105240000E943A93892B09F411606EE776E0CE0153
:105250000E943A93892B09F4126065E776E0CE014B
:105260000E943A93892B09F414606CE676E0CE0133
:105270000E943A93892B09F4186069E676E0CE0122
:105280000E943A93892B09F4106163E676E0CE011F
:105290000E943A93892B09F4106268E576E0CE010A
:1052A0000E943A93892B09F0D2CE1064D0CE2D2DD6
:1052B0003E2DA8016B2D70E080E090E0DF91CF9152
:1052C0001F910F91EF90DF90BF909F908F90089566
:1052D0005F926F927F928F929F92AF92BF92CF9286
:1052E000DF92EF92FF920F931F93CF93DF93782E6D
:1052F000C7E2DBE100E010E0F2E5EF2EF6E0FF2E82
:105300008170582E872D8270682EADE3CA2EA6E0DC
:10531000DA2EB5E4AB2EB6E0BB2E83E4882E86E011
:10532000982E772051F01F930F93FF92EF920E94D7
:1053300019940F900F900F900F905520A1F0898530
:105340008F9388858F93BF92AF920E9419940F908C
:105350000F900F900F906620C1F09F928F920E9445
:1053600019940F900F90662081F0DF92CF920E94E7
:105370001994288139814A815B816C817D818E817C
:105380009F810E9462240F900F900E94F20B0F5F8A
:105390001F4F2A960430110521F6DF91CF911F91FE
:1053A0000F91FF90EF90DF90CF90BF90AF909F90C4
:1053B0008F907F906F905F90089588E396E09F9321
:1053C0008F930E94199480912D1C90912E1CA09176
:1053D0002F1CB091301C0F900F90813027EA92075C
:1053E0002EE1A207B10519F48AE296E01DC08230D1
:1053F00026EA92072EE1A207B10519F48DE196E0A5
:1054000013C0823027EA92072EE1A207B10519F4F2
:105410008FE096E009C0823028EA92072EE1A207C9
:10542000B10549F481E096E09F938F930E9419940F
:105430000F900F900895BF93AF939F938F938BEF2F
:1054400095E09F938F930E9419940F900F900F9067
:105450000F900F900F9008958BEE95E09F938F9390
:105460000E9419940E94BF200E94DD290E94F20B25
:105470008EE09BE19F938F9383EE95E09F938F93B4
:105480000E941994609152027091530280915402CB
:105490009091550228EE33E040E050E00E94508D9C
:1054A0005F934F933F932F9383ED95E09F938F935B
:1054B0000E9419948AEC95E09F938F930E9419940F
:1054C0000E946B1080913D202DB73EB7225F3F4F69
:1054D0000FB6F8943EBF0FBE2DBF80FF05C041E060
:1054E00061E081E00E94151286EC95E09F938F9316
:1054F0000E94199480E00E949D220E94C320809106
:1055000057021F928F938DEB95E09F938F930E948C
:1055100019948091C1091F928F9384EB95E09F931A
:105520008F930E941994809183028F9380918202BD
:105530008F93809181028F93809180028F9386EA6E
:1055400095E09F938F930E9419941F9280E48F930C
:105550008EE895E09F938F930E9419948091132970
:105560001F928F93809112291F928F938BE795E062
:105570009F938F930E941994809156021F928F934C
:1055800082E795E09F938F930E941994809158022F
:1055900090915902A0915A02B0915B022DB73EB78B
:1055A000225E3F4F0FB6F8943EBF0FBE2DBF96FF51
:1055B00003C08EE895E002C081E995E09F938F9348
:1055C00088E695E09F938F930E94199483E00E9450
:1055D00068290F900F900F900F901D9B03C08EE8CD
:1055E00095E002C081E995E09F938F938CE595E06B
:1055F0009F938F930E94199482E595E09F938F93D8
:105600000E941994809158020F900F900F900F9064
:105610000F900F9081FF09C08CE495E09F938F93CA
:105620000E9419940F900F9013C080FF03C08EE862
:1056300095E002C081E995E09F938F9388E495E01F
:105640009F938F930E9419940F900F900F900F903B
:105650008091580290915902A0915A02B0915B0238
:1056600097FF03C08EE895E002C081E995E09F9323
:105670008F938FE395E09F938F930E94199488E313
:1056800095E09F938F930E9419946091C509709142
:10569000C60980E090E00E94D9220E94F20B0F9090
:1056A0000F900F900F900F900F90779903C08EE896
:1056B00095E002C081E995E09F938F938FE295E09A
:1056C0009F938F930E9419940E9492090E943C0B11
:1056D0009F938F937F936F9381E295E09F938F9336
:1056E0000E9419940E94EB0A9F938F937F936F936C
:1056F00083E195E09F938F930E94199481E090E05D
:105700000E9479218091E8289091E928A091EA28C7
:10571000B091EB28BF93AF939F938F9385E095E073
:105720009F938F930E9419948091FD288F9380916D
:10573000FC288F938091FB288F938091FA288F9378
:1057400081EF94E09F938F930E9419948091EC28AD
:105750009091ED28A091EE28B091EF28BF93AF93E0
:105760009F938F9383EE94E09F938F930E9419945D
:105770008DB79EB782960FB6F8949EBF0FBE8DBFB1
:10578000809101298F93809100298F938091FF2828
:105790008F938091FE288F938FEC94E09F938F934B
:1057A0000E94199461E070E080E090E00E94FB0BA1
:1057B00061E070E081E090E00E94FB0B0F900F90A1
:1057C0000F900F900F900F90299B03C08EE895E0EB
:1057D00002C081E995E09F938F9387EC94E09F93BB
:1057E0008F930E9419940F900F900F900F902A9B07
:1057F00003C08EE895E002C081E995E09F938F9306
:105800008FEB94E09F938F930E9419940F900F90C9
:105810000F900F900895F894E0E0F0E081E280931B
:1058200057008491E2E0F0E041E240935700449158
:10583000E4E0F0E091E290935700E49190E0A0E082
:10584000B0E0DC019927882750E060E070E0762F17
:10585000652F542F4427840F951FA61FB71F8E0F47
:10586000911DA11DB11D80932D1C90932E1CA09302
:105870002F1CB093301C78940895CF93DF93CDB74D
:10588000DEB761970FB6F894DEBF0FBECDBF48E21A
:1058900050E06EE170E087E29BE10E946D952091FF
:1058A000271B3091281B4091291B50912A1B609186
:1058B0002B1B70912C1B80912D1B90912E1BAFEFF9
:1058C0000E94888F09F05DC08DE48093271B80E8DB
:1058D0008093281B84E08093291B10922A1B10922E
:1058E0002B1B10922C1B10922D1B10922E1B8CE345
:1058F00090E09093301B80932F1B1092311B1092DD
:10590000321B1092331B1092341B1092351B1092D5
:10591000361B1092371B1092381B10923A1B1092B4
:10592000391B10923B1B10923C1B10923D1B109296
:105930003E1B10923F1B1092401B1092411B109275
:10594000421B1092441B1092431B1092451B109255
:10595000461B1092471B1092481B1092491B109235
:105960004A1B10924B1B10924C1B10924E1B109214
:105970004D1B48E250E06EE170E087E29BE10E943F
:105980008B9544E050E06AE170E0CE010B960E94F6
:105990006D958B859C85AD85BE858F3F2FEF9207DA
:1059A000A207B207A9F48AE090E4A0E0B0E08093F7
:1059B000580290935902A0935A02B0935B0244E0BC
:1059C00050E06AE170E088E592E00E948B9508C0A3
:1059D0008093580290935902A0935A02B0935B02AD
:1059E0008091580290915902A0915A02B0915B02A5
:1059F000A2FF02C02A9A03C080E00E94CD2242E0AA
:105A000050E066E570E0CE010F960E946D958F859F
:105A100098898F3F2FEF920769F41092C609109270
:105A2000C50942E050E066E570E085EC99E00E942F
:105A30008B9504C09093C6098093C50949E050E056
:105A40006AE070E082E099E20E946D950E94330D59
:105A500044E050E06AE470E0CE010B960E946D9540
:105A60008B859C85AD85BE8544E050E06AE470E09E
:105A70008F3F9F4FAF4FBF4F29F488E792E00E94BE
:105A80008B9504C088E792E00E946D9544E050E059
:105A900066E470E0CE010B960E946D958B859C8527
:105AA000AD85BE8544E050E066E470E08F3F9F4FD7
:105AB000AF4FBF4F29F484E792E00E948B9504C05A
:105AC00084E792E00E946D9544E050E06EE470E05F
:105AD000CE010B960E946D958B859C85AD85BE850C
:105AE00044E050E06EE470E08F3F9F4FAF4FBF4FF8
:105AF00029F48CE792E00E948B9504C08CE792E039
:105B00000E946D9541E050E069E170E0CE01419660
:105B10000E946D95898941E050E069E170E08F3F16
:105B200029F481EC99E00E948B9504C081EC99E006
:105B30000E946D9541E050E068E170E0CE01419631
:105B40000E946D95898941E050E068E170E08F3FE7
:105B500029F487E592E00E948B9504C087E592E0E6
:105B60000E946D9541E050E067E170E0CE01419602
:105B70000E946D95898941E050E067E170E08F3FB8
:105B800029F486E592E00E948B9504C086E592E0B8
:105B90000E946D954AE050E060E070E0CE01019611
:105BA0000E946D9589814AE050E060E070E08F3F8F
:105BB00029F48EE09BE10E948B9504C08EE09BE16E
:105BC0000E946D9544E050E062E570E0CE010B96D6
:105BD0000E946D958B859C85AD85BE8544E050E027
:105BE00062E570E08F3F9F4FAF4FBF4F29F480E8D1
:105BF00092E00E948B9504C080E892E00E946D952F
:105C000044E050E063E170E0CE010B960E946D9598
:105C10008B859C85AD85BE8544E050E063E170E0F6
:105C20008F3F9F4FAF4FBF4F29F482E592E00E9414
:105C30008B9504C082E592E00E946D9561960FB647
:105C4000F894DEBF0FBECDBFDF91CF910895CF9204
:105C5000DF92EF92FF92609171027091720280E088
:105C600090E00E944E9365E975E00E946293892B53
:105C700009F01FC18DE48093271B80E88093281BC7
:105C800084E08093291B10922A1B10922B1B1092E8
:105C90002C1B10922D1B10922E1B8CE390E09093E6
:105CA000301B80932F1B1092311B1092321B1092CD
:105CB000331B1092341B1092351B1092361B10921E
:105CC000371B1092381B10923A1B1092391B1092FE
:105CD0003B1B10923C1B10923D1B10923E1B1092DE
:105CE0003F1B1092401B1092411B1092421B1092BE
:105CF000441B1092431B1092451B1092461B10929E
:105D0000471B1092481B1092491B10924A1B10927D
:105D10004B1B10924C1B10924E1B10924D1B48E2D5
:105D200050E06EE170E087E29BE10E948B958AE093
:105D300090E4A0E0B0E08093580290935902A093C1
:105D40005A02B0935B0244E050E06AE170E088E5FB
:105D500092E00E948B951092C6091092C50942E00C
:105D600050E066E570E085EC99E00E948B9542E298
:105D7000C42EDD24DA944CECE42E4BE3F42EC092D6
:105D80007802D0927902E0927A02F0927B0244E0AB
:105D900050E06AE470E088E792E00E948B95C09240
:105DA0007402D0927502E0927602F092770244E09B
:105DB00050E066E470E084E792E00E948B9587ED06
:105DC00094E3AFEEBCE380937C0290937D02A093BA
:105DD0007E02B0937F0244E050E06EE470E08CE716
:105DE00092E00E948B958AE999E9A9E1B0E4809359
:105DF000800290938102A0938202B093830244E0D8
:105E000050E062E570E080E892E00E948B9510928D
:105E1000C10980E00E94996B41E050E069E170E0C7
:105E200081EC99E00E948B958AE1809357020E9451
:105E3000406A41E050E068E170E087E592E00E944E
:105E40008B958FE08093560241E050E067E170E06F
:105E500086E592E00E948B958AE0EEE0FBE1DF01AF
:105E60001D928A95E9F74AE050E060E070E0CF01CA
:105E70000E948B9580EA96E8A1E0B0E08093520200
:105E800090935302A0935402B093550244E050E023
:105E900063E170E082E592E00E948B9581E00E94D0
:105EA0009D2280E090E0FF90EF90DF90CF900C94E7
:105EB000470DFF90EF90DF90CF9008952F923F9283
:105EC0004F925F926F927F928F929F92AF92BF920A
:105ED000CF92DF92EF92FF920F931F93CF93DF93B6
:105EE000CDB7DEB72B970FB6F894DEBF0FBECDBF90
:105EF0009B878A874A01FC0180819181892B11F05F
:105F00000C946D426091710270917202CA010E94FC
:105F10004E9360E870E0C4010E948193009759F4A9
:105F20006091CD317091CE318AE090E00E94D5939E
:105F300081E00C9472428130910561F4F401B080EB
:105F40001B2D110F110B012F412E512E612E712E81
:105F5000A12EBCC082309105B9F4F401808199274B
:105F600087FD9095982F88272181820F911D27FD0D
:105F70009A95B82E192F092F000F000B402E502E86
:105F8000602E702EA02EA2C083309105B1F5F401D1
:105F90002081922F990F990B392F492F592F692F53
:105FA000792F892F00E10E942A8F19012A013B01D4
:105FB000B82FA92F2181922F990F990B392F492F93
:105FC000592F692F792F892F08E00E942A8F5901B4
:105FD0006A017B018C019101A201B3018B2F9A2FE1
:105FE0000E94618FA2801A2D110F110BB12EC12EAC
:105FF000D12EE12EF12E012F55C004970CF45DC077
:10600000F4012081922F990F990B392F492F592F85
:10601000692F792F892F08E10E942A8F19012A01FF
:106020003B01B82FA92F2181922F990F990B392F5E
:10603000492F592F692F792F892F00E10E942A8F2C
:1060400059016A017B018C019101A201B3018B2FDF
:106050009A2F0E94618FA3801A2D110F110BB12E60
:10606000C12ED12EE12EF12E012F0E94618F190138
:106070002A013B01B82FA92F2281922F990F990B4A
:10608000392F492F592F692F792F892F08E00E9426
:106090002A8F59016A017B018C019101A201B30190
:1060A0008B2F9A2F0E94618FB22E132F042F452E13
:1060B000562E672E782EA92E09C07AE0B72E10E052
:1060C00000E0412C512C612C712CA12C0E94F20B70
:1060D0002B2D312F402F542D652D762D872D9A2D68
:1060E0002537F3E63F07FDE64F07510561057105CA
:1060F0008105910511F40C94553D2537E3E63E07E3
:10610000EDE64E075105610571058105910511F018
:1061100008F0AAC12337F2E73F07410551056105A1
:1061200071058105910511F40C94E83F2337E2E7EE
:106130003E0741055105610571058105910511F085
:1061400008F0B2C02536F4E63F0741055105610568
:1061500071058105910509F4C8C62536E4E63E07B8
:1061600041055105610571058105910509F0B8F5F5
:10617000A6E70E94888F11F40C94EC390E94888F56
:1061800009F068F4A8E60E94888F09F4F4C6A5E730
:106190000E94888F11F40C94D6390C946B422B2DED
:1061A000312F402F542D652D762D872D9A2D2A3392
:1061B000F6E23F074105510561057105810591052D
:1061C00009F433C324363146410551056105710593
:1061D0008105910511F40C9410400C946B422B2D09
:1061E000312F402F542D652D762D872D9A2D273751
:1061F000FFE63F07410551056105710581059105E0
:1062000011F40C94BB3D2737EFE63E0741055105DD
:10621000610571058105910509F0C8F42436F9E698
:106220003F0741055105610571058105910511F48F
:106230000C94AF3925363E4641055105610571057F
:106240008105910511F40C94EF3D0C946B422B2DBC
:10625000312F402F542D652D762D872D9A2D2536E3
:10626000F2E73F074105510561057105810591057B
:1062700011F40C94B93E2936E2E73E074105510579
:10628000610571058105910511F40C94973F233345
:10629000314741055105610571058105910511F0F1
:1062A0000C946B420C9410402B2D312F402F542D09
:1062B000652D762D872D9A2D2236E5E63E07E4E6FC
:1062C0004E075105610571058105910509F40DC65B
:1062D0002236F5E63F07F4E64F07510561057105E3
:1062E0008105910511F008F054C02133E4E63E0722
:1062F000E1E64E075105610571058105910509F437
:10630000A4C22133F4E63F07F1E64F0751056105CA
:1063100071058105910509F0C0F42337E3E73E07D5
:1063200041055105610571058105910511F40C9434
:10633000FC3F28373447410551056105710581054A
:10634000910509F472C20C946B422B2D312F402F12
:10635000542D652D762D872D9A2D2336E4E63E07A4
:10636000E1E64E075105610571058105910511F4BE
:106370000C9410402837344641465105610571059B
:106380008105910511F00C946B420E94F9150C9453
:106390006D422B2D312F402F542D652D762D872DBD
:1063A0009A2D2D36E5E73E07E8E64E0751056105D3
:1063B00071058105910511F40C9426402D36F5E701
:1063C0003F07F8E64F075105610571058105910505
:1063D00009F0E0F42237E2E73E07E5E64E07510513
:1063E000610571058105910511F40C94143D233666
:1063F0003D4648465105610571058105910511F03D
:106400000C946B420E9471160C946D422B2D312F0F
:10641000402F542D652D762D872D9A2D2436E3E6B9
:106420003E07ECE64E0751056105710581059105B2
:1064300011F40C94773C2736FFE63F07FCE64F0744
:106440005105610571058105910511F40C947A3CA3
:106450002336324349465105610571058105910591
:1064600011F00C946B4211C22B2D312F402F542D63
:10647000652D762D872D9A2D2136FDE63F07F5E710
:106480004F07F8E65F07610571058105910511F475
:106490000C94D93D2136EDE63E07E5E74E07E8E6E8
:1064A0005E07610571058105910511F008F0D9C0FD
:1064B0002437F8E73F07F4E74F07510561057105F9
:1064C0008105910509F4F4C72437E8E73E07E4E7BE
:1064D0004E075105610571058105910511F008F020
:1064E00054C02133F1E33F07F1E74F075105610540
:1064F00071058105910511F40C94553D2133E1E3BB
:106500003E07E1E74E0751056105710581059105DB
:1065100009F0C8F42233F2E63F07F0E74F075105D0
:10652000610571058105910509F487C22033314366
:1065300041475105610571058105910511F40C94E0
:10654000143D0C946B422B2D312F402F542D652D73
:10655000762D872D9A2D2037F5E63F07F2E74F0776
:106560005105610571058105910511F40C94B93E41
:106570002C36344744475105610571058105910565
:1065800011F40C9494410C946B422B2D312F402F1D
:10659000542D652D762D872D9A2D2936FCE63F0743
:1065A000F1E64F07F3E65F07610571058105910587
:1065B00009F4D9C22936ECE63E07E1E64E07E3E6E8
:1065C0005E07610571058105910509F0E0F4243746
:1065D000F4E63F07F7E74F075105610571058105AF
:1065E000910511F40C94E24124373F464F46524640
:1065F000610571058105910511F00C946B420C94B5
:1066000000000C946D422B2D312F402F542D652D01
:10661000762D872D9A2D2633F9E63F07F5E74F07AC
:10662000F5E65F07610571058105910509F4A7C4C9
:106630002037ECE63E07E5E64E07E8E65E07610533
:1066400071058105910509F496C42E3631464846F8
:106650005346610571058105910509F4FDC60C9449
:106660006B422B2D312F402F542D652D762D872DEC
:106670009A2D2437E3E73E07E5E64E07E2E75E079B
:10668000610571058105910511F40C94693E24376B
:10669000F3E73F07F5E64F07F2E75F07610571058E
:1066A0008105910511F008F055C02337E2E73E0758
:1066B000E7E74E07E0E75E07610571058105910593
:1066C00011F40C946C3E2337F2E73F07F7E74F07CE
:1066D000F0E75F07610571058105910509F0C8F4D0
:1066E0002237E7E73E07E0E74E075E0761057105E1
:1066F0008105910509F406C22337354642475047C4
:10670000610571058105910511F40C94D6400C9436
:106710006B422B2D312F402F542D652D762D872D3B
:106720009A2D2436EDE63E07E3E64E07E2E75E07E4
:10673000610571058105910509F42CC521363C469A
:1067400045465247610571058105910509F434C438
:106750000C946B422B2D312F402F542D652D762D0F
:10676000872D9A2D2437E2E73E07E1E64E07E5E75D
:106770005E07610571058105910509F466C5243739
:10678000F2E73F07F1E64F07F5E75F07610571059F
:106790008105910509F0C8F42437E3E73E07E5E6F3
:1067A0004E07E4E75E07610571058105910509F46F
:1067B000AAC6273730474847544761057105810508
:1067C000910509F41FC60C946B422B2D312F402FDD
:1067D000542D652D762D872D9A2D2F36ECE63E070C
:1067E000EFE54E07E6E75E07610571058105910556
:1067F00009F47BC42C36F1E63F07F4E74F07F8E7CE
:106800005F07610571058105910511F40C945E41E6
:106810002237374640475547610571058105910587
:1068200011F00C946B420C94523C83E08093F0285E
:106830001092F2281092F12840EF58E262E184E3CE
:1068400092E00E94A3550C946D4221E042E161E088
:1068500080ED0E94DD6221E042E161E080ED0E9476
:10686000DD6221E042E161E080ED0E94DD6221E035
:1068700042E161E080ED0E94DD6221E042E161E001
:1068800080ED0E94DD620C946D4260917102709106
:10689000720280E090E00E944E936CE975E00E94E5
:1068A0006293892B09F0C5C06091710270917202E8
:1068B00080E090E00E944E935C01009709F497C03D
:1068C00060EE73E00E946293892BE1F488EE93E01E
:1068D000A0E0B0E08093520290935302A093540240
:1068E000B093550268EE73E080E090E00E9404618E
:1068F00044E050E063E170E082E592E00E948B9515
:106900000C946D4262EA75E0C5010E946293892B86
:10691000E1F480E197E2A0E0B0E08093520290932E
:106920005302A0935402B093550260E177E280E0F5
:1069300090E00E94046144E050E063E170E082E591
:1069400092E00E948B950C946D4265EA75E0C5015A
:106950000E946293892BE1F480EA96E8A1E0B0E01E
:106960008093520290935302A0935402B093550225
:1069700060EA76E881E090E00E94046144E050E043
:1069800063E170E082E592E00E948B950C946D4289
:1069900069EA75E0C5010E946293892BE1F480E801
:1069A0009AE1A6E0B0E08093520290935302A09344
:1069B0005402B093550260E87AE186E090E00E94CC
:1069C000046144E050E063E170E082E592E00E94FF
:1069D0008B950C946D4280E093E09F938F930E947F
:1069E00019940E94F20B0F900F900C946D426091DD
:1069F000520270915302809154029091550228EEF8
:106A000033E040E050E00E94508D5F934F933F93FE
:106A10002F938CEF92E09F938F930E9419940E9482
:106A2000F20B0F900F900F900F900F900F900C940F
:106A30006D420E946B100C946D42609171027091D6
:106A4000720280E090E00E944E938C016EE875E047
:106A50000E946293892BE1F480915802909159022F
:106A6000A0915A02B0915B02A46080935802909367
:106A70005902A0935A02B0935B022A9A44E050E074
:106A80006AE170E088E592E00E948B950C946D427B
:106A900061E975E0C8010E946293892BF1F480914D
:106AA000580290915902A0915A02B0915B02AB7FBB
:106AB0008093580290935902A0935A02B0935B02BC
:106AC00080E00E94CD2244E050E06AE170E088E579
:106AD00092E00E948B950C946D422A9B03C08EE835
:106AE00095E002C081E995E09F938F9384EF92E057
:106AF0009F938F930E9419940F900F900F900F9077
:106B00000C946D42609171027091720280E090E08D
:106B10000E944E938C016EE875E00E946293892B6F
:106B200019F477980C946D4261E975E0C8010E94F0
:106B30006293892B19F4779A0C946D42779903C06C
:106B40008EE895E002C081E995E09F938F9389EAF2
:106B500094E09F938F930E9419940F900F900F9041
:106B60000F900C946D42609171027091720280E0FE
:106B700090E00E944E938C0168E575E00E9462935C
:106B8000892B09F077C0609171027091720280E0E8
:106B900090E00E944E938C01009711F40C946D428A
:106BA0006DEA75E00E946293892BB1F482E29FEF57
:106BB000ACECBBE38093780290937902A0937A02C5
:106BC000B0937B0244E050E06AE470E088E792E032
:106BD0000E948B950C946D4263EB75E0C8010E9496
:106BE0006293892BB1F482E29FEFACECBAE380931D
:106BF000780290937902A0937A02B0937B0244E0EA
:106C000050E06AE470E088E792E00E948B950C9473
:106C10006D42C8010E9438922B013C0120E030E017
:106C2000A9010E94D3898823D9F081E00E94880AB3
:106C30009B01AC01C301B2010E94D7896093780225
:106C40007093790280937A0290937B0244E050E043
:106C50006AE470E088E792E00E948B950C946D42A4
:106C600087EE92E09F938F930E9419940F900F905C
:106C70000C946D426BE575E0C8010E946293892B0C
:106C800009F077C0609171027091720280E090E02B
:106C90000E944E938C01009711F40C946D426DEAA2
:106CA00075E00E946293892BB1F482E29FEFACEC15
:106CB000BBE38093740290937502A0937602B09325
:106CC000770244E050E066E470E084E792E00E94DE
:106CD0008B950C946D4263EB75E0C8010E94629342
:106CE000892BB1F482E29FEFACECBAE3809374029B
:106CF00090937502A0937602B093770244E050E03F
:106D000066E470E084E792E00E948B950C946D42FB
:106D1000C8010E9438922B013C0120E030E0A9011B
:106D20000E94D3898823D9F082E00E94880A9B01BF
:106D3000AC01C301B2010E94D789609374027093C1
:106D40007502809376029093770244E050E066E407
:106D500070E084E792E00E948B950C946D428AED7E
:106D600092E09F938F930E9419940F900F900C9430
:106D70006D4263E575E0C8010E946293892B09F0BA
:106D800073C0609171027091720280E090E00E9485
:106D90004E938C01009711F40C946D426DEA75E0EE
:106DA0000E946293892BB1F487ED94E3AFEEBCE3CC
:106DB00080937C0290937D02A0937E02B0937F0229
:106DC00044E050E06EE470E08CE792E00E948B9526
:106DD0000C946D4263EB75E0C8010E946293892BAD
:106DE00051F48BEC92E09F938F930E9419940F9033
:106DF0000F900C946D42C8010E9438922B013C0107
:106E000020E030E0A9010E94D389882319F180E0B5
:106E10000E94880A4B015C0121EE3AE744E95EE3F7
:106E2000C301B2010E940C89A50194010E94D78977
:106E300060937C0270937D0280937E0290937F0228
:106E400044E050E06EE470E08CE792E00E948B95A5
:106E50000C946D428EEB92E09F938F930E94199455
:106E60000F900F900C946D420E94D70A9F938F93BE
:106E70007F936F9387EB92E09F938F930E94199477
:106E800082E00E94880A209174023091750240913C
:106E90007602509177020E94588C162F072FF82EF9
:106EA000E92E81E00E94880AEF92FF920F931F93D0
:106EB000209178023091790240917A0250917B02C0
:106EC0000E94588C9F938F937F936F938BEA92E0ED
:106ED0009F938F930E9419940E94F20B0FB6F8941F
:106EE000DEBF0FBECDBF0C946D42609171027091F8
:106EF000720280E090E00E944E930097C1F00E94E1
:106F0000C7232091C5093091C6098217930709F15B
:106F10009093C6098093C50942E050E066E570E0B1
:106F200085EC99E00E948B9582EA94E002C08BE99F
:106F300094E09F938F930E9419946091C50970917A
:106F4000C60980E090E00E94D9220E94F20B0F90C7
:106F50000F9080E994E09F938F930E9419946FEFB4
:106F60007FEF80E090E00E94D9220E94F20B0F9008
:106F70000F900C946D420E94C81F0C946D42F40156
:106F80008481843329F440E061E080E00E9415129E
:106F900080917302882311F40C946D421F928F9399
:106FA0008DE894E09F938F930E9419940F900F9017
:106FB0000F900F900C946D42F4018481893709F091
:106FC00080C0609171027091720280E090E00E9436
:106FD0004E938C016EE875E00E946293892B51F408
:106FE0008091580290915902A0915A02B0915B028F
:106FF000906410C061E975E0C8010E946293892B1A
:10700000D1F48091580290915902A0915A02B09106
:107010005B029F7B8093580290935902A0935A027F
:10702000B0935B0244E050E06AE170E088E592E0F2
:107030000E948B9546C068EB75E0C8010E94629380
:10704000892B21F58091261B8F938091251B8F938F
:107050008091241B8F938091231B8F938091221BFF
:107060008F938091211B8F938091201B8F93809110
:107070001F1B8F9380E892E09F938F930E94199437
:107080000FB6F894DEBF0FBECDBF1BC08091580273
:1070900090915902A0915A02B0915B0296FF03C0F1
:1070A0008EE895E002C081E995E09F938F938CE78D
:1070B00092E09F938F930E9419940F900F900F90DE
:1070C0000F9080917302882311F40C946D421F92EB
:1070D0008F938AE894E09F938F930E9419940F9066
:1070E0000F900F900F900C946D42F40184818737BC
:1070F000E9F5609171027091720280E090E00E9467
:107100004E930097D9F00E9438922B013C0120E069
:1071100030E0A9010E94D389882381F04092800247
:1071200050928102609282027092830244E050E0A9
:1071300062E570E080E892E00E948B958091830286
:107140008F93809182028F93809181028F9380919F
:1071500080028F938EE692E09F938F930E94199402
:107160000F900F900F900F900F900F9080917302DF
:10717000882311F40C946D421F928F9387E894E05A
:107180009F938F930E9419940F900F900F900F90E0
:107190000C946D42609171027091720280E090E0F7
:1071A0000E944E938C016EE875E00E9462934090BD
:1071B00058025090590260905A0270905B02892BDD
:1071C00019F4689457F809C061E975E0C8010E9494
:1071D0006293892B99F4E89457F8409258025092A0
:1071E000590260925A0270925B0244E050E06AE1F8
:1071F00070E088E592E00E948B9513C057FE03C0B3
:107200008EE895E002C081E995E09F938F938AE62E
:1072100092E09F938F930E9419940F900F900F907C
:107220000F9080917302882311F40C946D421F9289
:107230008F9384E894E09F938F930E9419940F900A
:107240000F900F900F900C946D42609171027091AD
:10725000720280E090E00E944E935C016EEB75E05C
:107260000E946293892B11F489E108C062EC75E0F9
:10727000C5010E946293892B49F480E18093C40088
:107280001092C50082E08093C00055C066EC75E0A6
:10729000C5010E946293892B11F488E0EFCF6BEC5B
:1072A00075E0C5010E946293892B39F060ED75E0AD
:1072B000C5010E946293892B11F483E0DFCF809196
:1072C000C400893141F485E692E09F938F930E9438
:1072D00019940F900F908091C400803141F480E6A2
:1072E00092E09F938F930E9419940F900F9080913A
:1072F000C400883041F48AE592E09F938F930E9406
:1073000019940F900F908091C400833041F484E56C
:1073100092E09F938F930E9419940F900F90809109
:10732000C400883041F48EE492E09F938F930E94D2
:1073300019940F900F9080917302882311F40C948C
:107340006D421F928F9381E894E09F938F930E94E8
:1073500019940F900F900F900F900C946D426091C4
:1073600071027091720280E090E00E944E936DEA8B
:1073700075E00E946293892B11F481E001C080E0E6
:107380000E949D2280917302882311F40C946D4217
:107390001F928F938EE794E09F938F930E9419948E
:1073A0000F900F900F900F900C946D420E94C3208D
:1073B00080917302882311F40C946D421F928F9375
:1073C0008BE794E09F938F930E9419940F900F90F6
:1073D0000F900F900C946D420E94BF208091730219
:1073E000882311F40C946D421F928F9388E794E0E8
:1073F0009F938F930E9419940F900F900F900F906E
:107400000C946D42609171027091720280E090E084
:107410000E944E930E943C92803170F48093C10987
:107420000E94996B41E050E069E170E081EC99E0E5
:107430000E948B950C946D428091C1091F928F938D
:1074400084E492E09F938F930E9419940F900F9081
:107450000F900F900C946D426091710270917202C6
:1074600080E090E00E944E930E943C9295EF980F2E
:10747000903170F4809357020E94406A41E050E0DE
:1074800068E170E087E592E00E948B950C946D4274
:10749000809157021F928F938BE392E09F938F937B
:1074A0000E9419940F900F900F900F900C946D42C2
:1074B000609171027091720280E090E00E944E93A0
:1074C000009789F04AE050E0BC018EE09BE10E9409
:1074D00072934AE050E060E070E08EE09BE10E9431
:1074E0008B950C946D428EE09BE19F938F9385ED7D
:1074F00095E09F938F930E9407940F900F900F90A9
:107500000F900C946D42609171027091720280E054
:1075100090E00E944E935C0160EE73E00E946293E3
:10752000892BD9F4219A8091580290915902A09107
:107530005A02B0915B028061809358029093590285
:10754000A0935A02B0935B0244E050E06AE170E01D
:1075500088E592E00E948B95C0C76CE575E0C50197
:107560000E946293892BD9F4229A809158029091BB
:107570005902A0915A02B0915B0280628093580236
:1075800090935902A0935A02B0935B0244E050E0FA
:107590006AE170E088E592E00E948B959EC762ECFC
:1075A00073E0C5010E946293892BD9F4239A8091DC
:1075B000580290915902A0915A02B0915B028064E6
:1075C0008093580290935902A0935A02B0935B02A1
:1075D00044E050E06AE170E088E592E00E948B951B
:1075E0007CC76FEF74E0C5010E946293892BD9F4C8
:1075F000239A8091580290915902A0915A02B09119
:107600005B0280688093580290935902A0935A02BB
:10761000B0935B0244E050E06AE170E088E592E0FC
:107620000E948B955AC76CE679E0C5010E9462936F
:10763000892B71F581E08093542487E29BE190933C
:1076400056248093552410925824109257248091E8
:10765000580290915902A0915A02B0915B02916038
:107660008093580290935902A0935A02B0935B0200
:1076700044E050E06AE170E088E592E00E948B957A
:1076800044E554E262E184E392E00E94A35525C7F9
:1076900069EE73E0C5010E946293892B11F5E7E55D
:1076A000FBE1119211922BE1E737F207D1F78091BC
:1076B000580290915902A0915A02B0915B029260D7
:1076C0008093580290935902A0935A02B0935B02A0
:1076D00044E050E06AE170E088E592E00E948B951A
:1076E000FCC661E975E0C5010E94629340915802B1
:1076F0005091590260915A0270915B02892BC1F43A
:107700004F705C7F409358025093590260935A0225
:1077100070935B022B9A44E050E06AE170E088E5E8
:1077200092E00E948B958091F9280E94556AD5C6F7
:1077300044FF03C08EE895E002C081E995E09F9385
:107740008F9380E392E09F938F930E94199480918E
:1077500058020F900F900F900F9085FF03C08EE896
:1077600095E002C081E995E09F938F9385E292E0D6
:107770009F938F930E941994809158020F900F90BD
:107780000F900F9086FF03C08EE895E002C081E95C
:1077900095E09F938F938AE192E09F938F930E944D
:1077A0001994809158020F900F900F900F9087FFBF
:1077B00003C08EE895E002C081E995E09F938F9326
:1077C0008FE092E09F938F930E94199480915802CA
:1077D00090915902A0915A02B0915B020F900F90C4
:1077E0000F900F9090FF03C08EE895E002C081E9F2
:1077F00095E09F938F9384E092E09F938F930E94F4
:1078000019948091580290915902A0915A02B09116
:107810005B020F900F900F900F9091FF03C08EE8C6
:1078200095E002C081E995E09F938F9389EF91E005
:107830009F938F930E9419948091580290915902BE
:10784000A0915A02B0915B020F900F900F900F9091
:1078500091FF43C68DED95E00E943D9457E5A52E1E
:107860005BE1B52E0BE010E065EE862E65E0962E0E
:10787000F50180819181F2E0AF0EB11C9F938F934F
:107880001F930F939F928F920E9407940F5F1F4F39
:107890000F900F900F900F900F900F900B311105DC
:1078A00039F71BC684E794E09F938F930E94199445
:1078B000809173020F900F90882361F01F928F9335
:1078C00081E794E09F938F930E9419940F900F90FB
:1078D0000F900F90F89428E088E190E00FB6F894AC
:1078E000A895809360000FBE20936000FFCF0E9498
:1078F0008E62F3C5609171027091720280E090E037
:107900000E944E938C016EE875E00E946293892B71
:10791000E9F40E9441698091580290915902A09126
:107920005A02B0915B028D7F8160809358029093E0
:107930005902A0935A02B0935B0244E050E06AE11E
:1079400070E088E592E00E948B95C7C561E975E01B
:10795000C8010E946293892BE1F40E94F96880912A
:10796000580290915902A0915A02B0915B028C7F0B
:107970008093580290935902A0935A02B0935B02ED
:1079800044E050E06AE170E088E592E00E948B9567
:10799000A4C560EF75E0C8010E946293892BE9F4E9
:1079A0000E94F9688091580290915902A0915A0260
:1079B000B0915B028E7F826080935802909359024F
:1079C000A0935A02B0935B0244E050E06AE170E099
:1079D00088E592E00E948B9580C58091580281FFD6
:1079E0000FC080EF95E09F938F9385EF91E09F9379
:1079F0008F930E9419940F900F900F900F906DC568
:107A000080FF03C08EE895E002C081E995E09F9376
:107A10008F9381EF91E09F938F930E9419940F9021
:107A20000F900F900F9059C5809152248F938091A1
:107A300051248F93809150248F9380914F248F9362
:107A400080914E248F9380914D248F9380914C246C
:107A50008F9380914B248F9380914A248F938091B0
:107A600049248F93809148248F93809147248F934A
:107A70008EE494E09F938F930E94199480917302F7
:107A80000FB6F894DEBF0FBECDBF882309F425C51D
:107A90001F928F938BE494E09F938F930E9419948D
:107AA0000F900F900F900F9018C5F89481E090E020
:107AB00029E0FC0120935700C895E02C80E090E07D
:107AC000FC0120935700C895F02C7894F89483E03B
:107AD00090E0FC0120935700C895002D82E090E0D3
:107AE000FC0120935700C895102D78948091301C8C
:107AF0008F9380912F1C8F9380912E1C8F93809158
:107B00002D1C8F9321E434E03F932F930E9419940E
:107B10001F92EF921F92FF921F920F931F921F933B
:107B20008AE194E09F938F930E9419940E945D21B3
:107B3000809166001F928F938EE094E09F938F93C5
:107B40000E9419940E94F20B809173020FB6F89470
:107B5000DEBF0FBECDBF882309F4BFC41F928F9331
:107B60008BE094E09F938F930E9419940F900F9055
:107B70000F900F90B2C460E070E080E090E00E944F
:107B8000FB0B60E070E081E090E00E94FB0B8091D5
:107B90007302882309F4A1C41F928F9388E094E0B4
:107BA0009F938F930E9419940F900F900F900F90B6
:107BB00094C40E948B1F0E94F20B80917302882351
:107BC00009F48BC41F928F9385E094E09F938F9369
:107BD0000E9419940F900F900F900F907EC46091A7
:107BE00071027091720280E090E00E944E9365EF06
:107BF00075E00E946293892B31F5F8948CEF99E03F
:107C00000E9490565C01009769F0C5010F960E9492
:107C10009459B50184E092E00E944A56C5010E9441
:107C20003857F0CF8CEF99E00E941D57892B29F02F
:107C30008CEF99E00E94C956F5CF8CEF99E00E9435
:107C40008C56789434C08CEF99E00E9490565C0179
:107C50000BEF15E0A114B10451F1F50186811F92DB
:107C60008F9380851F928F9385811F928F9381853B
:107C70001F928F9387811F928F9384811F928F937E
:107C800083811F928F9382811F928F9382851F928F
:107C90008F931F930F930E940794C5010E9438573A
:107CA0005C010FB6F894DEBF0FBECDBFD3CF80917D
:107CB0007302882309F411C41F928F9382E094E029
:107CC0009F938F930E9419940F900F900F900F9095
:107CD00004C40E94272E01C4609171027091720247
:107CE00080E090E00E944E938C016AE376E00E946F
:107CF0006293892BD1F48091580290915902A091FE
:107D00005A02B0915B02977F809358029093590278
:107D1000A0935A02B0935B0244E050E06AE170E045
:107D200088E592E00E948B95D8C363EB75E0C801AB
:107D30000E946293892BD1F480915802909159024C
:107D4000A0915A02B0915B02986080935802909380
:107D50005902A0935A02B0935B0244E050E06AE1FA
:107D600070E088E592E00E948B95B7C30E9492096B
:107D7000B4C3609171027091720280E090E00E9441
:107D80004E93FC0120812332B1F44AE050E060E0E0
:107D900070E001960E94F08F1B016091710270915A
:107DA000720280E090E00E944E93F4E02F163104BE
:107DB0000CF094C002C0212C312C009709F48EC025
:107DC0001982BE016F5F7F4F0E94C62729013A01C9
:107DD0004B01B82FA92F8AE0829DF001839DF00D01
:107DE0001124E95DF44E20812A8331813B83828115
:107DF0008C8393819D8324812E8335813F8386816B
:107E00008887978199879201A301B4018B2F9A2FBC
:107E1000AA80BB80CC80DD80EE80FF80088519853C
:107E20000E947F8F09F45DC08981882351F18CF015
:107E30002A81422A3B81532A8C81682A9D81792A92
:107E40002E81822A3F81932A8885B82B9985A92B78
:107E500018C0409450946094709480949094B0951D
:107E6000A0952A8142223B8153228C8168229D81E8
:107E700079222E8182223F8193228885B823998599
:107E8000A923408251826282738284829582B68362
:107E9000A78348E250E06EE170E087E29BE10E9438
:107EA0008B958AEF93E09F938F930E9419948AE0B9
:107EB000829DF001839DF00D1124E95DF44E208137
:107EC00031814281538164817581868197810E94CD
:107ED00062240E94F20B0F900F9003C082E00E9478
:107EE00068298EEE93E09F938F930E9419942FEF51
:107EF0003FEF4FEF5FEF6FEF7FEF8FEF9FEF0E944E
:107F000062240E94F20B809173020F900F908823DD
:107F100009F4E3C21F928F938BEE93E09F938F93AC
:107F20000E9419940F900F900F900F90D6C26091FD
:107F300071027091720280E090E00E944E93FC0109
:107F400020812332A1F44AE050E060E070E0019625
:107F50000E94F08F8B01609171027091720280E03B
:107F600090E00E944E9304301105ECF402C000E052
:107F700010E00097C1F04AE050E060E070E00E943D
:107F800024912AE0209FF001219FF00D1124E95D4A
:107F9000F44E7187608748E250E06EE170E087E25E
:107FA0009BE10E948B9581E00E9468298091730279
:107FB000882309F492C21F928F9388EE93E09F93D7
:107FC0008F930E9419940F900F900F900F9085C27D
:107FD0000E94CD5980917302882309F47EC21F92BA
:107FE0008F9385EE93E09F938F930E9419940F9047
:107FF0000F900F900F9071C20E942C2A80917302F3
:10800000882309F46AC21F928F9382EE93E09F93B4
:108010008F930E9419940F900F900F900F905DC254
:1080200080E090E00E94792180917302882309F416
:1080300054C21F928F938FED93E09F938F930E9472
:1080400019940F900F900F900F9047C280913D2090
:1080500081FF2DC00E940F1F892B49F58091341C90
:108060008F938091331C8F938091321C8F938091DA
:10807000311C8F9384ED93E09F938F930E9419940A
:10808000809111298F93809110298F9380910F29CE
:108090008F9380910E298F9387EC93E09F938F931A
:1080A0000E9419940FB6F894DEBF0FBECDBF0E9498
:1080B000F20B80913D2090913E2090FF63C081E0C3
:1080C00090E00E94861E3B014C0180E090E00E94FF
:1080D000861E1B012C010E94E41D9F928F927F92AD
:1080E0006F9286EB93E09F938F930E9419945F9217
:1080F0004F923F922F9286EA93E09F938F930E9434
:108100001994222D332D442D552D662D772D882D34
:10811000992D0E94871C9F938F937F936F938BE978
:1081200093E09F938F930E941994222D332D442D19
:10813000552D662D772D882D992D0E94E81C9F9333
:108140008F937F936F938DE893E09F938F930E941B
:108150001994222D332D442D552D662D772D882DE4
:10816000992D0E94491D9F938F937F936F938AE768
:1081700093E09F938F930E9419940FB6F894DEBFFB
:108180000FBECDBF0E94F20B80917302882309F4C9
:10819000A4C11F928F9387E793E09F938F930E94D0
:1081A00019940F900F900F900F9097C180913D20E0
:1081B00082FF2BC021E048E061E083E00E948A1347
:1081C00080912B1C8F9380912A1C8F938091291C66
:1081D0008F938091281C8F938091271C8F9380917F
:1081E000261C8F938091251C8F938091241C8F9344
:1081F00080E693E09F938F930E9419940E94F20B64
:108200000FB6F894DEBF0FBECDBF80913D20909198
:108210003E2091FF41C00E94D417B62EA72E982E63
:10822000892E20E030E048EC52E4D501F4016B2FB8
:108230007A2F8F2F9E2F0E94588C20E836EE45EC27
:1082400057E40E94D78921E03EED42E45EE30E94BC
:10825000BB8C9B01AC0160E070E080E89FE30E9472
:108260000C892BE43AE34DEB57E30E94D7899F93A7
:108270008F937F936F938F929F92AF92BF9287E479
:1082800093E09F938F930E9419940E94F20B0FB674
:10829000F894DEBF0FBECDBF80917302882309F42E
:1082A0001CC11F928F9384E493E09F938F930E944D
:1082B00019940F900F900F900F900FC16091710261
:1082C0007091720280E090E00E944E936FE376E03E
:1082D0000E946293892BB1F46091710270917202D5
:1082E00080E090E00E944E93009709F4F6C00E944F
:1082F0003C92803108F0F1C090915201982B9093FC
:108300005201EBC0809152018F701F928F9384EEC7
:1083100091E09F938F930E9419940E94F20B0F900B
:108320000F900F900F90D9C06091710270917202FE
:1083300080E090E00E944E93009711F14AE050E0F7
:1083400060E070E00E94F08F603198F46093560214
:108350001F926F9387E393E09F938F930E941994EA
:1083600041E050E067E170E086E592E00E948B9585
:1083700011C0809156021F928F938EE293E006C047
:10838000809156021F928F9385E293E09F938F9383
:108390000E9419940F900F900F900F900E94F20B73
:1083A00080917302882309F498C01F928F9382E210
:1083B00093E09F938F930E9419940F900F900F90CA
:1083C0000F908BC0609171027091720280E090E01A
:1083D0000E944E938C016EE875E00E946293892B97
:1083E000E1F40E94AA678091580290915902A091ED
:1083F0005A02B0915B0290618093580290935902A7
:10840000A0935A02B0935B0244E050E06AE170E04E
:1084100088E592E00E948B9560C061E975E0C80133
:108420000E946293892B81F5F8940E94B86788E1D5
:108430000FB6F89480936000109260000FBE84B76E
:10844000877F84BF80916000886180936000109274
:10845000600078948091580290915902A0915A023C
:10846000B0915B029F7E8093580290935902A09333
:108470005A02B0935B0244E050E06AE170E088E5A4
:1084800092E00E948B9529C064E476E0C8010E94C6
:108490006293409158025091590260915A02709132
:1084A0005B02892B21F454FF18C0F894FFCF54FFCE
:1084B00003C08EE895E002C081E995E09F938F9319
:1084C00080EE91E09F938F930E9419940F900F90EC
:1084D0000F900F9002C00E94AF1FEA85FB851182AA
:1084E000108283E02B960FB6F894DEBF0FBECDBF8F
:1084F000DF91CF911F910F91FF90EF90DF90CF9080
:10850000BF90AF909F908F907F906F905F904F90B3
:108510003F902F9008950F931F93CF93DF93EC011B
:108520008A0188819981009711F1813C904121F065
:108530001982188283E020C06231E9F4A80162E167
:1085400070E08DEE99E00E945E2F84E08093F02829
:108550001092F2281092F1281093F4280093F32837
:1085600040EF58E262E184E392E00E94A35581EC7F
:1085700090E19983888381E0DF91CF911F910F91E2
:1085800008950E949E676C9A6B9A6A9A6F9A729A83
:10859000749A739A779A809880B3897F80BB839806
:1085A000849887E080937E00549A0E940B2C0E944E
:1085B0003D2C81E00E94FC0980E090E00E94470D84
:1085C0006091520270915302809154029091550231
:1085D0000E9404610E94EB0A60933F247093402440
:1085E00080934124909342248091580286FD239ADF
:1085F000219A229A239A1D9B05C01092C3091092BA
:10860000C209089581E090E09093C3098093C20964
:108610000895CF93DF93EC0188819981009741F011
:108620008C3A904109F48CC01982188283E093C07F
:108630000E94C1428091580280FD05C081FF01C0A7
:108640001D9B0E94F968809170008C7F8093700060
:108650008091B60080628093B6001092B20082E0F2
:108660008093B1008091B6008770E1F7809170002F
:1086700081608093700060EB79E080E090E00E9480
:1086800088670E94BF2080E00E949D228FE69FE0C5
:108690009F938F930E9419940E946B1080913D20AC
:1086A0000F900F9086FD0E943A6280913D2090913C
:1086B0003E2090FD0E94A01D80913D2087FF06C0B6
:1086C00021E04CE061E080ED0E94DD628091C10913
:1086D0000E94996B809157020E94406A0E943D6AF5
:1086E0008093EC09809157020E94406A8091C109F1
:1086F0001F928F938091EC091F928F9389E496E0EB
:108700009F938F930E9407941092EE091092ED09A7
:108710000F900F900F900F900F900F9088E492E0C1
:1087200090930C2980930B2983E290E09093FF11A2
:108730008093FE118CEA90E19983888381E00BC0DD
:108740006332E1F748E654E260E070E08DEE99E0D4
:108750000E945E2FE3CFDF91CF910895843691057B
:1087600014F19F938F938BE596E09F938F930E94D4
:1087700007948091472490914824A0914924B09176
:108780004A240196A11DB11D80934724909348244B
:10879000A0934924B0934A240F900F900F900F900C
:1087A00081E090E0089580E090E008952F923F925C
:1087B0004F925F926F927F928F929F92AF92BF92F1
:1087C000CF92DF92EF92FF920F931F93CF93DF939D
:1087D000CDB7DEB7C859D1090FB6F894DEBF0FBECA
:1087E000CDBFCF56DF4F99838883C159D0408A01CE
:1087F000633871F481EF99E0C856DF4F6883C85938
:10880000D0400E94E653C856DF4F6881C859D04017
:10881000CF56DF4FA881B981C159D0402D913C91ED
:108820002935B0E13B0709F4C9C340F421153105EE
:1088300081F027393E4009F407C4FBC32B3640E1E1
:10884000340709F4D7C32237304111F40C94EE50A9
:10885000F0C34AEE52E061E870E081EF99E00E94D7
:10886000CC5387E99EE0A1C3E3E0F0E0EC0FFD1FED
:10887000E20FF31F1082C9010E94AE43892B89F7D2
:1088800020E030E040E050E0C357DF4F6881CD5832
:10889000D040627070E080E090E0A0E00E94888F9D
:1088A00009F084C6C557DF4F2881CB58D0402870C7
:1088B00030E040E050E060E070E080E090E0A0E078
:1088C0000E94888FA1F127E04AE250E06BE270E05D
:1088D00089E290E00E941E5E82E099E20E948C6034
:1088E000BC01882777FD8095982F0E94768A20E02A
:1088F00030E048EC52E40E94D7899F938F937F9396
:108900006F938FE896E09F938F931F9287E78F93E3
:10891000CE018E0D9F1D03969F938F930E946A94A4
:10892000E80EF91E0FB6F894DEBF0FBECDBFC557D7
:10893000DF4F2881CB58D040207130E040E050E03C
:1089400060E070E080E090E0A0E00E94888FF1F1AC
:1089500026E04AE250E06BE270E089E290E00E949B
:108960001E5E81E090E00E94800B8093C00980E849
:108970009BE10E948C60BC01882777FD8095982F31
:108980000E94768A20E030E048EC52E40E94D789C9
:108990009F938F937F936F9389E996E09F938F9333
:1089A0001F9287E78F93C7010296E1E0F0E0EC0F9A
:1089B000FD1F8E0F9F1F9F938F930E946A94E80E56
:1089C000F91E0FB6F894DEBF0FBECDBF272D30E0E5
:1089D00040E050E060E070E080E090E0A0E00E94C5
:1089E000888F01F10E943C0B9F938F937F936F932D
:1089F00084EA96E09F938F931F9287E78F93C70136
:108A0000029641E050E04C0F5D1F840F951F9F932D
:108A10008F930E946A94E80EF91E0FB6F894DEBF99
:108A20000FBECDBFC557DF4F2881CB58D040207433
:108A300030E040E050E060E070E080E090E0A0E0F6
:108A40000E94888F31F1809142248F93809141243C
:108A50008F93809140248F9380913F248F9382EB5A
:108A600096E09F938F931F9287E78F93C70102969B
:108A7000A1E0B0E0AC0FBD1F8A0F9B1F9F938F93A7
:108A80000E946A94E80EF91E0FB6F894DEBF0FBE7E
:108A9000CDBFC557DF4F2881CB58D040207830E07C
:108AA00040E050E060E070E080E090E0A0E00E94F4
:108AB000888F41F1F8948091E8289091E928A0915D
:108AC000EA28B091EB287894BF93AF939F938F934C
:108AD00080EC96E09F938F931F9287E78F93C70157
:108AE000029621E030E02C0F3D1F820F931F9F93D1
:108AF0008F930E946A94E80EF91E0FB6F894DEBFB9
:108B00000FBECDBF20E0C457DF4F3881CC58D040D6
:108B1000317040E050E060E070E080E090E0A0E084
:108B20000E94888F09F054C520E0C457DF4F388178
:108B3000CC58D040327040E050E060E070E080E01F
:108B400090E0A0E00E94888F09F0B5C520E0C457EE
:108B5000DF4F3881CC58D040347040E050E060E0C6
:108B600070E080E090E0A0E00E94888F09F0D4C51A
:108B700020E0C457DF4F3881CC58D040387040E0F7
:108B800050E060E070E080E090E0A0E00E94888F1C
:108B900009F0F1C520E0C457DF4F3881CC58D040F0
:108BA000307140E050E060E070E080E090E0A0E0F4
:108BB0000E94888F09F052C620E0C457DF4F3881E9
:108BC000CC58D040307240E050E060E070E080E08F
:108BD00090E0A0E00E94888F09F070C620E030E0AD
:108BE00040E050E0C357DF4F6881CD58D0406470FB
:108BF00070E080E090E0A0E00E94888F09F08CC6D1
:108C000020E0C057DF4F3881C059D04040E050E0ED
:108C100060E070E080E090E0A0E00E94888F09F0C2
:108C2000E8C620E0CA56DF4F3881C659D04040E040
:108C300050E060E070E080E090E0A0E00E94888F6B
:108C400009F005C720E030E0402F417050E060E0BF
:108C500070E080E090E0A0E00E94888F09F025C7D6
:108C600020E030E0402F427050E060E070E080E0B3
:108C700090E0A0E00E94888F09F04AC720E030E031
:108C8000C657DF4F4881CA58D04050E060E070E0DE
:108C900080E090E0A0E00E94888F09F06CC720E09F
:108CA00030E0402F487050E060E070E080E090E0FD
:108CB000A0E00E94888F09F088C720E030E0402FB4
:108CC000407150E060E070E080E090E0A0E00E9441
:108CD000888F09F0AAC720E030E0402F407250E0B2
:108CE00060E070E080E090E0A0E00E94888F09F0F2
:108CF000CCC720E030E0402F407450E060E070E0EE
:108D000080E090E0A0E00E94888F09F0EFC7F02F8C
:108D1000F078BF2E20E030E04F2F50E060E070E0B0
:108D200080E090E0A0E00E94888F11F00C94A74EA4
:108D3000212F2170C22E20E030E040E05C2D60E069
:108D400070E080E090E0A0E00E94888F11F00C9429
:108D5000B44E20E030E04B2D50E060E070E080E069
:108D600090E0A0E00E94888F11F00C94C24E20E0A9
:108D700030E040E05C2D60E070E080E090E0A0E05A
:108D80000E94888F11F00C94F74E20E030E040E014
:108D9000512F527060E070E080E090E0A0E00E940F
:108DA000888F11F00C942C4F20E030E040E0512FE0
:108DB000547060E070E080E090E0A0E00E94888F56
:108DC00011F00C945F4F20E030E040E0512F5071E3
:108DD00060E070E080E090E0A0E00E94888F11F0F9
:108DE0000C94924F20E030E040E0512F507260E050
:108DF00070E080E090E0A0E00E94888F11F00C9479
:108E0000D14F20E030E040E0512F507460E070E03E
:108E100080E090E0A0E00E94888F11F00C94105048
:108E200020E030E040E0512F587060E070E080E0DA
:108E300090E0A0E00E94888F11F00C944F5020E049
:108E400030E040E05D2D60E070E080E090E0A0E088
:108E50000E94888F11F00C948050779A8091C509F8
:108E60009091C60992FD749AC557DF4F2881CB585F
:108E7000D040C457DF4F3881CC58D040A801C357E9
:108E8000DF4F6881CD58D040CD56DF4F7881C35930
:108E9000D040CC56DF4F8881C459D040CB56DF4FED
:108EA0009881C559D040A0E08E010D5F1F4F0E94F0
:108EB000888F11F00C94BC50809156028061898398
:108EC0008091E5098A83F801EE0DFF1D10828091E3
:108ED000C5099091C60987010D5F1F4F80FF0CC027
:108EE0001F930F9387E598E09F938F930E940794B9
:108EF0000F900F900F900F90B801CE0101960E9435
:108F0000155D8091580282FF0AC028EE34E2A80164
:108F1000BE016F5F7F4F81E692E00E94AA6180915F
:108F2000C5099091C60982FD73980E94416981EF3D
:108F300099E00E94E8538091580290915902A091C3
:108F40005A02B0915B0290FF40C03FEFE31AF30A70
:108F50000E943D6AD82E89E10E94556A40915802CC
:108F60005091590260915A0270915B0250FF29C0E2
:108F700073988091E5098F5F8093E5098A83B70133
:108F80006F5F7F4FCE0101960E94155D81EF99E0E2
:108F90000E94E85340E050E065E880910212909111
:108FA00003120E94A35589E590E1CF56DF4FA881B7
:108FB000B981C159D0408D939C9338C0E12CF12CDC
:108FC000CDCF8D2D0E94556A739A8091C2099091E0
:108FD000C309892B11F00E94F9688091E5098F5F20
:108FE0008093E5098091C5099091C60982FF39CC2B
:108FF000739A37CC8DED99E00E944958892BB1F0D6
:109000000E9441698091580287FD2B9860E470E0CE
:109010008DED99E00E94225882E790E1CF56DF4F14
:10902000E881F981C159D0409183808381E00C941B
:109030000151CF56DF4FA881B981C159D0401D924F
:109040001C9283E00C940151623181F7C090580268
:10905000D0905902E0905A02F0905B02D1FC01CC12
:10906000F8018081813091F50180F281E02D20812D
:10907000C557DF4F2883CB58D0403181C457DF4FCD
:109080003883CC58D040028113814481C357DF4FCD
:109090004883CD58D0405581CD56DF4F5883C359B2
:1090A000D0408681CC56DF4F8883C459D040978109
:1090B000CB56DF4F9883C559D04020843184C257A6
:1090C000DF4F19821882CE58D0406AC08230E9F44E
:1090D000A381B481C257DF4FB983A883CE58D04053
:1090E000212C312CB1E0C557DF4FB883CB58D0408D
:1090F000C457DF4F1882CC58D04000E010E8C35767
:10910000DF4F1882CD58D0403CC08330F9F0843016
:1091100009F0A7CB212C312CC257DF4F19821882BE
:10912000CE58D040E5E0C557DF4FE883CB58D0405C
:10913000C457DF4F1882CC58D04000E010E0F2E076
:10914000C357DF4FF883CD58D0401BC0212C312CA2
:10915000C257DF4F19821882CE58D04025E0C5573C
:10916000DF4F2883CB58D040C457DF4F1882CC58EC
:10917000D04000E010E031E0C357DF4F3883CD58D6
:10918000D040CD56DF4F1882C359D040CC56DF4F68
:109190001882C459D040CB56DF4F1882C559D040F1
:1091A00080903F2490904024A0904124B09042248D
:1091B0004090800250908102609082027090830201
:1091C0002DEC3CEC4CE45EE3C301B2010E940D893E
:1091D0009B01AC01C501B4010E94998B87FD0BC0B6
:1091E000E894E0F8C0925802D0925902E0925A02F4
:1091F000F0925B024AC0A3019201C501B4010E9432
:10920000D38987FF42C080914B2490914C24A09138
:109210004D24B0914E240196A11DB11D80934B2485
:1092200090934C24A0934D24B0934E24E0FC19CB92
:109230006894E0F8C0925802D0925902E0925A0223
:10924000F0925B0245E4C557DF4F4883CB58D040CE
:1092500050E2C457DF4F5883CC58D04000E010E0B4
:1092600084E0C357DF4F8883CD58D040CD56DF4FC1
:109270001882C359D040CC56DF4F1882C459D04011
:10928000CB56DF4F1882C559D040902F9470C657E7
:10929000DF4F9883CA58D04020E030E0492F50E09B
:1092A00060E070E080E090E0A0E00E94888F09F02C
:1092B0008C9AC557DF4FA881CB58D040A0727A2E28
:1092C0002A2F30E040E050E060E070E080E090E085
:1092D000A0E00E94888F11F00E943C0BC457DF4F22
:1092E000B881CC58D040B074C057DF4FB883C05954
:1092F000D04020E03B2F40E050E060E070E080E0B4
:1093000090E0A0E00E94888F11F00E940F1FC457C8
:10931000DF4FE881CC58D040E078CA56DF4FE88371
:10932000C659D04020E03E2F40E050E060E070E0C1
:1093300080E090E0A0E00E94888F51F00E94D70A60
:109340006093F5287093F6288093F7289093F82877
:10935000C557DF4F2881CB58D040217030E040E026
:1093600050E060E070E080E090E0A0E00E94888F34
:10937000F1F08EE09BE19F938F938FE696E09F93B1
:109380008F931F9287E78F93CE0103969F938F93BE
:109390000E946A946C010E94AE430FB6F894DEBF3F
:1093A0000FBECDBF892B09F05CCA760102C0E12C4B
:1093B000F12CC557DF4F2881CB58D040227030E0C8
:1093C00040E050E060E070E080E090E0A0E00E94CB
:1093D000888FD1F1C701029667E776E041E050E05F
:1093E0004C0F5D1F840F951F0E946B9353E0E50E99
:1093F000F11C22E0A22E29E2B22E32EFC32E33E07E
:10940000D32E47E7942ED5018D915D011F928F9346
:10941000DF92CF921F929F92C7010296E1E0F0E0A7
:10942000EC0FFD1F8E0F9F1F9F938F930E946A94D6
:10943000E80EF91E0FB6F894DEBF0FBECDBF3AE0BE
:10944000A31639E2B306F9F6C557DF4F2881CB588A
:10945000D040247030E040E050E060E070E080E018
:1094600090E0A0E00E94888F09F447C0C7010296EF
:109470006BE776E041E050E04C0F5D1F840F951FD5
:109480000E946B9354E0E50EF11C4E018AE7880EB2
:10949000911C80E1D4011D928A95E9F728E0A4018E
:1094A00068E980EB0E94CE115401B8E0AB0EB11C0C
:1094B00082EFC82E83E0D82E97E7692EF4018191C0
:1094C0004F011F928F93DF92CF921F926F92C7012D
:1094D000029621E030E02C0F3D1F820F931F9F93D7
:1094E0008F930E946A94E80EF91E0FB6F894DEBFBF
:1094F0000FBECDBF8A149B0409F7512F5078D52E8B
:1095000020E030E040E060E070E080E090E0A0E04B
:109510000E94888FE1F48091C2099091C3099F93C2
:109520008F9380E896E09F938F931F9287E78F93A6
:10953000CE018E0D9F1D03969F938F930E946A9478
:10954000E80EF91E0FB6F894DEBF0FBECDBF20E0C7
:1095500030E040E050E0C357DF4F6881CD58D04045
:10956000617070E080E090E0A0E00E94888F09F4D4
:1095700087C9E3E0F0E0EC0FFD1FEE0DFF1D80E278
:109580008083EBE6F4E2808197012F5F3F4F790102
:10959000882309F469C98081A1E0B0E0AC0FBD1F48
:1095A000AE0DBF1D12968C933196EDCFCE018E0D70
:1095B0009F1D67E876E003960E946B9397E0E90EA3
:1095C000F11CC7010E94AE43892B09F04AC96AC940
:1095D0002114310409F4A8CAF8944090E828509066
:1095E000E9286090EA287090EB2878948091781BA5
:1095F0009091791BA0917A1BB0917B1BA3019201E2
:10960000281B390B4A0B5B0BCA01B9010E94748AF3
:109610004B015C01B10180E090E00E94748A9B01E3
:10962000AC01C501B4010E94D789B82EC92E9F9301
:109630008F937F936F938BEC96E09F938F931F9202
:1096400087E78F939E012E0D3F1D2D5F3F4F3F9368
:109650002F93C856DF4F6883C859D040C956DF4F93
:109660007883C759D0400E946A94E80EF91EC85604
:10967000DF4F6881C859D040C956DF4F7881C7593C
:10968000D040862F972FAB2DBC2D8093FA28909336
:10969000FB28A093FC28B093FD284092781B5092A1
:1096A000791B60927A1B70927B1B0FB6F894DEBF19
:1096B0000FBECDBF39CA2114310409F447CAF8944A
:1096C00080914F1B9091501BA091511BB091521B48
:1096D00078949F938F9380915F028F9380915E0225
:1096E0008F9388ED96E09F938F931F9287E78F93D8
:1096F000C7010296A1E0B0E0AC0FBD1F8A0F9B1F0F
:109700009F938F930E946A94E80EF91E0FB6F89407
:10971000DEBF0FBECDBF1ACAF8948091EC2890919D
:10972000ED28A091EE28B091EF287894BF93AF93E5
:109730009F938F9388EE96E09F938F931F9287E776
:109740008F93C701029621E030E02C0F3D1F820F5E
:10975000931F9F938F930E946A94E80EF91EC7018E
:109760000E94AE430FB6F894DEBF0FBECDBF892B6B
:1097700009F077C8FDC92114310409F40BCAF89423
:109780004090EC285090ED286090EE287090EF28E3
:10979000789480917C1B90917D1BA0917E1BB09151
:1097A0007F1BA3019201281B390B4A0B5B0BCA01DB
:1097B000B9010E94748A4B015C01B10180E090E024
:1097C0000E94748A9B01AC01C501B4010E94D78933
:1097D000B82EC92E9F938F937F936F9383EF96E05C
:1097E0009F938F931F9287E78F939E012E0D3F1DAE
:1097F0002D5F3F4F3F932F93C856DF4F6883C85963
:10980000D040C956DF4F7883C759D0400E946A9430
:10981000E80EF91EC856DF4F6881C859D040C956B6
:10982000DF4F7881C759D040862F972FAB2DBC2DA5
:109830008093FE289093FF28A0930029B0930129DC
:1098400040927C1B50927D1B60927E1B70927F1B0E
:109850000FB6F894DEBF0FBECDBF9CC9232809F414
:10986000ABC9F8948091531B9091541BA091551B48
:10987000B091561B78949F938F9380915D028F9344
:1098800080915C028F9380E097E09F938F931F926B
:1098900087E78F93C7010296A1E0B0E0AC0FBD1F30
:1098A0008A0F9B1F9F938F930E946A94E80EF91E64
:1098B0000FB6F894DEBF0FBECDBF7EC980914324A2
:1098C00090914424A0914524B0914624BF93AF9336
:1098D0009F938F9380E197E09F938F931F9287E7E9
:1098E0008F93C701029621E030E02C0F3D1F820FBD
:1098F000931F9F938F930E946A94E80EF91EC701ED
:109900000E94AE430FB6F894DEBF0FBECDBF892BC9
:1099100011F00C94314462C980914E248F93809150
:109920004D248F9380914C248F9380914B248F935F
:1099300080914A248F93809149248F938091482469
:109940008F93809147248F938BE197E09F938F9320
:109950001F92B7E7CB2ECF92C7010296A1E0B0E0ED
:10996000AC0FBD1F8A0F9B1F9F938F930E946A9419
:10997000E80EF91EC7010E94AE430FB6F894DEBF91
:109980000FBECDBF892B11F00C94314480913D2046
:1099900090913E2090FF34C9809152248F93809102
:1099A00051248F93809150248F9380914F248F93D3
:1099B0008FE397E09F938F931F92CF92C7010296F8
:1099C00021E030E02C0F3D1F820F931F9F938F9358
:1099D0000E946A94E80EF91EC7010E94AE430FB6BA
:1099E000F894DEBF0FBECDBF892B11F00C9431442B
:1099F00007C98091341C8F938091331C8F93809181
:109A0000321C8F938091311C8F9381E597E09F9357
:109A10008F931F9287E78F93C7010296A1E0B0E072
:109A2000AC0FBD1F8A0F9B1F9F938F930E946A9458
:109A3000E80EF91EC7010E94AE430FB6F894DEBFD0
:109A40000FBECDBF892B11F00C943144EAC8809130
:109A5000F8288F938091F7288F938091F6288F9321
:109A60008091F5288F938CE597E09F938F931F92B9
:109A700087E78F93C701029621E030E02C0F3D1F4E
:109A8000820F931F9F938F930E946A94E80EF91E92
:109A9000C7010E94AE430FB6F894DEBF0FBECDBF24
:109AA000892B11F00C943144CDC881E00E94880AC2
:109AB000209178023091790240917A0250917B0294
:109AC0000E94588C9F938F937F936F9389E697E0C2
:109AD0009F938F931F9287E78F93C7010296A1E010
:109AE000B0E0AC0FBD1F8A0F9B1F9F938F930E9406
:109AF0006A94E80EF91EC7010E94AE430FB6F894AF
:109B0000DEBF0FBECDBF892B11F00C943144A8C825
:109B100082E00E94880A209174023091750240917F
:109B20007602509177020E94588C9F938F937F9377
:109B30006F9386E797E09F938F931F9287E78F93AA
:109B4000C701029621E030E02C0F3D1F820F931FCA
:109B50009F938F930E946A94E80EF91EC7010E949A
:109B6000AE430FB6F894DEBF0FBECDBF892B11F008
:109B70000C94314483C883E00E94880A9F938F939A
:109B80007F936F9383E897E09F938F931F9287E76C
:109B90008F93C7010296A1E0B0E0AC0FBD1F8A0F02
:109BA0009B1F9F938F930E946A94E80EF91E8C98D6
:109BB000C7010E94AE430FB6F894DEBF0FBECDBF03
:109BC000892B11F00C9431446AC880913D2087FFA5
:109BD00074C821E042E161E080ED0E94DD629F9364
:109BE0008F937F936F9380E997E09F938F931F925A
:109BF00087E78F93C701029621E030E02C0F3D1FCD
:109C0000820F931F9F938F930E946A94E80EF91E10
:109C1000C7010E94AE430FB6F894DEBF0FBECDBFA2
:109C2000892B11F00C94314448C880913D2087FF66
:109C300052C821E042E162E080ED0E94DD629F9324
:109C40008F937F936F938EE997E09F938F931F92EB
:109C500087E78F93C7010296A1E0B0E0AC0FBD1F6C
:109C60008A0F9B1F9F938F930E946A94E80EF91EA0
:109C7000C7010E94AE430FB6F894DEBF0FBECDBF42
:109C8000892B11F00C94314426C880913D2087FF28
:109C900030C821E042E163E080ED0E94DD629F93E5
:109CA0008F937F936F938CEA97E09F938F931F928C
:109CB00087E78F93C701029621E030E02C0F3D1F0C
:109CC000820F931F9F938F930E946A94E80EF91E50
:109CD000C7010E94AE430FB6F894DEBF0FBECDBFE2
:109CE000892B11F00C9431440C94794680913D20DD
:109CF00087FF0DC821E042E164E080ED0E94DD6253
:109D00009F938F937F936F938AEB97E09F938F93AB
:109D10001F9287E78F93C7010296A1E0B0E0AC0FD6
:109D2000BD1F8A0F9B1F9F938F930E946A94E80E1A
:109D3000F91EC7010E94AE430FB6F894DEBF0FBEF6
:109D4000CDBF892B11F00C9431440C94874680913F
:109D50003D2082FD02C00C94984646E061E083E01D
:109D60000E948A130C94984680913D2082FD02C087
:109D70000C94A94621E046E061E083E00E948A134A
:109D80000C94A94680913D2082FD02C00C94B746F8
:109D90008091271C8F938091261C8F938091251C86
:109DA0008F938091241C8F9388EC97E09F938F93DF
:109DB0001F9287E78F93C701029641E050E04C0F56
:109DC0005D1F840F951F9F938F930E946A94E80EE6
:109DD000F91EC7010E94AE430FB6F894DEBF0FBE56
:109DE000CDBF892B11F00C9431440C94B74680916F
:109DF0003D2082FD02C00C94C54680912B1C8F93A0
:109E000080912A1C8F938091291C8F938091281C0C
:109E10008F9380ED97E09F938F931F9287E78F93A7
:109E2000C7010296E1E0F0E0EC0FFD1F8E0F9F1FCF
:109E30009F938F930E946A94E80EF91EC7010E94B7
:109E4000AE430FB6F894DEBF0FBECDBF892B11F025
:109E50000C9431440C94C54680913D2090913E2055
:109E600090FD02C00C94D44680E090E00E94861ED3
:109E70009F938F937F936F938BED97E09F938F9337
:109E80001F9287E78F93C701029641E050E04C0F85
:109E90005D1F840F951F9F938F930E946A94E80E15
:109EA000F91EC7010E94AE430FB6F894DEBF0FBE85
:109EB000CDBF892B11F00C9431440C94D446809181
:109EC0003D2090913E2090FD02C00C94E34681E03D
:109ED00090E00E94861E9F938F937F936F938BEEEB
:109EE00097E09F938F931F9287E78F93C701029606
:109EF000E1E0F0E0EC0FFD1F8E0F9F1F9F938F930B
:109F00000E946A94E80EF91EC7010E94AE430FB684
:109F1000F894DEBF0FBECDBF892B11F00C943144F5
:109F20000C94E34680913D2090913E2090FD02C02C
:109F30000C94F24681E090E00E94861E4B015C0189
:109F400080E090E00E94861E9B01AC01C501B40137
:109F50000E94871C9F938F937F936F938CEF97E062
:109F60009F938F931F9287E78F93C701029641E0DB
:109F700050E04C0F5D1F840F951F9F938F930E949D
:109F80006A94E80EF91EC7010E94AE430FB6F8941A
:109F9000DEBF0FBECDBF892B11F00C9431440C9461
:109FA000F24680913D2090913E2090FD02C00C949D
:109FB000014781E090E00E94861E4B015C0180E039
:109FC00090E00E94861E9B01AC01C501B4010E9475
:109FD000E81C9F938F937F936F9387E098E09F9304
:109FE0008F931F9287E78F93C7010296E1E0F0E01D
:109FF000EC0FFD1F8E0F9F1F9F938F930E946A94FB
:10A00000E80EF91EC7010E94AE430FB6F894DEBFFA
:10A010000FBECDBF892B11F00C9431440C94014735
:10A0200080913D2090913E2090FD02C00C941047FD
:10A0300081E090E00E94861E4B015C0180E090E090
:10A040000E94861E9B01AC01C501B4010E94491DFE
:10A050009F938F937F936F9385E198E09F938F9366
:10A060001F9287E78F93C701029641E050E04C0FA3
:10A070005D1F840F951F9F938F930E946A94E80E33
:10A08000F91EC7010E94AE430FB6F894DEBF0FBEA3
:10A09000CDBF892B11F00C9431440C941047809162
:10A0A0003D2090913E2091FD02C00C941F470E94DC
:10A0B000D4179F938F937F936F9388E298E09F9339
:10A0C0008F931F9287E78F93C7010296E1E0F0E03C
:10A0D000EC0FFD1F8E0F9F1F9F938F930E946A941A
:10A0E000E80EF91EC7010E94AE430FB6F894DEBF1A
:10A0F0000FBECDBF892B11F00C9431440C941F4737
:10A10000C257DF4FA881B981CE58D04016968C91A6
:10A1100016971F928F9315968C9115971F928F9378
:10A1200013968C9113971F928F9312968C911F9276
:10A130008F9389E398E09F938F931F9287E78F9384
:10A14000C7010296E1E0F0E0EC0FFD1F8E0F9F1FAC
:10A150009F938F930E946A94E80EF91EC7010E9494
:10A16000AE430FB6F894DEBF0FBECDBF892B11F002
:10A170000C9431440C942D478091C5099091C609E7
:10A1800082FD0CC08091580280FD08C081FD02C094
:10A190000C945C471D9902C00C945C471F930F936D
:10A1A00080E598E09F938F930E94079480917302BB
:10A1B0000F900F900F900F90882311F40C945C4730
:10A1C0001F928F938CE69FE09F938F930E94199428
:10A1D0000F900F900F900F900C945C478DED99E0CD
:10A1E0000E944958892B11F40C9416480E94F96872
:10A1F0008091580287FD02C00C9431442B9A0C9434
:10A200003144C856DF4F0FB6F894DEBF0FBECDBF46
:10A21000DF91CF911F910F91FF90EF90DF90CF9042
:10A22000BF90AF909F908F907F906F905F904F9076
:10A230003F902F9008950C940F544F925F926F921D
:10A240007F928F929F92AF92BF92CF92DF92EF92C6
:10A25000FF920F931F93CF93DF93CDB7DEB7609735
:10A260000FB6F894DEBF0FBECDBF6B010E943D6AF2
:10A27000E82FF0E0EE0FFF1FEF5BF44E808191813D
:10A280000196918380838091C5099091C60981FDD3
:10A2900074988090580290905902A0905A02B09001
:10A2A0005B020E94695C7C01FC018081982F929581
:10A2B0009F70913099F48F7051F48091251B90918B
:10A2C000261B01969093261B8093251B07C1B60180
:10A2D00082E199E20E948553892B51F08091231BE2
:10A2E0009091241B01969093241B8093231BF6C00E
:10A2F000D501C4011EE0B695A795979587951A9547
:10A30000D1F7F82FF1708F2E8CEF99E00E949056C4
:10A310008C01009709F448C0B601C80102960E945A
:10A320008553892BE9F198014AEC59E060E074E625
:10A33000C8010F960E941059F7019181F80184819C
:10A34000981321C082858F5F82878091211B909115
:10A35000221B01969093221B8093211B84E00E9474
:10A36000865DF801208530E02817390708F0A9C17B
:10A3700084E00E94865DF8018087F70180818F70FC
:10A38000F8018187ABC0F801128684E00E94865DE7
:10A39000F8018087F70180818F70F801818792C171
:10A3A000C8010E943857B4CF84E092E00E9425563D
:10A3B0008C01009709F492C0B601C80102960E9470
:10A3C0007C53F70181818150F801848380E091E022
:10A3D000A0E0B0E083879487A587B687128684E0E3
:10A3E0000E94865DF8018087F70180818F70F801F7
:10A3F0008187B8018CEF99E00E94F05698014AECF1
:10A4000059E060E074E6C8010F960E941059992443
:10A410009394F7018181F8018483F70180818F7023
:10A42000F801878384E00E94865DF801858383E0DC
:10A430000E94865D5C01F801868387818F3009F078
:10A44000912CF7014180F8018481481A512C612C2C
:10A45000712C76E0440C551C661C771C7A95D1F75C
:10A460002385348545855685A0ECB0E00E94BC8DDF
:10A47000BB27A92F982F872F480E591E6A1E7B1EB7
:10A4800043865486658676868091C5099091C60973
:10A4900081FD2EC08091580280FD2AC081FD26C01A
:10A4A0008091580290915902A0915A02B0915B029A
:10A4B00097FDD2C0992091F082E0809354241092AD
:10A4C000562410925524109358240093572444E5A1
:10A4D00054E262E184E392E00E94A3558091C509B1
:10A4E0009091C60981FFF0C0749AEEC01D9BD8CF31
:10A4F000A4E6B0E0A30192010E94BC8D672F782FE3
:10A50000892F992724E630E040E050E00E94508DEA
:10A510007F936F93452C562C672C77245F924F9234
:10A52000BB24BF92AF92F80185811F928F93F701F0
:10A5300080818F701F928F9381811F928F93F6017C
:10A5400081811F928F9380811F928F93C701029602
:10A550009F938F9388E698E09F938F930E94079430
:10A56000809173020FB6F894DEBF0FBECDBF882373
:10A5700061F01F928F9389E69FE09F938F930E94D3
:10A5800019940F900F900F900F9080915802909116
:10A590005902A0915A02B0915B0296FF2DC088200B
:10A5A00059F1F7012081322F3F70832F90E00297FD
:10A5B000D4F08FEF830F207F822B808381EF99E08F
:10A5C0000E941B5180911F1B9091201B019690931C
:10A5D000201B80931F1B8091C5099091C60996FF8F
:10A5E0000BC0739809C08091251B9091261B019682
:10A5F0009093261B8093251B80913D2086FF50CF92
:10A600000E942C62C70105960E94F861F7018181C2
:10A610001F928F93F80186811F928F9385811F92DD
:10A620008F938CEA98E09F938F931F9280E18F9392
:10A630009E012F5F3F4F6901DF922F930E946A9422
:10A6400082E00E941262C6010E94F8610FB6F8947F
:10A65000DEBF0FBECDBF24CF8EE09BE120910E1B4D
:10A66000222309F427CF9F938F938FEB98E09F933A
:10A670008F93FE0131966F01DF92EF930E94A794B2
:10A680005C01B601C70102960E948C930F900F9057
:10A690000F900F900F900F90009709F40BCF95013A
:10A6A0002F5F3F4F280F391FA9012F5F3F4FFA013E
:10A6B00080818032C9F362E18CE092E00E94A35570
:10A6C000F9CE812C912CA5CE60960FB6F894DEBF02
:10A6D0000FBECDBFDF91CF911F910F91FF90EF90F3
:10A6E000DF90CF90BF90AF909F908F907F906F90B2
:10A6F0005F904F9008950895FB012081FC01208315
:10A70000FB012181FC0121830895FC019081DB0183
:10A710008C91981309C081E090E0318111962C91C1
:10A72000321721F080E0089580E090E00895BC01A8
:10A7300082E199E20C947C53DC011996ED91FC9135
:10A740001A970280F381E02D309709F0099408955B
:10A750000F931F93CF93DF9300D0CDB7DEB78C015B
:10A7600088E10E94995DBC01CE0101960E947C5354
:10A77000D8011996ED91FC911A970190F081E02D86
:10A78000BE016F5F7F4FC80109950F900F90DF9159
:10A79000CF911F910F910895EF92FF920F931F9306
:10A7A000CF93DF93EC018B017A0142E053E00E94EA
:10A7B000F553FA86E98666E073E0C801DF91CF9130
:10A7C0001F910F91FF90EF900C944E540C940D54E8
:10A7D000CF93DF93EC0162E179E288E10E948F5D23
:10A7E000CE01DF91CF910C940F54EF92FF920F9313
:10A7F0001F93CF93DF93EC018B017A010E942A54BF
:10A80000F886EF826AE073E0C801DF91CF911F9173
:10A810000F91FF90EF900C944E540C9432540C9482
:10A82000B76EDC011796ED91FC9118970190F081BD
:10A83000E02D0994DC011796ED91FC9118970280A8
:10A84000F381E02D309709F00994089580E092E1BA
:10A850000C948C56FC0173836283BC0180E092E10E
:10A860000C94F056BC0180E092E10C94D556CF9345
:10A87000DF93EC0180E092E10E949056009749F04E
:10A88000FC01228133812C173D0729F00E943857A3
:10A89000F5CF80E090E0DF91CF9108950F931F9363
:10A8A000CF93DF938B010E943754EC01009731F076
:10A8B0001D830C83C8010E94E8708E83DF91CF91C5
:10A8C0001F910F9108951F93CF93DF93EC01162FE3
:10A8D000EC81FD813097D1F09093031280930212A6
:10A8E00082E08887CE0106960995992787FD909585
:10A8F0000297029710F0133839F4BE01CE01DF91B0
:10A90000CF911F910C94905481E08887DF91CF9173
:10A910001F910895FC01208520FD0C946354089537
:10A92000CF92DF92EF92FF920F931F93CF93DF931B
:10A93000EC016B01E0900212F090031200910412FE
:10A9400010910512F801EC17FD0739F0309709F462
:10A950004AC00190F081E02DF6CF209709F443C062
:10A960008885882309F118860115110561F0C01743
:10A97000D10729F0AE0167E8C8010E948A54F801A6
:10A9800000811181F1CFEC81FD81309769F0CC1508
:10A99000DD0551F0D0930312C093021240E050E065
:10A9A00063E8CE0106960995E0910412F091051234
:10A9B000CE17DF0769F488819981909305128093FF
:10A9C00004120DC0808191818C179D0721F0FC013C
:10A9D0003097C1F704C08881998191838083F09278
:10A9E0000312E0920212DF91CF911F910F91FF901D
:10A9F000EF90DF90CF9008951F93CF93DF93109245
:10AA00000E12C0910412D091051211E0209779F036
:10AA10008985882341F01887198640E050E062E874
:10AA2000CE010E9463540990D881C02DEFCFDF91F1
:10AA3000CF911F9108958091B11291E0980F90935A
:10AA4000B112089560910212709103120C94905407
:10AA50008AE88093B1121092AF121092B012109245
:10AA6000051210920412109203121092021208950D
:10AA700080910E1281110E94FC547091B0127723C4
:10AA800009F451C0E091AF122E2F30E085E0E89F2D
:10AA9000F0011124E15FFD4E608160930D12418150
:10AAA000528150930C1240930B12838194819093A6
:10AAB0000A12809309122F5F3F4F2F713327209383
:10AAC000AF1271507093B012009731F5809104125B
:10AAD00090910512909308128093071280910712AB
:10AAE00090910812892BF9F080910E1281110E9429
:10AAF000FC5440910B1250910C1260910D128091F8
:10AB00000712909108120E948A54E0910712F09166
:10AB1000081280819181DECF613819F421E0FC01B7
:10AB200020870E948A5480910E122091B01290E0EA
:10AB3000820F911D089580910E122091B01290E025
:10AB4000820F911D08952091B0122032B9F0E0914A
:10AB5000AF12E20FEF71E093061235E0E39FF001D0
:10AB60001124E15FFD4E608352834183948383838C
:10AB70002F5F2093B01280E090E0089581E090E094
:10AB80000895CF93DF93C0910212D09103120E94D7
:10AB90008A54D0930312C0930212DF91CF9108958B
:10ABA000AB013091041220910512E32FF22FE81728
:10ABB000F907B1F0309721F00190F081E02DF7CF47
:10ABC000009771F0FC0130832183909305128093EC
:10ABD000041221E020871782168261E80C94C15587
:10ABE0000895009749F0FC0120852150223020F47F
:10ABF00021E0218720930E12089521E030E0FC012E
:10AC00008085811102C020E030E0C9010895CF9312
:10AC1000DF93EC014A815B8160E070E08C819D8173
:10AC20000E945B932A813B8188819981289FA001A2
:10AC3000299F500D389F500D112460E070E08E81E7
:10AC40009F81DF91CF910C945B93FC018281938172
:10AC500020E030E028173907D1F0A481B581A20F98
:10AC6000B31F4C91411110C081E08C938081918180
:10AC7000289FA001299F500D389F500D11248681D7
:10AC80009781840F951F08952F5F3F4FE3CF80E09A
:10AC900090E00895FC01268137814281538180E054
:10ACA00090E084179507C9F02617370781F4A4812F
:10ACB000B581A80FB91F2C91121614F421502C93B2
:10ACC0000480F581E02DE80FF91F80810895A081AF
:10ACD000B1812A0F3B1F0196E4CF8FEF0895FC014D
:10ACE0008681978168177907A0F0A081B1814281A0
:10ACF0005381A49F9001A59F300DB49F300D112466
:10AD0000280F391F81E090E06217730720F080E080
:10AD1000089580E090E00895FC011182108208956A
:10AD2000FC01808191810895FB0120813181FC012A
:10AD3000318320830895DC01ED91FC91309731F04F
:10AD400080819181009729F0FC01FACF80E090E0AA
:10AD50000895CF010895DC01ED91FC911197309792
:10AD6000A9F020813181232B21F41D921C92CF0167
:10AD70000895A081B1818D919C911197892B11F03B
:10AD8000FD01F7CF11821082CD01089580E090E09F
:10AD90000895DC01ED91FC911197309721F020810D
:10ADA00031812D933C93CF010895DC01ED91FC910D
:10ADB0003097A9F0A0E0B0E020813181E617F707D5
:10ADC00041F4109709F4DC012D933C931182108219
:10ADD00008952115310519F0DF01F901EDCF08952E
:10ADE0000F931F93CF93DF938C01EB010E94D556F5
:10ADF00019821882C8010E949B56009711F4F8012D
:10AE000001C0FC01D183C083DF91CF911F910F91CD
:10AE100008950F931F93CF93DF93EC018B010E9452
:10AE2000D55688819981F80191838083198308839D
:10AE3000DF91CF911F910F910895DC01ED91FC916D
:10AE400080E090E0309729F001960190F081E02DAC
:10AE5000F9CF0895FB01309719F4BA010C94095702
:10AE600080819181DA018D939C9351834083089571
:10AE7000009721F0FC0180819181089580E090E0AD
:10AE800008958091B4129091B512892B29F41092F3
:10AE9000B3121092B21208950E944466E091B41267
:10AEA000F091B5122281338140815181240F351FE9
:10AEB000281B390B0480F581E02D309769F0428121
:10AEC000538160817181460F571F481B590B4217F0
:10AED000530780F79A01EECF280F391F3093B31232
:10AEE0002093B212089586E892E00C94F155EF9207
:10AEF000FF920F931F93CF93DF938C01FC0180810E
:10AF00009181009799F08A359105D9F0F801118265
:10AF1000108283E068C0868197818417950709F0C5
:10AF200049C00480F581E02D3097A9F71092B51241
:10AF30001092B4128AE590E0F8019183808381E059
:10AF400052C0673891F16238A9F7C091B412D0911C
:10AF5000B512E12CF12C209769F3CE010E94B9744F
:10AF6000892BF1F0AE0168E88E819F810E94A35584
:10AF7000892BA1F41F821E828C819D81E114F10432
:10AF800021F0F7019583848304C09093B5128093D8
:10AF9000B4121D821C820E944157D7CF0E94735762
:10AFA0007E010C80DD81C02DD6CFE091B412F091EE
:10AFB000B512BACFF093B512E093B412A481B58163
:10AFC000109709F4B7CF16968D919C911797841717
:10AFD000950711F0FD01F2CF14968D919C91159774
:10AFE00095838483EBCFDF91CF911F910F91FF90D9
:10AFF000EF900895CF93DF93EC010E9473578E81F9
:10B000009F813091B4122091B512892B59F0E32F12
:10B01000F22F309739F0EC17FD0781F00480F581AD
:10B02000E02DF7CF80910212909103129F838E83BF
:10B030003C832D83D093B512C093B412DF91CF918E
:10B040000C944157CF93DF93EC010E949974CE0189
:10B05000DF91CF910C94FA57CF93DF93EC010E94CC
:10B06000A574CE01DF91CF910C94FA57CF93DF9363
:10B07000EC010E94AF74CE01DF91CF910C94FA578E
:10B08000FC0120813181260F371F318320830C94EE
:10B09000415721E030E0FC0186819781892B11F036
:10B0A00020E030E0C9010895FC01228133818081D4
:10B0B0009181820F931F0895FC01808191810895F1
:10B0C00081E090E02091B4123091B512232B11F45D
:10B0D00080E090E008958091B4129091B512892B90
:10B0E00029F08091B2129091B312089580E090E01F
:10B0F0000895CF93DF93EC01E091B412F091B51273
:10B100008E179F0769F48C819D819093B51280936F
:10B11000B4120DC0848195818C179D0721F0FC012C
:10B120003097C1F706C08C819D81958384830E94EE
:10B1300041571D821C821F821E82DF91CF9108958C
:10B14000EF92FF920F931F93CF93DF938C017A01BD
:10B15000FC0180819181009741F08B34910501F1D0
:10B16000F8011182108283E048C087EB92E10E94CF
:10B170009056EC01209751F06C817D81CE010296B2
:10B180000E9422580990D881C02DF4CF81E080938D
:10B19000B6128BE490E0F8019183808381E02DC0AA
:10B1A0006838E1F787EB92E10E949056EC01209716
:10B1B00081F3CE010296E816F906D9F4BE0187EBB9
:10B1C00092E10E94D556E0900212F09003128A8517
:10B1D0009B859093031280930212EC85FD85309736
:10B1E00019F08E859F850995F0920312E092021264
:10B1F000D0CF0990D881C02DDACFDF91CF911F91A8
:10B200000F91FF90EF9008951092B61287EB92E1A4
:10B210000E948C5660E070E080E992E00C94D0557A
:10B220000F931F93CF93DF93EC01009102121091C3
:10B2300003121B870A875D874C873F872E87809183
:10B24000B612882379F080E992E0909303128093FC
:10B250000212CE0102960E9422581093031200930C
:10B26000021202C07D836C83BE0187EB92E10E94D3
:10B27000D556BE0187EB92E1DF91CF911F910F91DF
:10B280000C94F0560F931F93CF93DF93EC018091B2
:10B29000B612882391F0009102121091031280E9F6
:10B2A00092E09093031280930212CE0102960E94C4
:10B2B0002C581093031200930212BE0187EB92E107
:10B2C0000E94D556BE0187EB92E1DF91CF911F918D
:10B2D0000F910C94F0560F931F93CF93DF93EC01D3
:10B2E0008091B612882391F00091021210910312FE
:10B2F00080E992E09093031280930212CE010296AD
:10B300000E9436581093031200930212BE0187EB7D
:10B3100092E10E94D556BE0187EB92E1DF91CF9179
:10B320001F910F910C94F056CF93DF93EC01809115
:10B33000B612882329F0CE0102960E94795804C0E3
:10B340001F821E8219861886BE0187EB92E1DF916B
:10B35000CF910C94D556CF93DF93EC018091B61228
:10B36000882331F0CE010296DF91CF910C94495899
:10B3700087EB92E10E949056009739F08C179D0759
:10B3800039F0FC0180819181F7CF81E090E002C02B
:10B3900080E090E0DF91CF9108952F923F924F92FD
:10B3A0005F926F927F928F929F92AF92BF92CF9255
:10B3B000DF92EF92FF920F931F93CF93DF93CDB75E
:10B3C000DEB7E8970FB6F894DEBF0FBECDBFE9E455
:10B3D000FBE22081318142815381E5E4FBE2508030
:10B3E000418032802380E1E4FBE280818983918186
:10B3F0009A83A281AB836380EDE3FBE2B081BC83DF
:10B4000081818D8392819E83A381AF83E9E3FBE2F7
:10B41000B081B8878181898792819A87A381AB8720
:10B42000E5E3FBE2B081BC8781818D8792819E87B5
:10B43000A381AF87E1E3FBE2B081B88B8181898B87
:10B4400092819A8BA381AB8BEDE2FBE2B081BC8B46
:10B4500081818D8B92819E8BA381AF8BE9E2FBE290
:10B46000B081B88F8181898F92819A8FA381AB8FB0
:10B47000E5E2FBE2B081BC8F81818D8F92819E8F4E
:10B48000A381AF8FE1E2FBE2B081B8A3818189A300
:10B4900092819AA3A381ABA3EDE1FBE2B081BCA3AF
:10B4A00081818DA392819EA3A381AFA3E9E1FBE2F9
:10B4B000B081B8A7818189A792819AA7A381ABA700
:10B4C000E5E1FBE2B081BCA781818DA792819EA7B7
:10B4D000A381AFA7E1E1FBE2B081B8AB818189AB89
:10B4E00092819AAB7380EDE0FBE2B080A180928004
:10B4F0008380E9E0FBE2F080E180D280C380E5E078
:10B50000FBE2A081AFABB181B8AF128103812BAB5D
:10B510003CAB4DAB5EAB0E9472665EA95F934DA9DA
:10B520004F933CA93F932BA92F932F923F924F9279
:10B530005F926F922B812F932A812F9329812F93D2
:10B540002F812F932E812F932D812F932C812F9339
:10B550002B852F932A852F9329852F9328852F9329
:10B560002F852F932E852F932D852F932C852F9309
:10B570002B892F932A892F9329892F9328892F93F9
:10B580002F892F932E892F932D892F932C892F93D9
:10B590002B8D2F932A8D2F93298D2F93288D2F93C9
:10B5A0002F8D2F932E8D2F932D8D2F932C8D2F93A9
:10B5B0002BA12F932AA12F9329A12F9328A12F9359
:10B5C0002FA12F932EA12F932DA12F932CA12F9339
:10B5D0002BA52F932AA52F9329A52F9328A52F9329
:10B5E0002FA52F932EA52F932DA52F932CA52F9309
:10B5F0007F922AA92F9329A92F9328A92F938F925D
:10B600009F92AF92BF92CF92DF92EF92FF920F93F1
:10B610001F9328AD2F932FA92F939F938F937F93E1
:10B620006F93A3E1B9E28C911F928F93E2E1F9E26B
:10B6300080811F928F9384EE9FE09F938F930E944F
:10B640001994E9E7FBE22081318142815381E5E7EA
:10B65000FBE25080418032802380E9E6FBE290806B
:10B66000818072806380E5E6FBE28081898391813D
:10B670009A83A281AB83B381BC83E1E6FBE2808144
:10B680008D8391819E83A281AF83B381B887EDE5DD
:10B69000FBE28081898791819A87A281AB87B38100
:10B6A000BC87E9E5FBE280818D8791819E87A2813D
:10B6B000AF87B381B88BE5E5FBE28081898B91810F
:10B6C0009A8BB280A380E1E5FBE2F080E180D2803A
:10B6D000C380EDE4FBE2A081AB8BB181BC8B128116
:10B6E00003810FB6F894DEBF0FBECDBF2BAB3CABD2
:10B6F0004DAB5EAB0E9472665EA95F934DA94F93FE
:10B700003CA93F932BA92F932F923F924F925F9288
:10B710006F927F928F929F922C812F932B812F93E8
:10B720002A812F9329812F9328852F932F812F935F
:10B730002E812F932D812F932C852F932B852F9343
:10B740002A852F9329852F9328892F932F852F932F
:10B750002E852F932D852F93AF92BF922A892F93F9
:10B7600029892F93CF92DF92EF92FF920F931F932D
:10B770002C892F932B892F939F938F937F936F9374
:10B78000A3E1B9E28C911F928F93E2E1F9E280810B
:10B790001F928F9385E79FE09F938F930E94199448
:10B7A0000FB6F894DEBF0FBECDBFE8960FB6F89483
:10B7B000DEBF0FBECDBFDF91CF911F910F91FF90E4
:10B7C000EF90DF90CF90BF90AF909F908F907F9041
:10B7D0006F905F904F903F902F90089580E38093FB
:10B7E0006D130895CF93DF9360916D1370E0C0E304
:10B7F000D0E0C61BD70B65547D4EAE010E9452931C
:10B80000CE01DF91CF910895CF92DF92EF92FF9218
:10B810000F931F93CF93DF937C01C0907013D09050
:10B82000711360916D1370E0E601E096C61BD70BB3
:10B83000C138D105D8F400E310E0061B170B65549E
:10B840007D4EA8010E9452936091B9127091BA1274
:10B8500080916E1390916F13680F791FA601C70135
:10B86000800F911F0E945293CE0102C080E090E0B1
:10B87000DF91CF911F910F91FF90EF90DF90CF90CC
:10B88000089590916D13980F90936D1308954091C2
:10B890007013509171134817590798F020916E1347
:10B8A00030916F13280F391F30936F1320936E134D
:10B8B000481B590B509371134093701381E090E033
:10B8C000089580E090E00895909371138093701331
:10B8D000089580916E1390916F1385519D4E089538
:10B8E00080916D1390E085549D4E089581E090E025
:10B8F0002091B9123091BA122B5E324111F480E0DE
:10B9000090E008950E94765C892B61F06091B912F5
:10B910007091BA1240917013509171138BEE92E1B5
:10B920000C94529320916E1330916F1321153105B1
:10B93000B9F08091701390917113C096EBEEF2E123
:10B94000AF014B5B52414817590734F4DF01A20F96
:10B95000B31F4C914193F4CF10926F1310926E135A
:10B9600008958091B9129091BA1208958091701340
:10B9700090917113089590916D1380E3891B089540
:10B9800020E380916D13281B8091701390917113A7
:10B99000820F911D08951F93CF93DF93EC011091B7
:10B9A0006D13812F90E08C179D076CF00E94C05C96
:10B9B0008C0F9D1F8138910530F41C1B10936D1363
:10B9C00081E090E002C080E090E0DF91CF911F9194
:10B9D0000895CF93DF93ECE1F9E21192119289E29D
:10B9E000EC34F807D1F7C4E1D9E260E073E0CE01AE
:10B9F0000E947C53229689E2CC31D807B1F7DF91BF
:10BA0000CF91089510926F1310926E1310927113CC
:10BA10001092701380E380936D138BEE92E19093FC
:10BA2000BA128093B9120C94E95CEF92FF920F93D3
:10BA30001F93CF93DF9300D0CDB7DEB78C0169831E
:10BA40007A830E94025D6981E62E7A81F72E81E871
:10BA5000E816F10418F080E8E82EF12CA701B801EF
:10BA60008091B9129091BA120E945293F092711380
:10BA7000E0927013C7010F900F90DF91CF911F914B
:10BA80000F91FF90EF9008950F931F93CF93DF9343
:10BA90008C01EB010E94025D1093BA120093B9125F
:10BAA000D0937113C0937013DF91CF911F910F91B9
:10BAB000089520E3ECE1F9E2DC0101900D922A9572
:10BAC000E1F788E0E4E1F9E2DB0101900D928A956B
:10BAD000E1F7089520E3FC01ACE1B9E201900D9299
:10BAE0002A95E1F788E0FB01A4E1B9E201900D920B
:10BAF0008A95E1F70895E82FF0E0EE0FFF1FE45E6E
:10BB0000F64D7183608381E090E00895E82FF0E0C6
:10BB1000EE0FFF1FE45EF64D80819181089590E065
:10BB2000880F991F8C51974D0E947C5381E090E0C3
:10BB3000089590E0880F991F8C51974D08958115B5
:10BB4000910511F00197F1F70895E0914F29F091D7
:10BB50005029908180914E2989230895E0914C29A4
:10BB6000F0914D29808190914E29892B8083E0911D
:10BB70005129F0915229808190914E29892B8083FF
:10BB80000895E0914C29F0914D29908180914E29A2
:10BB9000809589238083E0915129F09152299081E9
:10BBA00080914E2980958923808308951F93CF9398
:10BBB000DF93E0914C29F0914D29908180914E299D
:10BBC000809589238083E0915129F09152298081C9
:10BBD00090914E29892B80838FEB93E00E949F5D8B
:10BBE0001FB7F894E0915129F091522990818091EA
:10BBF0004E2980958923808383E890E00E949F5D91
:10BC0000E0914F29F0915029D081C0914E291FBF5A
:10BC100078948BE393E00E949F5DE0914F29F0912F
:10BC20005029908180914E29982319F08D2F8C23D3
:10BC300001C081E0DF91CF911F9108955093522967
:10BC40004093512970934D2960934C29909350292A
:10BC500080934F2981E001C0880F2A95EAF78093ED
:10BC60004E290C94D65DCF93DF93C82FDFB7F8949D
:10BC7000E0915129F0915229808190914E29892B90
:10BC8000808383E090E00E949F5DCC2351F0E0919F
:10BC90005129F0915229808190914E2990959823B5
:10BCA000908387E190E00E949F5DE0914F29F091A1
:10BCB0005029808190914E29892309F4C0E089E5BB
:10BCC00090E00E949F5DE0915129F091522980817E
:10BCD00090914E29909598239083DFBF8BE390E05D
:10BCE0000E949F5D8C2FDF91CF910895CF93DF93BA
:10BCF000C82FD8E08C2F81700E94335EC6958111C9
:10BD0000C068D150B9F78C2FDF91CF9108958FEF94
:10BD10000C94765EDF92EF92FF920F931F93CF9376
:10BD2000DF93E82EEB010E94D65D81112FC080EFDA
:10BD30000E94765EF12C10E488EFD82ED10E81E0BF
:10BD40000E94335E082F81E00E94335E882319F041
:10BD5000002361F01DC0011109C01E1528F0888163
:10BD600080FF04C0E11611F0F12E01E0802F0E9447
:10BD7000335E9881969501119068988311501D113A
:10BD8000DECF21961111D8CF8F2D03C08FEF01C0C8
:10BD90008EEFDF91CF911F910F91FF90EF90DF9089
:10BDA0000895FF920F931F93CF93DF93F82EEB012B
:10BDB0000E94D65D209769F085E50E94765E8E012F
:10BDC000085F1F4F89910E94765EC017D107D1F797
:10BDD00003C08CEC0E94765E8F2DDF91CF911F9176
:10BDE0000F91FF900C94765E0F931F93CF93DF9388
:10BDF000DB01EC9111969C911197F0E0F92B8031C9
:10BE000081F4BF016E7FE3E0660F771FEA95E1F7EB
:10BE100016969C911697ECE0F0E0E91BF109E60F0D
:10BE2000F71FF7FF07C091E0EA019883F195E195CC
:10BE3000F10902C0EA011882883279F414968C91D3
:10BE4000982F9076903649F086FF02C0EE7F05C0AD
:10BE500085FF02C0EC7F01C0E87FCF0144E09695EA
:10BE600087954A95E1F7D9018C93EF70E801E88353
:10BE700080E0DF91CF911F910F9108950F931F9351
:10BE8000CF93DF93EC018B01B80188810E948A5E19
:10BE9000888381508D3F30F4F8018081883211F021
:10BEA000803191F7DF91CF911F910F910895CF933A
:10BEB000DF93EC010E94D65DBE0184EB0E94D15E4F
:10BEC00081E00E94335EC82F0E94D65D81E0C111DF
:10BED00001C080E0DF91CF9108951F93CF93DF934E
:10BEE00000D0CDB7DEB7182F69837A830E94D65D64
:10BEF0000E94A55D69817A81882341F084E40E94D3
:10BF0000D15E113029F00E94AE5D02C082E001C016
:10BF100080E00F900F90DF91CF911F9108954F9285
:10BF20005F926F927F928F929F92AF92BF92CF92C9
:10BF3000DF92EF92FF920F931F93CF93DF93CDB7D2
:10BF4000DEB729970FB6F894DEBF0FBECDBF6C01E8
:10BF50005B014A0189010E94D65DB6018EEB0E9409
:10BF6000D15ECE0101967C013E019AE0690E711C02
:10BF700027010E94875EF70181937F01E615F7058F
:10BF8000C1F769E070E0C2010E942A79811109C0FD
:10BF90009401A501B201F60180810E94F45E80E067
:10BFA00001C083E029960FB6F894DEBF0FBECDBF67
:10BFB000DF91CF911F910F91FF90EF90DF90CF9085
:10BFC000BF90AF909F908F907F906F905F904F90B9
:10BFD00008955F926F927F928F929F92AF92BF92DD
:10BFE000CF92DF92EF92FF920F931F93CF93DF9345
:10BFF000CDB7DEB729970FB6F894DEBF0FBECDBF21
:10C00000582E6B015A01890160E070E08EEB0E94AE
:10C01000D15ECE0101967C014E019AE0890E911C01
:10C0200037010E94875EF70181937F01E815F905CA
:10C03000C1F769E070E0C3010E942A79811108C04C
:10C040009501A601B301852D0E94F45E80E001C038
:10C0500083E029960FB6F894DEBF0FBECDBFDF9107
:10C06000CF911F910F91FF90EF90DF90CF90BF90F5
:10C07000AF909F908F907F906F905F9008950F93F7
:10C080001F93CF93DF93CDB7DEB728970FB6F89401
:10C09000DEBF0FBECDBF182F062F98E0ECE0F3E017
:10C0A000DE01119601900D929A95E1F7242F332726
:10C0B00027FD309541E752E0249FC001259F900D58
:10C0C000349F900D112464E670E00E943C8DCB01FA
:10C0D00044E6049F800D911D1124FE013196AE01AE
:10C0E000475F5F4F619170E02617370711F40196A3
:10C0F00003C0E417F507B1F7112319F09195819565
:10C10000910928960FB6F894DEBF0FBECDBFDF9120
:10C11000CF911F910F910895EF92FF920F931F936C
:10C12000CF93DF93CDB7DEB72B970FB6F894DEBF72
:10C130000FBECDBFF82EE92E682F792F88E08F0D26
:10C140000E946D5F882319F084E391E243C066E4A6
:10C1500071E48FE090E00E94F7608E01075F1F4F4F
:10C160009801AE01465F5F4FBE01655F7F4F8F2D27
:10C170009E2D0E948F5F8111E7CF88E0ECE0F3E015
:10C18000DE01119601900D928A95E1F7498521E72C
:10C1900032E0429FC001439F900D112464E670E09D
:10C1A0000E943C8D8A8594E6899F600D711D112443
:10C1B000FE0131968191481303C06F5F7F4F03C02A
:10C1C000E017F107B9F78B85882319F07195619510
:10C1D0007109CB012B960FB6F894DEBF0FBECDBF11
:10C1E000DF91CF911F910F91FF90EF900895DC01A7
:10C1F000CB0181159105A105B10529F08150904031
:10C20000A040B040D9F708959B01AC011092B9004D
:10C2100060E072E18AE790E00E94508D2051310980
:10C220004109510956954795379527952093B800B0
:10C23000089594EA9093BC0040EA56E861E070E00B
:10C240009091BC0097FD0BC04150510961097109E3
:10C25000411551056105710599F781E008959091A7
:10C26000B900987F983011F09031B9F78093BB00F6
:10C2700084E88093BC0080EA96E8A1E0B0E02091D9
:10C28000BC0027FD08C00197A109B1090097A105CD
:10C29000B105A9F7E2CF8091B900887F883111F00C
:10C2A0008034D9F680E0089524EA34E844E9209304
:10C2B000BC009091BC0097FFFCCF9091B900987F93
:10C2C000983011F0903199F78093BB003093BC0007
:10C2D0009091BC0097FFFCCF9091B900987F90326D
:10C2E00011F0983539F44093BC009091BC0094FD56
:10C2F000FCCFDDCF08950C94196184E98093BC00D4
:10C300008091BC0084FDFCCF08958093BB0084E83D
:10C310008093BC008091BC0087FFFCCF9091B90056
:10C32000987F81E0983209F480E0089584EC80934E
:10C33000BC008091BC0087FFFCCF8091BB000895BA
:10C3400084E88093BC008091BC0087FFFCCF809183
:10C35000BB000895E0E1DC01FD91CD01F0933F01C8
:10C36000E150C9F780913C018F7D80933C01809121
:10C370003C01877F80933C01FB0180E19191909388
:10C380003E018150D9F780913C01806880933C0147
:10C3900080913D0180FFFCCF4051510980913C01CB
:10C3A000806280933C0180913C01877F80933C01B7
:10C3B000141615069CF4FB0180E1919190933E01C7
:10C3C0008150D9F780913C01806880933C01809135
:10C3D0003D0180FFFCCF40515109EACFF90180E1D6
:10C3E00090913E0191938150D9F781E090E00895BA
:10C3F0000F931F93CF93DF93EC018CE70E9454615E
:10C400008CE70E9485618E01005F1F4F89910E9419
:10C410008561C017D107D1F7DF91CF911F910F919F
:10C420000C947D61813019F440E050E002C040EC92
:10C4300050E060E070E08CE790E00C94B711813040
:10C4400019F44EE050E002C048E050E060E070E0D7
:10C450008CE790E00C94B71141E050E060E070E0B0
:10C460008CE790E00E94B7116AE67AE080E090E005
:10C470000C94F76048E350E060E070E08CE790E0F7
:10C480000E94B71149E350E060E070E08CE790E073
:10C490000E94B71144E150E060E070E08CE790E06A
:10C4A0000E94B71148E750E060E070E08CE790E050
:10C4B0000E94B7114EE550E060E070E08CE790E03C
:10C4C0000E94B7114DE650E060E070E08CE790E02C
:10C4D0000E94B7116CE17AE186E090E00E94F7607B
:10C4E0004CE050E060E070E08CE790E00E94B71113
:10C4F00041E050E060E070E08CE790E00E94B7110E
:10C5000046E050E060E070E08CE790E00E94B711F8
:10C510006AE67AE080E090E00C94F760CF93DF93D6
:10C52000CDB7DEB7A2970FB6F894DEBF0FBECDBF72
:10C5300081E1E0E4F9E0DE01529601900D928A95E6
:10C54000E1F781E1E1E5F9E0DE01119601900D925C
:10C550008A95E1F70E943A62CE0142960E94F86104
:10C5600082E00E9412626AE67AE080E090E00E9437
:10C57000F760CE0101960E94F86160E17EEA88E2F0
:10C5800090E00E94F76080E00E941F6260E17EEA16
:10C5900088E290E00E94F7604EE050E060E070E0DA
:10C5A0008CE790E00E94B711A2960FB6F894DEBF18
:10C5B0000FBECDBFDF91CF910895CF92DF92EF9262
:10C5C000FF920F931F93CF93DF9300D01F92CDB7AD
:10C5D000DEB7F82E042F122F213031F0223031F047
:10C5E000243031F0283031F090E005C091E003C0F4
:10C5F00092E001C093E00C3059F00E3011F49460D9
:10C6000007C0003111F4986003C0023109F49C6046
:10C61000613059F0623011F4906207C0633011F458
:10C62000906403C0643009F490669068692F70E0EC
:10C6300023E030E0AE014F5F5F4F8F2D90E00E940E
:10C64000CE1169E07AE180E090E00E94F7608F2DE2
:10C650008160F82E0E9419610E94966189830E9470
:10C6600096618A83023119F40E9496618B830E943D
:10C67000966187FDF1CF0E94A0610E947D6169E013
:10C680007AE180E090E00E94F7608F2D0E941961AE
:10C690000E94966189830E9496618A83023119F40F
:10C6A0000E94A0618B830E94A0610E947D613981FC
:10C6B0002A81023149F5832F90E0A0E0B0E04B8160
:10C6C0007727662731FF0EC030E0322F2227620F16
:10C6D000731F811D911D640F711D811D911D8C6F34
:10C6E0009F6F0BC030E0322F2227620F731F811D16
:10C6F000911D640F711D811D911D0E94768A20E895
:10C700003FEF4FEF57E420C0632F70E0762F66278E
:10C71000620F711D882777FD8095982F0E94768A79
:10C720000C3029F420E030EE4FEF54E40DC00E3011
:10C7300029F420E038EF4FEF55E406C0003131F422
:10C7400020E03EEF4FEF56E40E94D7892FE632E11A
:10C7500043E050E40E94588C6B017C01612F70E033
:10C7600080E090E00E94768A9B01AC01C701B6018F
:10C770000E94D7890F900F900F90DF91CF911F915A
:10C780000F91FF90EF90DF90CF900895E6E4F1E0F5
:10C7900080812081908130818295869586958370F5
:10C7A00022952F70822B832B92959F70892B089551
:10C7B0000F931F93CF93DF9300D0CDB7DEB746E042
:10C7C0006CE080E00E94086789E18093C4001092C9
:10C7D000C50082E08093C00080E00E9495670E94BF
:10C7E000346684B784B784B784B784B7E3EDF1E3E4
:10C7F00022E432E4318320833A968DB79EB70A97BC
:10C80000E817F907B8F382E699E09F938F9381E3E5
:10C8100091E19F938F930E9419940E946D750E94DD
:10C82000285560E070E086E892E00E94D0550E94B2
:10C830000459E0911403F091150309950E94C66311
:10C8400090E00E94A975CE0101960E9469650F9043
:10C850000F900F900F90882341F081E191E19F9319
:10C860008F930E9419940F900F90CE0101960E9411
:10C8700097530E9477658C010E947365AE014F5FEC
:10C880005F4FB8010E945F6A0E94E3640E94406AA1
:10C890000E947B650E94996B84E091E19F938F9346
:10C8A0000E9419948A811F928F9300E011E11F93D7
:10C8B0000F930E94199489811F928F931F930F9356
:10C8C0000E9419948EEF90E19F938F930E94199488
:10C8D0000E94AD75E0915103F09152030995E091EA
:10C8E0004303F09144030995E0912A03F0912B034F
:10C8F00009950E94A06B182F0E943D6A1F921F93FA
:10C900001F928F93809150038F9380914F038F9349
:10C91000809142038F93809141038F9383EE90E146
:10C920009F938F930E941994E0915B03F0915C03B5
:10C930000FB6F894DEBF0FBECDBF309791F00995CA
:10C94000BC0180E890E00E94288D7F936F9380ED7A
:10C9500090E19F938F930E9419940F900F900F90E6
:10C960000F908EEC90E19F938F930E94199460E05A
:10C9700070E08CED92E00E94D05580EF92E00E9432
:10C980007D7486EC90E19F938F930E9419940F9091
:10C990000F900F900F900F900F90DF91CF911F91FC
:10C9A0000F9108957F936F939F938F9380EC90E105
:10C9B0009F938F930E9419940F900F900F900F9058
:10C9C0000F900F9008951F93CF93DF93CDB7DEB7ED
:10C9D000A0970FB6F894DEBF0FBECDBF8DE590E0F7
:10C9E0000E948595182F282F35EF380F303108F029
:10C9F000982F9095291709F461C08CE491E19F93D9
:10CA00008F930E941994E1E9F1E10F900F90DE01FC
:10CA1000119684918D93319681E1E939F807C9F730
:10CA2000F89448E050E069E770E0CE0101960E947A
:10CA30008B95E3E8F1E1DE01119684918D933196B7
:10CA400081E1E139F807C9F74EE050E06BE670E0AC
:10CA5000CE0101960E948B95E9E7F1E1DE01119686
:10CA600084918D93319681E1E338F807C9F74AE064
:10CA700050E061E670E0CE0101960E948B956DEC6E
:10CA80007BEA8BE590E00E94A39560E070E089E589
:10CA900090E00E94A39560E088E590E00E94959563
:10CAA00060E070E08FE590E00E94A3951AE16AE1F2
:10CAB00075EE8DE590E00E94A3957894812FA09665
:10CAC0000FB6F894DEBF0FBECDBFDF91CF911F919F
:10CAD0000895F89442E050E069E770E00E946D9597
:10CAE000789480E008958BE590E00C94859589E535
:10CAF00090E00C94859588E590E00C947D954091AC
:10CB0000612950916229609163297091642990E0B4
:10CB1000A0E0B0E0480F591F6A1F7B1F40936129B6
:10CB200050936229609363297093642940915D2931
:10CB300050915E2960915F2970916029480F591FBB
:10CB40006A1F7B1F40935D2950935E2960935F2984
:10CB5000709360292091012B2223A1F04091592943
:10CB600050915A2960915B2970915C29480F591F97
:10CB70006A1F7B1F4093592950935A2960935B2960
:10CB800070935C2908951F920F920FB60F92112493
:10CB90000BB60F922F933F934F935F936F937F93B7
:10CBA0008F939F93AF93BF93EF93FF9380917413F1
:10CBB00090917513019690937513809374138091DF
:10CBC00073138F5F809373138038A9F410927313DB
:10CBD0008091612990916229A0916329B091642983
:10CBE0000196A11DB11D8093612990936229A093A4
:10CBF0006329B09364298091012B8823E1F080910F
:10CC000072138F5F809372138038A9F4109272139D
:10CC10008091592990915A29A0915B29B0915C2962
:10CC20000196A11DB11D8093592990935A29A09373
:10CC30005B29B0935C290E946058892B11F00E94F7
:10CC40007357FF91EF91BF91AF919F918F917F911A
:10CC50006F915F914F913F912F910F900BBE0F906D
:10CC60000FBE0F901F901895F8941092B60016BC46
:10CC700083EF87BD82E084BD94E095BD95B395BBFD
:10CC800080936E0078940895809174139091751339
:10CC9000209174133091751382179307A9F70895A3
:10CCA000009751F022E330E00000215031092115B6
:10CCB0003105D1F70197F4CF08950F931F93CF93C8
:10CCC000DF93EC010E9444668C010E944466801B45
:10CCD000910B8C179D07C8F3DF91CF911F910F9196
:10CCE000089508950F931F936091612970916229AF
:10CCF00080916329909164290091612910916229A2
:10CD00002091632930916429601771078207930786
:10CD100059F71F910F9108951F920F920FB60F921E
:10CD200011241092B2020F900FBE0F901F90189511
:10CD30001F920F920FB60F9211240BB60F922F93E2
:10CD40003F934F935F936F937F938F939F93AF9393
:10CD5000BF93EF93FF93E091A802F091A902808125
:10CD6000E091B302F091B402309709F00995FF9178
:10CD7000EF91BF91AF919F918F917F916F915F9153
:10CD80004F913F912F910F900BBE0F900FBE0F90C0
:10CD90001F9018951F920F920FB60F9211241092A8
:10CDA000BF020F900FBE0F901F9018951F920F9209
:10CDB0000FB60F9211240BB60F922F933F934F9300
:10CDC0005F936F937F938F939F93AF93BF93EF93F3
:10CDD000FF93E091B502F091B6028081E091C0022C
:10CDE000F091C102309709F00995FF91EF91BF9141
:10CDF000AF919F918F917F916F915F914F913F91F3
:10CE00002F910F900BBE0F900FBE0F901F90189593
:10CE10009DE0899FF0011124E855FD4FA281B38167
:10CE20001C92A481B5816C93A681B78188ED8C9307
:10CE3000A085B1854C9312861486138608959DE0D3
:10CE4000899FF0011124E855FD4F81E08287A08180
:10CE5000B1816C933A9680818111FDCF08951F9323
:10CE6000CF93DF93182FEB01FE018491882339F0D3
:10CE7000FE016491812F0E941F672196F5CFDF91FB
:10CE8000CF911F9108951F93CF93DF93182FEB013C
:10CE90008881882369F08A3021F46DE0812F0E9417
:10CEA0001F6769916D30A1F3812F0E941F67F0CF3A
:10CEB000DF91CF911F910895CF93DF93CDB7DEB768
:10CEC0009E01285F3F4F4E815F8160E470E086E7FE
:10CED00093E10E94D69466E773E18D810E944367D7
:10CEE000DF91CF910895CF93C82F8A3031F46DE050
:10CEF0008091B6130E941F6702C08D3029F06C2FFD
:10CF00008091B6130E941F6780E090E0CF91089552
:10CF10009DE0899FF0011124E855FD4F74876387D8
:10CF20000895682F80E00C941F678093B6138AE9F8
:10CF300092E09093CE318093CD31089584B7877F6E
:10CF400084BF88E10FB6F89480936000109260006F
:10CF50000FBE08952FE088E190E00FB6F894A895F1
:10CF6000809360000FBE209360000895A8950895F7
:10CF700088E10FB6F89480936000109260000FBEB5
:10CF80000895F89428E088E190E00FB6F894A89509
:10CF9000809360000FBE20936000FFCF80916C29CA
:10CFA00080916C2990E0089540E06FE181E491E088
:10CFB0000C94356DE9E3F1E0808180818D7F808381
:10CFC0008DE090E00197F1F723E040E06FE182E42B
:10CFD00091E00E943F6D83E090E00197F1F70895A2
:10CFE0009091390191FD0AC0282F803108F02FE07F
:10CFF00040E06FE085E491E00C943F6D08958091EE
:10D00000390181FD0EC040E06FE181E491E00E94B2
:10D01000356D282F2F7E81E090E0213021F080E0D7
:10D02000089580E090E008958091390181FD10C05D
:10D0300040E06FE181E491E00E94356D8F3131F085
:10D04000982F9F7E915081E0923018F480E00895EF
:10D0500081E008950E9414688823E1F30895CF9336
:10D06000DF93C82F0E942A680E94D467D82FC81760
:10D0700089F1C83019F40E94DA6725C0C93121F45A
:10D08000863189F429E005C0C63169F4893159F443
:10D0900026E040E06FE182E491E00E943F6DE3E032
:10D0A000F0E03197F1F72C2F40E06FE182E491E05E
:10D0B0000E943F6DD83019F4E9E6F1E002C0E3E0E8
:10D0C000F0E03197F1F70E94D4678C1719F083E4F0
:10D0D00090E002C080E490E0DF91CF9108950E943B
:10D0E0002A681092012B0E94DA67809139018260D0
:10D0F000809339018091842B8823D9F18091940009
:10D10000909195004091952B5091962B84179507FF
:10D11000A0F48091612B9091622BA091632BB09130
:10D12000642B8C57914EAF4FBF4F8093612B9093E0
:10D13000622BA093632BB093642B209194003091C9
:10D140009500241B350B8091612B9091622BA0914F
:10D15000632BB091642B820F931FA11DB11D80938F
:10D16000612B9093622BA093632BB093642B10924E
:10D17000842B8091862B8823D9F180919400909103
:10D1800095004091992B50919A2B84179507A0F404
:10D190008091692B90916A2BA0916B2BB0916C2B95
:10D1A0008C57914EAF4FBF4F8093692B90936A2B52
:10D1B000A0936B2BB0936C2B209194003091950031
:10D1C000241B350B8091692B90916A2BA0916B2BBE
:10D1D000B0916C2B820F931FA11DB11D8093692B01
:10D1E00090936A2BA0936B2BB0936C2B1092862B91
:10D1F00008958091012B882381F080913A14811148
:10D2000004C00E941468811106C081E08093381424
:10D2100081E090E008950E946F6880E090E00895BA
:10D22000809194009091950090939A2B8093992BE4
:10D2300021E02093862B8091390181FD08C08091E7
:10D24000390181FD1AC086E10E942F6816C0209323
:10D25000002B80919400909195009093962B809351
:10D26000952B2093842B809139018D7F80933901F8
:10D270008091002B8111FCCFE2CF81E08093012BC4
:10D2800008958091012B81110AC080913A1488235E
:10D2900021F081E08093391402C00E94106981E07E
:10D2A00090E008951F93CF93DF931F92CDB7DEB721
:10D2B0008FB7898380913A14811126C0F8948091A8
:10D2C000012B882351F08091390181FD1BC00E9400
:10D2D00014688823B9F080E003C00E94416981E0AE
:10D2E0002091470191E02E3008F090E0192F119520
:10D2F00081110E94F968107429F089818FBF81E043
:10D3000090E004C089818FBF80E090E00F90DF91B2
:10D31000CF911F91089580913914882321F00E94A4
:10D3200010691092391480913814882321F00E94DA
:10D330006F681092381410923A1408950F931F9347
:10D34000AB0121E020933A140091452B1091462B1C
:10D350002091472B3091482B0F5F1F4F2F4F3F4F8E
:10D360000093452B1093462B2093472B3093482B4B
:10D3700022E0260F27FF0CC08091FE2A9091FF2A01
:10D3800001969093FF2A8093FE2A0FEF1FEF07C0AC
:10D39000BC0187EB93E10E94529300E010E00E94F1
:10D3A0008B69C8011F910F91089580933C140895D3
:10D3B0000E94D467823011F0823111F480E0089528
:10D3C00081E0089508958FEF80934E0122E044E0BC
:10D3D00060EF8CE691E00E943F6D25E041E06EE059
:10D3E0008CE290E00E943F6D80E880936F01809115
:10D3F000460180936D0121E045E060E284E491E024
:10D400000C943F6D8DEF93E00197F1F70E942B6D27
:10D41000109275291092F7291092792A1092742986
:10D4200010927329E9E3F1E080818E7F808380810F
:10D430008D7F80838DE090E00197F1F7808181609E
:10D44000808323E040E06FE182E491E00E943F6D41
:10D450008DEF93E00197F1F780915D0180915E017E
:10D460000E94E36960E070E082EC92E00E94D05597
:10D470000E94106981E090E0089580913B14089526
:10D48000CF93DF931F92CDB7DEB789830E942A68BE
:10D49000898180933B14282F40E06FE188E491E07C
:10D4A0000F90DF91CF910C943F6D0E94406A809164
:10D4B000390181FD03C086E00C942F680895FA01BC
:10D4C00080936201909363016093600170936101A6
:10D4D0003097C1F0808180936B01818180936A01D4
:10D4E0008281809369018381809368018481809324
:10D4F00067018581809366018681809365018781BC
:10D5000080936401089582EC92E00E94F15581E0DD
:10D5100080936C2980916D2990916E29019690934A
:10D520006E2980936D2981E090E00895809174299F
:10D5300092E8899FF0011124EB58F64D10828F5F1D
:10D54000833018F48093742902C010927429E091FA
:10D55000742982E8E89FF0011124EB58F64D808190
:10D5600081110C94836A10926C2908951F93CF93B4
:10D57000DF932091742912E8129F90011124D901A0
:10D58000AB58B64D4C91411103C00E94966A93C0AE
:10D590005091390151FD8FC05091012B552309F451
:10D5A0008AC047FF16C00E94966A8091352B9091E1
:10D5B000362BA091372BB091382B0196A11DB11DB0
:10D5C0008093352B9093362BA093372BB093382B29
:10D5D00072C04330B0F40E94966A8091312B9091D2
:10D5E000322BA091332BB091342B0196A11DB11D8C
:10D5F0008093312B9093322BA093332BB093342B09
:10D600005AC050E0EA0122976C177D07B0F40E94DF
:10D61000966A80912D2B90912E2BA0912F2BB0915B
:10D62000302B0196A11DB11D80932D2B90932E2B95
:10D63000A0932F2BB093302B3EC0B9016A58764D82
:10D640000E945293E09174291E9FF0011124EB5027
:10D65000F64D8081809365290E94966A80914701EA
:10D660008093662990916B29992311F0891710F402
:10D6700080936B296091662970E084E00E947B5D55
:10D680006091652970E083E00E947B5D4091492BA9
:10D6900050914A2B60914B2B70914C2B4F5F5F4FF9
:10D6A0006F4F7F4F4093492B50934A2B60934B2BE6
:10D6B00070934C2B02C0C0E0D0E0CE01DF91CF913F
:10D6C0001F910895CF93DF93EC0188819981009792
:10D6D000E9F08730954021F01982188283E026C056
:10D6E0006238C1F410926C290E94025D0E94695C4C
:10D6F00060E870E00E94B66A181619066CF40E9481
:10D70000645CE0915503F0915603099587E095E03C
:10D710009983888381E00AC08091692990916A2960
:10D72000019690936A2980936929F0CFDF91CF9178
:10D73000089591E090933A140E94F0670C948B69DD
:10D740008091390181FD06C040E06FE085E491E001
:10D750000C94356D80E108950F931F93CF93DF9361
:10D76000182F21E020933A140091012B8091390168
:10D7700081FF16C080919400909195009093962B14
:10D780008093952B2093842B2093002B809139013B
:10D790008D7F809339018091002B8111FCCF00E0B7
:10D7A0000E942A688091012B882309F43FC0809150
:10D7B000862B8823D9F18091940090919500E09177
:10D7C000992BF0919A2B8E179F07A0F44091692B0B
:10D7D00050916A2B60916B2B70916C2B4C57514E72
:10D7E0006F4F7F4F4093692B50936A2B60936B2B45
:10D7F00070936C2B20919400309195002E1B3F0B61
:10D800004091692B50916A2B60916B2B70916C2B1E
:10D81000420F531F611D711D4093692B50936A2B5A
:10D8200060936B2B70936C2B1092862B8091390137
:10D8300081FD03C089E10E942F6886E00E94865D19
:10D84000892B51F00E94A06BC82F86E00E94865D54
:10D8500081500E94F06702C0C0E0D0E020919400A7
:10D86000309195003093982B2093972B81E08093F3
:10D87000852BF894809139018260809339018091E1
:10D8800039018D7F8093390162E0610F87EB93E16D
:10D890000E946E6D78942091FB2A3091FC2A2F5FB4
:10D8A0003F4F3093FC2A2093FB2A0E942A6845E0D0
:10D8B00060EE82E491E00E94356D182F86E00E94B0
:10D8C000865D892B19F08C2F0E94F067002319F0D8
:10D8D0000E94106902C00E946F688091852B882386
:10D8E000D9F18091940090919500E091972BF0915F
:10D8F000982B8E179F07A0F44091652B5091662BB3
:10D900006091672B7091682B4C57514E6F4F7F4F32
:10D910004093652B5093662B6093672B7093682B15
:10D9200020919400309195002E1B3F0B4091652B68
:10D930005091662B6091672B7091682B420F531F9B
:10D94000611D711D4093652B5093662B6093672B6F
:10D950007093682B1092852B8091012B882361F0A6
:10D96000209194003091950030939A2B2093992B1D
:10D9700081E08093862B07C023E040E06FE182E4E2
:10D9800091E00E943F6D0E948B691130E9F01330E5
:10D99000A9F480913D2B90913E2BA0913F2BB0910B
:10D9A000402B0196A11DB11D80933D2B90933E2BE2
:10D9B000A0933F2BB093402B12E009C0153031F0FB
:10D9C000173029F411E003C010E001C013E0812FEB
:10D9D00090E0DF91CF911F910F910895CF93DF9346
:10D9E000EB010E949E69009729F4CE010E94AC6B66
:10D9F000009751F02091FE2A3091FF2A2F5F3F4F70
:10DA00003093FF2A2093FE2ADF91CF910895CF9380
:10DA1000DF938091012B811104C00E944169D1E004
:10DA200001C0D0E00E94D467863111F0813119F431
:10DA3000C091470109C040E06FE186E491E00E9497
:10DA4000356DC82FCC0FC80FD1110E94F9688C2FEB
:10DA5000DF91CF91089510923E1410923D14EFE69D
:10DA6000F0E08081806280830895FC0180818623BC
:10DA700090E002C0959587954A95E2F70895F8944D
:10DA8000FC015081362F30955323042E01C0220F04
:10DA90000A94EAF72623522B5083789408954091F4
:10DAA0007B01FC014193A0E8B1E050E8540F9D01D7
:10DAB0002F5F3F4F6C916193521711F0D901F7CF4F
:10DAC0004150E42FF0E0E058FE4F2181FC01E05886
:10DAD000FF4F2083319621E02083089560938001D9
:10DAE000E1E8F1E061589F012F5F3F4FDC014D916C
:10DAF000CD014083621711F0F901F5CF08951F920F
:10DB00000F920FB60F9211240BB60F922F933F93E3
:10DB10004F935F936F937F938F939F93AF93BF9335
:10DB2000EF93FF9380914701809366298091732939
:10DB300022E8829FC00111248B58964D0E944F6DA0
:10DB4000809173298F5F833018F48093732902C00A
:10DB5000109273290E94836AFF91EF91BF91AF9158
:10DB60009F918F917F916F915F914F913F912F91F5
:10DB70000F900BBE0F900FBE0F901F9018951F9225
:10DB80000F920FB60F9211240F900FBE0F901F909F
:10DB900018951F920F920FB60F9211240F900FBE7F
:10DBA0000F901F9018951F920F920FB60F9211248D
:10DBB0000F900FBE0F901F9018951F920F920FB6E7
:10DBC0000F9211241092002B0F900FBE0F901F90F8
:10DBD00018951F920F920FB60F9211241092002BDE
:10DBE0000F900FBE0F901F9018951F920F920FB6B7
:10DBF0000F9211248F9381E080936C298F910F9065
:10DC00000FBE0F901F9018951F920F920FB60F9294
:10DC100011241092002B0F900FBE0F901F9018959B
:10DC20001F920F920FB60F9211248F939F938091A2
:10DC30003D1490913E14019690933E1480933D14B0
:10DC40009F918F910F900FBE0F901F901895CF92BC
:10DC5000DF92EF92FF920F931F93CF93DF937C019C
:10DC60008B016A018FE394E10E949056EC010097CA
:10DC700051F0EC81FD81309711F0C8010995CE017A
:10DC80000E943857F3CFA601B801C701DF91CF91A9
:10DC90001F910F91FF90EF90DF90CF900C941A544A
:10DCA0000F931F93CF93DF9300D0CDB7DEB7809152
:10DCB000092B90910A2BA0910B2BB0910C2B019664
:10DCC000A11DB11D8093092B90930A2BA0930B2BC0
:10DCD000B0930C2B0E94BA708C018FE394E10E94E8
:10DCE0009056009779F0DC011296ED91FC91139714
:10DCF000309729F089839A8309959A8189810E94B6
:10DD00003857EFCF0115110549F0C8010F900F905A
:10DD1000DF91CF911F910F910C9411540F900F90A0
:10DD2000DF91CF911F910F9108950E94AD750E94D0
:10DD3000025D0E94E16E81E493E09093042B809356
:10DD4000032B0E94B8702FEF31E040E05EE160E00D
:10DD500074E082E090E00C948170BC018FE394E168
:10DD60000C94F056BC018FE394E10C94D556CF93FC
:10DD7000DF93EC014091052B5091062B6091072B0E
:10DD80007091082B4F5F5F4F6F4F7F4F4093052B74
:10DD90005093062B6093072B7093082B0E94CD7035
:10DDA000009761F00E94825CE0914503F091460388
:10DDB000BE0187E29EE6099581E090E0DF91CF9178
:10DDC000089585E494E10C948C560F93CF93DF93E0
:10DDD000EC017B836A8318865F834E83BC0185E4F4
:10DDE00094E10E94F056E0914114F0914214309772
:10DDF00049F04C815D8101E020E030E068858A8156
:10DE00009B810995DF91CF910F910895BC0185E425
:10DE100094E10C94D5560F93DC0118961C92189738
:10DE2000E0914114F0914214309759F000E020E065
:10DE300030E040E050E060E012968D919C911397A5
:10DE400009950F9108950F93DC01AB0114962D9164
:10DE50003C91159781E018968C93189715967C93B2
:10DE60006E931497E0914114F0914214309739F079
:10DE700000E061E012968D919C91139709950F91A6
:10DE800008950F93DC01E0914114F0914214309712
:10DE900071F014964D915C91159701E09A011896D6
:10DEA0006C91189712968D919C91139709950F91EB
:10DEB0000895E0914314F0914414309709F00994C7
:10DEC00008959093441480934314089590934214BA
:10DED00080934114089585E494E10C949056EF9258
:10DEE000FF920F931F93CF93DF938C01EB017A0185
:10DEF00085E494E10E9490560097D9F0DC011296D7
:10DF00002D913C9113972C173D0781F41696ED91B6
:10DF1000FC911797309769F09701AE01B801DF9136
:10DF2000CF911F910F91FF90EF9009940E94385765
:10DF3000E3CFDF91CF911F910F91FF90EF90089564
:10DF40000895CF93DF93C8E7D4E16881798120E019
:10DF500030E040EC5FE682E694E10E9410590E94B6
:10DF6000AB75688179810E94288D20E030E044ED16
:10DF70005FE6BC0182E594E1DF91CF910C941059EA
:10DF800080917814909179142091761430917714BF
:10DF9000880F991F2817390708F4C901909379143D
:10DFA000809378140C94A16FCF93DF930E94025D4D
:10DFB0000E94695CEC01198218820E946B6F2881B3
:10DFC0003981009719F1FC0140854423F9F0FC01E7
:10DFD00042815381F901EE0FFF1FEE0FFF1FEC0F7F
:10DFE000FD1F53834283FC01448155812F5F3F4FC6
:10DFF000F901EE0FFF1FEE0FFF1FEC0FFD1F518306
:10E000004083398328830E943857D9CFC901880FAC
:10E01000991F880F991F02960E94645C88819981DC
:10E02000892B31F087E494E1DF91CF910C94E85390
:10E03000DF91CF910895AF92BF92CF92DF92EF928E
:10E04000FF920F931F93CF93DF9300D0CDB7DEB72E
:10E050006B010E94695CFC01008111811A830983B4
:10E060000C30110518F4E12CF12C0DC01F930F9307
:10E0700080E899E09F938F930E9407940F900F90F0
:10E080000F900F9021C0E016F106F1F00E94695C3C
:10E09000F701EE0FFF1FEE0FFF1FE80FF91FA28021
:10E0A000B3800E94695CFFEFEF1AFF0AF701EE0FE1
:10E0B000FF1FEE0FFF1FE80FF91F40815181B501CF
:10E0C000C6010E946F6FDFCF0F900F90DF91CF914D
:10E0D0001F910F91FF90EF90DF90CF90BF90AF9086
:10E0E00008950F93013059F4809172149091731434
:10E0F00090937914809378140F910C94A16F0F91E1
:10E100000895EF92FF920F931F93CF93DF938B01AC
:10E11000EA0179014EE253E0BC0187E494E10E94F8
:10E12000CC531093731400937214D0937514C0934E
:10E130007414F0927714E092761481E790E7DF91FF
:10E14000CF911F910F91FF90EF900C94666F82E634
:10E1500094E10E94945982E594E10E94945987E4E5
:10E1600094E10C94E6538091781490917914089579
:10E170000C942654CF93DF93E0913203F091330354
:10E180000995EC01009729F06A817B8181E00E946A
:10E190007B5DCE01DF91CF9108950F931F93CF93B5
:10E1A000DF93EC01E0913403F091350309958C0184
:10E1B0006A817B8181E00E947B5D81E090E0012BA0
:10E1C00011F480E090E0DF91CF911F910F910895BD
:10E1D000E0913603F0913703099420E030E0029695
:10E1E000FC0132974081442331F0FC01319740819A
:10E1F000240F311DF4CFC9010895FC01208130E0C6
:10E20000322F22278181282B02C0220F331F6A95CB
:10E21000E2F7832F9927FA01E85CFC4F208130E078
:10E220008223932328E030E0241B350B02C096950F
:10E2300087952A95E2F708956F927F928F929F9229
:10E24000AF92BF92CF92DF92EF92FF920F931F9304
:10E25000CF93DF938C01EB016A01790128303105FE
:10E2600024F4A901B601CE014AC0590123E0B594B6
:10E27000A7942A95E1F74115510521F04801612C39
:10E28000712C03C0D801FB0120C048E050E0B6016A
:10E29000CE01860D971D0E94FD70F40181934F0100
:10E2A000FFEF6F1A7F0A6A147B047CF3C501B7FE87
:10E2B00002C080E090E0A701477055274115510545
:10E2C00011F1080F191FB60118C0CF018C1B9D0B4F
:10E2D0008A159B051CF481918D93F7CFC501B7FE7C
:10E2E00002C080E090E0A701477055274115510515
:10E2F00051F0080F191F60E070E08C0F9D1F0E9405
:10E30000FD70F8018083DF91CF911F910F91FF90F5
:10E31000EF90DF90CF90BF90AF909F908F907F90C5
:10E320006F9008958F929F92AF92BF92CF92DF929B
:10E33000EF92FF920F931F93CF93DF9300D0CDB74F
:10E34000DEB70E94695C8C0182E090E00E94475C2D
:10E35000892B19F480E090E05DC0F801818190E0A4
:10E36000982F88272081820F911D0E9437547C01AD
:10E37000009781F30E94695C4C01F7012681822F8E
:10E3800086958695869590E0422F477021E030E093
:10E3900011F420E030E0820F931F0E94475C892B2C
:10E3A000C9F2F70104811581C12CD12CF8018081BB
:10E3B000882379F1F801A180B12CB60133E075957D
:10E3C00067953A95E1F7A60147705527680D791DC5
:10E3D000883168F09501CE0101960E941C71BE0142
:10E3E0006F5F7F4FF80180810E948F5D0DC01A82A0
:10E3F00019829501CE0101960E941C7169817A8172
:10E40000F80180810E947B5DCA0CDB1C0E5F1F4FF0
:10E41000CDCFC7010F900F90DF91CF911F910F913A
:10E42000FF90EF90DF90CF90BF90AF909F908F9034
:10E430000895DC0150E0E0E1F0E0E61BF70BE21BA1
:10E44000F30B02C0440F551FEA95E2F78C91852B20
:10E450008C9311968C911197842B11968C9308951F
:10E460006F927F928F929F92AF92BF92CF92DF92E4
:10E47000EF92FF920F931F93CF93DF938C016B0169
:10E48000EA017901283031051CF44881C8015CC0DB
:10E49000390153E0759467945A95E1F76115710558
:10E4A00021F04E01A12CB12C03C0D801FE0127C0E0
:10E4B000F40141914F0128E030E0B601C8018A0D16
:10E4C0009B1D0E941972FFEFAF1ABF0AA614B70472
:10E4D0007CF3C30177FE02C080E090E097012770D3
:10E4E00033272115310509F43FC0C80FD91F4881D2
:10E4F00050E0B601621B730B685F7F4F1CC0CF01F9
:10E500008C1B9D0B861597051CF481918D93F7CF7D
:10E51000C30177FE02C080E090E0970127703327A7
:10E520002115310509F1C80FD91F488150E068E075
:10E5300070E0621B730B02C0559547956A95E2F730
:10E5400060E070E0800F911FDF91CF911F910F91DC
:10E55000FF90EF90DF90CF90BF90AF909F908F9003
:10E560007F906F900C941972DF91CF911F910F9152
:10E57000FF90EF90DF90CF90BF90AF909F908F90E3
:10E580007F906F9008956F927F928F929F92AF923B
:10E59000BF92CF92DF92EF92FF920F931F93CF9390
:10E5A000DF9300D0CDB7DEB78C01FC018681E82E69
:10E5B000E694E694E694F12C282F277081E090E011
:10E5C00011F480E090E0E80EF91EC70102960E9467
:10E5D000CB5C009709F445C00E94705CF801228171
:10E5E000FC012083F8012381FC0121830E94705CDF
:10E5F00002965C01A70160E070E00E945B93F80165
:10E6000004811581E12CF12CF8018081882339F1F6
:10E61000F8018180912C670163E0D594C7946A95D5
:10E62000E1F73701F7E06F227724CA0CDB1C883151
:10E6300028F00E94995D9401AC0108C00E94865D9B
:10E640009A8389839401AE014F5F5F4FB301C60186
:10E650000E943072E80CF91C0E5F1F4FD5CF81E08D
:10E6600090E00F900F90DF91CF911F910F91FF904D
:10E67000EF90DF90CF90BF90AF909F908F907F9062
:10E680006F900895E0915303F09154030994E09141
:10E690002C03F0912D030994E0915703F091580356
:10E6A0000994E0915903F0915A03099480E090E0B5
:10E6B00008950895E0912403F0912503099480E0E2
:10E6C00090E008950F931F93CF93DF93CDB7DEB7FC
:10E6D000E0970FB6F894DEBF0FBECDBF0E94B65CC8
:10E6E0008C010E94695CAE014F5F5F4F602F0E94FA
:10E6F000327B882309F446C088A99801281B310978
:10E70000C9010E94475C892BE9F12E8121110CC0BF
:10E71000BE016A5E7F4F88E10E948F5DE0914703F2
:10E72000F091480309952EC08A859B858D3C3BEA74
:10E73000930711F0019631F5223019F088E090E04E
:10E7400002C082E090E001979C012F5F3F4F1216BC
:10E750001306F4F6E1E0F0E0EC0FFD1FE80FF91FFF
:10E7600023852F3F81F3BE01645F7F4F89E10E94C3
:10E770008F5D89E10E94995D62E179E20E94855393
:10E78000892B31F6E0960FB6F894DEBF0FBECDBFF1
:10E79000DF91CF911F910F910895AF92BF92CF92C9
:10E7A000DF92EF92FF920F931F93CF93DF93CDB73A
:10E7B000DEB7E0970FB6F894DEBF0FBECDBF8C0179
:10E7C0006B01CE0101967C0180E3F70111928A95DD
:10E7D000E9F781E089838CE00E94865D8C831D824D
:10E7E0001F8280917C1491E0980F90937C1489870C
:10E7F00083E0B82EB8868DEC9BEA9B878A8789E1F7
:10E800000E94995D60E073E00E948553892B31F08E
:10E8100082E08E838FEF8C878D8709C089E10E940B
:10E82000995DBC01CE010C960E947C53BE828DEC9A
:10E830009BEA9D8B8C8B62E179E2CE0146960E9429
:10E840007C530E94695C9FA78EA70E94B65C88AB30
:10E85000C7010E942B7AB82E90E00E94CB5C892BD6
:10E8600031F10E94705CBC014B2DC7010E94497AB6
:10E87000E0901A03F0901B030E94C05C5C010E94B0
:10E88000705CB501F70109950115110581F000973C
:10E8900039F0019761F441E050E064E070E004C0B9
:10E8A00041E050E060E070E0C601F8010995E096B3
:10E8B0000FB6F894DEBF0FBECDBFDF91CF911F9191
:10E8C0000F91FF90EF90DF90CF90BF90AF900895A1
:10E8D0000E94AB7580937C14E0912403F091250392
:10E8E0000994892B29F0E0912403F091250304C0B9
:10E8F000E0912603F09127030994CF93DF93EC0175
:10E9000089919991009729F060E070E00E94D055BC
:10E91000F7CFDF91CF910895CF93DF93EC018991E9
:10E920009991009719F00E942255F9CFDF91CF916C
:10E930000895CF93DF93EC017B836A830E94446642
:10E9400099838883DF91CF910895FC018081918123
:10E9500022813381820F931F918380830895CF9307
:10E96000DF93EC010E94446699838883DF91CF9105
:10E970000895CF93DF93EC010E944466288139818A
:10E98000821B930B9C012F5F3F4F81E090E04A81F7
:10E990005B814217530710F080E090E0DF91CF9148
:10E9A0000895CF93DF93FC01C281D381808191814F
:10E9B000C80FD91F0E9444669E01281B390BC9014C
:10E9C000DF91CF910895CF93DF93EBE8FBE2CDE4A5
:10E9D000DBE2AFE7BBE21192119219921992199200
:10E9E00019921D928BE2E33AF807A9F7DF91CF91D4
:10E9F0000895CF93DF93FC01E158F44D40819C01D1
:10EA0000220F331F220F331F442301F1A0919400E2
:10EA1000B0919500FC01EE0FFF1FE557F44D80818A
:10EA20009181AD01481B590BCA01E901C35BD44D6B
:10EA3000488159816A817B81480F591F611D711D71
:10EA4000488359836A837B83B183A083F901E35BA5
:10EA5000F44D6081718182819381DF91CF9108951E
:10EA600060E070E0CB010895FC01EE0FFF1FEE0F98
:10EA7000FF1FE35BF44D40835183628373830895EA
:10EA8000CF93DF932FE73BE2CDE4DBE2EBE8FBE261
:10EA9000D9018D919D018823B9F040919400509146
:10EAA000950080819181BA01681B790B88819981D9
:10EAB000AA81BB81860F971FA11DB11D88839983F1
:10EAC000AA83BB835183408324963296BBE22B38C2
:10EAD0003B07F1F6DF91CF9108950C94BA790F932B
:10EAE0001F93FC01CB0140917D1450917E14338320
:10EAF00022831583048371836083F0937E14E093F3
:10EB00007D14452B11F40E94D47980E090E01F9190
:10EB10000F91089580917D1490917E140097C1F01B
:10EB200010927E1410927D14DC0114966D917C91EC
:10EB300015971296ED91FC9113970995E0917D142C
:10EB4000F0917E14309721F0808191810C94D479DA
:10EB500008950C94E58F0C94E18F84ED92E00E946F
:10EB600007568CEC92E00C940756CF93DF930E94EB
:10EB7000765C892BA9F08CEC92E00E942556EC0182
:10EB8000009721F10E94B65C998388830E94B15C52
:10EB90009B838A83CE0104960E94F25B8CAB14C0E7
:10EBA00084ED92E00E942556EC01009779F00296E0
:10EBB0000E94045C99838883BE016E547F4FCE010E
:10EBC0008E579F4F0E94595DCE0102C080E090E0B9
:10EBD000DF91CF910895BC016E547F4F8E579F4FA8
:10EBE0000C94595DCF93DF93EC01BC0184ED92E06E
:10EBF0000E946F56BE01892B19F084ED92E009C086
:10EC00008CEC92E00E946F56892B39F0BE018CEC9F
:10EC100092E0DF91CF910C944A56DF91CF91089505
:10EC20000F931F93CF93DF93EC01BC0184ED92E02F
:10EC30000E946F56892B91F0FE0161917191CF0175
:10EC40000E94155DBE016E547F4FCE018E579F4FBF
:10EC5000DF91CF911F910F910C946A5DBE018CECF6
:10EC600092E00E946F56892BD1F00E94025D68816C
:10EC700079818A819B810E94155D8CA990E00E9418
:10EC8000CB5C0CA910E00E94705CBE016C5F7F4FF2
:10EC9000A801DF91CF911F910F910C945293DF91B6
:10ECA000CF911F910F910895CF93DF93EC01BC0199
:10ECB00084ED92E00E946F56892B19F0CE010296E6
:10ECC0000CC0BE018CEC92E00E946F56892B19F0AB
:10ECD0008A819B8102C080E090E0DF91CF9108950E
:10ECE000FC01808191810895860F911D860F911DF1
:10ECF0008E579F4F0895860F911D860F911D8E5739
:10ED00009F4FFC0180819181089508958CED9AE1D7
:10ED10000E944958892B21F08CED9AE10C943658C9
:10ED20000895E091C81AF091C91A309709F0099432
:10ED300080E00895EF92FF920F931F93CF93DF939C
:10ED40007C01EA01FC0180819181009741F08C30C7
:10ED5000934071F1F7011182108283E0F2C080E0EC
:10ED600024E0829FF0011124E653F54E11821082B7
:10ED70008F5F8430A8F38093C71A8091021290911C
:10ED800003129093DB1A8093DA1A0E941B5580932A
:10ED9000A32B60E470E08CED9AE10E9422580E945F
:10EDA000A77C8CE093E0F7019183808381E0C9C068
:10EDB0006230D9F48091A42B9091A52B892B89F3F3
:10EDC0008091B52B863029F48091CD2B81FD0E9456
:10EDD000867681E00E94E47D8091A42B9091A52B02
:10EDE000892BF9F20E94AA78DCCF633060F56111BB
:10EDF00014C02097B1F2D093B230C093B13083E009
:10EE00000E94E47D8091A42B9091A52B892B11F079
:10EE10000E9491760E948676C4CF613011F62097C9
:10EE200009F4BFCFD093AE30C093AD3085E00E94DF
:10EE3000E47D8091A42B9091A52B892B09F4B1CF6F
:10EE40000E949176AECF6738E9F51092C61A0AECA7
:10EE50001AE18091C61A8430B8F4F8018281938156
:10EE60008C179D0749F4808191810E94B17DF80142
:10EE700011821082138212820C5F1F4F8091C61A7A
:10EE80008F5F8093C61AE5CFECECF0E38381948129
:10EE90008C179D0719F4148213821082B09621E317
:10EEA000EC34F20799F7E9E4F1E3818592858C1758
:10EEB0009D0711F4158214823D9681E3EB3CF8071F
:10EEC000A1F76FCF683809F06CCFCC5DDA4109F05B
:10EED00068CF8CED9AE10E944958892B09F461CFE3
:10EEE0001092C61AE091C61AE43008F05ACF20E218
:10EEF000E29FF0011124ED54FF4C818D8823D9F05D
:10EF00008CED9AE10E9436588091C61AE0E28E9FFD
:10EF1000C00111248D549F4C9093B2308093B13036
:10EF200082E00E94E47D8091A42B9091A52B892BF7
:10EF300011F00E9491768091C61A8F5F8093C61A55
:10EF4000D1CFDF91CF911F910F91FF90EF90089556
:10EF50009093C91A8093C81A089520910212309193
:10EF6000031260E0EAECFAE1643098F440815181E8
:10EF70004817590759F4428153814217530731F416
:10EF80006093C51A118210820C94B17D34966F5F24
:10EF9000EBCF6093C51A089540E0EAECFAE1443003
:10EFA000A8F451E0540F20813181232B61F4409368
:10EFB000C41A91838083209102123091031233830B
:10EFC00022830C94CB7D3496452FE9CF4093C41A0D
:10EFD00008952091021230910312FC01358F248F85
:10EFE000778F668F08952091021230910312FC01F1
:10EFF00032872187748763870895CF93DF93EA016F
:10F000000E94547D009749F0209102123091031222
:10F01000FC0132872187D487C387DF91CF91089580
:10F020000F931F93CF93DF9300D000D0CDB7DEB7FF
:10F030008C01AB018FEF89838A838B838C83B8012A
:10F04000CE0101960E94FD77009719F0FC0115830F
:10F0500004830F900F900F900F90DF91CF911F912D
:10F060000F91089540E050E062E08CED92E00E9444
:10F07000C1551092A52B1092A42B0895AC0161E00C
:10F080008CED92E00C94A355AC0160E08CED92E025
:10F090000C94A3550F931F93CF93DF938A010E9483
:10F0A000D37CEC01009759F08091021290910312E9
:10F0B0009D8F8C8F1F8F0E8FCE010E944478CE01C2
:10F0C000DF91CF911F910F910895CF93DF93A0917E
:10F0D000B130B091B230109719F0ED016C9605C0C7
:10F0E000C091AD30D091AE3029968091AC3086FF82
:10F0F00022C01092C31A40E0EAECFAE14430B8F4BE
:10F100002081318114968D919C911597281739078C
:10F1100059F482819381009739F04093C31A9983FF
:10F1200088831B821A8205C034964F5FE7CF4093D5
:10F13000C31A0E94867688819981009741F04A819E
:10F140005B816091A32BDF91CF910C94C155DF912E
:10F15000CF9108950F931F93CF93DF938091B52B99
:10F16000863009F071C08091A42B9091A52B811558
:10F17000954009F069C0C4E9D2E0D093A52BC093B3
:10F18000A42B02E00093AE2B14E91093AF2B109246
:10F19000D12B1092D02B0E94A17C809590959093BA
:10F1A000D12B8093D02B1092B72B1092B62B0E94AC
:10F1B000907C809590959093B72B8093B62B0E946E
:10F1C0009176D093A52BC093A42B0093AE2B1093D4
:10F1D000AF2BA091AF30B091B030FD01E459FD4F9D
:10F1E0008CE692E001900D920197E1F76CE672E0F7
:10F1F00084EC9BE20E944F7C8091A82B8093C42BCF
:10F200008091A92B8093C52B8091AA2B8093C62B2C
:10F210008091AB2B8093C72B1092D12B1092D02BC7
:10F220000E94A17C809590959093D12B8093D02BB8
:10F230001092B72B1092B62B0E94907C80959095DF
:10F240009093B72B8093B62BDF91CF911F910F91A5
:10F250000C949176FC01680F791F80E048E1E61775
:10F26000F70781F0219198E0322F3827532F517002
:10F2700030FD84278695513009F480682695915099
:10F2800099F7EDCF08951F920F920FB60F921124A8
:10F290000BB60F922F933F934F935F936F937F9390
:10F2A0008F939F93AF93BF93EF93FF9380919400BD
:10F2B000909195009093902B80938F2B81E0809379
:10F2C000812B80917100807D809371000E948A75EE
:10F2D0008091812B8823D9F18091940090919500A1
:10F2E00040918F2B5091902B84179507A0F480911B
:10F2F000552B9091562BA091572BB091582B8C5792
:10F30000914EAF4FBF4F8093552B9093562BA093A8
:10F31000572BB093582B2091940030919500241BCB
:10F32000350B8091552B9091562BA091572BB09176
:10F33000582B820F931FA11DB11D8093552B9093C5
:10F34000562BA093572BB093582B1092812BFF91E3
:10F35000EF91BF91AF919F918F917F916F915F914D
:10F360004F913F912F910F900BBE0F900FBE0F90BA
:10F370001F9018959FB7F894E1E7F0E08081807DB9
:10F38000808388B38F6288BB10929000E1E9F0E03F
:10F390001082109292001092950010929400808139
:10F3A000856080839FBF08952FB7F894909399004C
:10F3B0008093980088B38F6288BBE1E7F0E080819A
:10F3C000826080832FBF0895CF93DF93FC01DB0120
:10F3D00085E0EB0119928A95E9F78581837011F038
:10F3E00082E08C938781837021F082E012968C9367
:10F3F00012978581837081F08781837069F02389FA
:10F400003489818592852817390731F481E0848316
:10F4100012961C92129701C01482858183708230EB
:10F4200021F0833021F080E003C082E001C088E059
:10F4300011968C93119787818370823021F08330ED
:10F4400021F080E003C082E001C088E013968C9335
:10F45000DF91CF910895CF93DF9300D000D01F921A
:10F46000CDB7DEB7BE016F5F7F4F0E94E47989811F
:10F470009A81890F8D5F9B81890F9C81890F9D8166
:10F48000890F0F900F900F900F900F90DF91CF91F9
:10F4900008954F925F926F927F928F929F92AF9258
:10F4A000BF92CF92DF92EF92FF920F931F93CF9371
:10F4B000DF9300D000D000D0CDB7DEB78C017B0148
:10F4C000BE016F5F7F4F4E830E94E479B981AA81AC
:10F4D0005B804C808B2F90E003962A2F30E0820FC8
:10F4E000931F850D911D642D70E0860F971F5D8120
:10F4F000850F911D4E8150E0481759070CF49AC0B2
:10F50000F801818180FB662460F8712C43E0660C71
:10F51000771C4A95E1F7828180FB882480F8912C42
:10F5200054E0880C991C5A95E1F7862880818770F1
:10F53000882A838180FBAA24A0F8B12C85E0AA0C3C
:10F54000BB1C8A95E1F78A28848180FBCC24C0F813
:10F55000D12C96E0CC0CDD1C9A95E1F78C28F701B4
:10F560008082F80145814370F4E04F9FA00111248F
:10F57000F80186818370F0E18F9FC0011124482B30
:10F58000F8018781F0E48F9FC0011124482BF70117
:10F590004183F8018085F7018283B23059F4F80184
:10F5A0008185F7018383F8018285F701848395E0E3
:10F5B000C92E02C083E0C82EB0E080E090E0200FAA
:10F5C000311FDB2EDC0C0197BA1761F0A901480F3F
:10F5D000591FFA01B384A7014D0D511DFA01B082E4
:10F5E000BF5FEFCF9D2DF2E05F120EC0D701AD0DD2
:10F5F000B11DF80183898C9381E08D0DD701A80F8F
:10F60000B11D9E5F84898C9340E020E030E0060FBE
:10F61000171F842F890F21503109441561F0D8013B
:10F62000A20FB31F55965C91D701A80FB11D5C9333
:10F630004F5FEFCF80E026960FB6F894DEBF0FBE87
:10F64000CDBFDF91CF911F910F91FF90EF90DF9091
:10F65000CF90BF90AF909F908F907F906F905F9072
:10F660004F900895BF92CF92DF92EF92FF920F9347
:10F670001F93CF93DF937C01D62EEA0182E0861799
:10F6800008F0B1C0F701808186FBBB24B0F89181FE
:10F69000292F269526952370C92EC294C694C69408
:10F6A00053E0C522382F3770388383FB332730F976
:10F6B000398384FB332730F93A8385FB882780F927
:10F6C0008B83BC822D83892F829583708E83CF821A
:10F6D00082818887222389F13381848190E0982F69
:10F6E0008827830F911D9A87898787010B5F1F4F9A
:10F6F000223071F460E073E0CE010B960E947C53DF
:10F70000F70186818B8785818C870E5F1F4F20C014
:10F710002330F1F4F7013D9680E090E03E2F2F2F4B
:10F720004291DE01A80FB91F1B964C9301968830B9
:10F730009105B1F7032F122F0BC087010D5F1F4FEB
:10F7400060E073E0CE010B960E947C531A86198606
:10F75000CC20B9F1B1100DC0F8012081818190E079
:10F76000982F8827820F911D9C8B8B8B0E5F1F4FCC
:10F7700004C089859A859C8B8B8BF2E0CF120EC0DA
:10F7800060E073E0CE0145960E947C53F8018181D0
:10F790008D8B80818E8B0E5F1F4F1BC0F3E0CF12CD
:10F7A00018C0085F1F4FF80180E090E02291DE0151
:10F7B000A80FB91F55962C93019688309105B1F783
:10F7C00008C060E073E0CE0145960E947C531C8A1D
:10F7D0001B8AC8018E199F092D2D281B2FA71EA734
:10F7E0000DA7D81608F480E0DF91CF911F910F91FB
:10F7F000FF90EF90DF90CF90BF900895FB014150B4
:10F800005109460F571FE417F50778F4208130E0BF
:10F81000322F22276181260F311D820F931F8217FD
:10F82000930708F401963296EECFE417F50751F4EA
:10F83000208130E0322F2227820F931F82179307F7
:10F8400008F401960895CF93DF93C091AF2BD0E0D9
:10F8500064972091AE2B30E0322F2227C20FD31FA6
:10F8600048E050E068EB7BE29E01280F311DC901A2
:10F870000E94FE7BAE0160EC7BE20E94FE7B009763
:10F8800021F098278927982702C08FEF9FEFDF91FB
:10F89000CF9108959093F51A8093F41A0895FC017E
:10F8A0005381560F5093AB2B872F99274281480FD6
:10F8B0004093AA2BA181A093A92BE081E093A82BD0
:10F8C000242F30E02817390748F481E08A0F80930D
:10F8D000A92B811103C0EF5FE093A82B852F90E047
:10F8E00077278617970788F44F5F4093AA2B41111B
:10F8F0000CC08091A92B8F5F8093A92B811105C02B
:10F900008091A82B8F5F8093A82B0895AB01BC0139
:10F9100080E090E00E94FE7B982789279827089531
:10F9200044E150E06CEA7BE280E090E00E94FE7BE4
:10F93000009721F098278927982708958FEF9FEF48
:10F94000089586E00C94237C81E10C94237C80E074
:10F95000E82FF0E0EE0FFF1FED5CFE4C11821082ED
:10F960008F5F8430A8F380E090E2899FF00111243A
:10F97000ED54FF4C118E8F5F8430B0F380E094E043
:10F980009093EF1A8093EE1A80E09DE0989FF0012B
:10F990001124E75BFE4C158214828F5F8A30B0F32E
:10F9A0008093ED1A0895CF932091EE1A3091EF1ABB
:10F9B0002F5F3F4F21154DE7340710F020E030E175
:10F9C000522F432FE3EBF0E3C0E0C43059F0A18D98
:10F9D000AA2329F0A481B581A417B50749F3CF5F05
:10F9E000B096F3CF3093EF1A2093EE1A1092ED1ADF
:10F9F00020E0E0E0F0E02430E8F430E2239FD001A2
:10FA00001124AD54BF4C59963C915997311104C003
:10FA10002093ED1AFD0110C0373041F4309739F0D2
:10FA20005A964C915A97328D341708F0DF012F5FA8
:10FA3000FD01E1CF2093ED1A309799F122E0218F5B
:10FA40002091F01A24872091F11A25872091F21A2B
:10FA500026872091F31A278728ED34E0338B228BF9
:10FA6000358B248B21E030E0318B208B138E228F5D
:10FA700023E0208F168A20E1278B2091EE1A309107
:10FA8000EF1A32272327322735832483778366832F
:10FA9000DC014D915D916D917C9140835183628336
:10FAA0007383CF01CF910895CF93DF932091EE1A06
:10FAB0003091EF1A2F5F3F4F21154DE7340710F0BB
:10FAC00020E030E1522F432FEDE4F1E3C0E0CA30F3
:10FAD00041F0A081B181CF5F3D96A417B507B9F77A
:10FAE000E9CF3093EF1A2093EE1A40E05DE04A3000
:10FAF000A0F4A1E0A40F549FF0011124E75BFE4C99
:10FB000024813581232B39F44093ED1A309741F449
:10FB100080E090E023C04A2FEACF4093ED1AF8CF5F
:10FB20002091EE1A3091EF1A32272327322735839E
:10FB3000248377836683009729F4108211821282CE
:10FB4000138209C0EC0188819981AA81BB818083DD
:10FB50009183A283B38380E48087CF01DF91CF912B
:10FB6000089540E04430A0F4E42FF0E051E0540F59
:10FB7000EE0FFF1FED5CFE4C208131812817390705
:10FB800029F44093ED1A118210820895452FEACF8F
:10FB90004093ED1A089540E0443098F4E42FF0E0EB
:10FBA00051E0540FEE0FFF1FED5CFE4C20813181C0
:10FBB000232B29F44093ED1A918380830895452FD8
:10FBC000EBCF4093ED1A0895AF92BF92CF92DF92A0
:10FBD000EF92FF920F931F93CF93DF93C091B130B9
:10FBE000D091B230843009F4DCC124ED3BE2309393
:10FBF000B0302093AF303093A72B2093A62B8330C7
:10FC000059F4898D8F70833009F06BC08889998988
:10FC1000892B09F0DFC67FC0823009F080C0809157
:10FC2000F31A8F5F8093F31A811113C08091F21A37
:10FC30008F5F8093F21A81110CC08091F11A8F5F4F
:10FC40008093F11A811105C08091F01A8F5F809323
:10FC5000F01A1092A52B1092A42B109248311092FA
:10FC60004731298D822F8D7F853041F48A8D8F5FBA
:10FC70008A8F843109F0AEC6198EACC6222309F4EE
:10FC8000A9C688899989892B09F441C08A8D9FEF7B
:10FC9000980F9A8F81119EC68B8D883031F09FEF1F
:10FCA000920F923048F4853039F4198E80E88093B1
:10FCB000AC300E94657847C5853038F493E0082E53
:10FCC00001C0990F0A94EAF701C090E39A8F8F5F01
:10FCD0008B8F822F8F708330A1F048F4813009F42C
:10FCE0004FC3823009F076C61092CD2B4CC38630BC
:10FCF00009F4C8C4883009F4C5C4843009F06AC660
:10FD0000C1C484E08093AC300E9465784EC52F70EA
:10FD1000233009F05FC688E08093AC3009C5853098
:10FD200019F5E091AD30F091AE3084819581892B49
:10FD300009F450C61092B2301092B13088EC9BE2B8
:10FD40009093B0308093AF309093A72B8093A62BE5
:10FD500010924831109247311092A52B1092A42B8B
:10FD600088E08093AC301BC18091AC2B853409F0C6
:10FD700031C60091AE2B10E0102F00278091AF2BE1
:10FD8000080F111D8091A42B9091A52B801791072E
:10FD900008F420C61093A52B0093A42B8091B22BBE
:10FDA0008F7309F017C68091B32B811113C6809110
:10FDB000433190914431C0915D03D0915E038C1723
:10FDC0009D0759F4409145315091463120915F0390
:10FDD0003091600342175307A1F02091BC2B309162
:10FDE000BD2B2817390709F0F5C52091BE2B30919E
:10FDF000BF2B80914531909146312817390709F082
:10FE0000E9C50E94907C019609F0E4C58091B52B6C
:10FE1000863009F429C18131E9F1813009F0DAC570
:10FE20008091C02B883009F0D5C51092C02B8091ED
:10FE3000C22B9091C32B873F3FEF930710F0099699
:10FE400001C008969093C32B8093C22B8091B82B4E
:10FE50009091B92BA091BA2BB091BB2B8093BC2B66
:10FE60009093BD2BA093BE2BB093BF2B80914331B9
:10FE700090914431A0914531B09146318093B82B97
:10FE80009093B92BA093BA2BB093BB2B80E48093B3
:10FE9000B42B7DC50C5111091093A52B0093A42BF5
:10FEA00088EC9BE29093B0308093AF308091C62B6A
:10FEB0009091C72B892B29F00E94A47C019609F010
:10FEC00089C52091C22B3091C32B2115310509F42E
:10FED00081C589E491E39093AE308093AD30A090DA
:10FEE000C02BB090C12B40915F0350916003609193
:10FEF000610370916203A0916303B0916403009168
:10FF0000B82B1091B92BE090BA2BF090BB2BE0915D
:10FF1000AD30F091AE3081E3EB3CF80708F05AC504
:10FF200084819581009721F12817390709F5868189
:10FF30009781009719F0A816B906D1F480819181B4
:10FF40008C179D0729F4C280D380C416D506B1F062
:10FF50008617970729F4C280D380CA16DB0671F092
:10FF60000817190729F482819381E816F90631F000
:10FF70003D96F093AE30E093AD30C9CF1092B230E1
:10FF80001092B13082E08093AC3088EC9BE2909389
:10FF9000A72B8093A62B10924831109247310E94D4
:10FFA00065788091473190914831009709F412C5E6
:10FFB0009C01245E3F4F3093A52B2093A42B3093BC
:10FFC000AE2B2093AF2BE091AD30F091AE30208579
:10FFD0002093B42B21E12093B52B089698278927ED
:10FFE00098279093C52B8093C42B1092C72B109207
:10FFF000C62B848195819093C12B8093C02B8681E1
:020000021000EC
:1000000097819093C32B8093C22B80914331909121
:100010004431A0914531B09146318093B82B9093F3
:10002000B92BA093BA2BB093BB2B80819181A28175
:10003000B3818093BC2B9093BD2BA093BE2BB09328
:10004000BF2B84ED9BE29093B0308093AF300E9441
:10005000A47C80959095009711F48FEF9FEF90937B
:10006000C72B8093C62B93C40E94A17C019609F0F4
:10007000B1C48091C22B9091C32B009709F4AAC4FC
:100080002091C02B3091C12B2115310509F4A2C458
:100090004091B82B5091B92B6091BA2B7091BB2B2A
:1000A000ECECF0E3C3EBD0E3F080FF20A9F0AC81EF
:1000B000BD818A179B0781F4AE81BF812A173B0758
:1000C00059F4A881B9814A175B0731F4AA81BB8131
:1000D0006A177B0709F46FC1A096B096A1E3C333FA
:1000E000DA0711F72091CD2B2F732230D9F490939A
:1000F000EB1A8093EA1A40E0443090F4E42FF0E0E9
:10010000EE0FFF1FED5CFE4C208131814F5F8217A7
:10011000930791F71092ED1A20E0C0E0D0E07EC086
:100120004093ED1A8091CD2B82FD54C484E18093DD
:10013000CD2B88E290E09093A52B8093A42B80E5B3
:100140008093CC2B8091C72B9091CB2B9093C72B76
:100150003091C62B9091CA2B9093C62B3093CA2B0B
:100160002091C52B9091C92B9093C52B2093C92B1F
:100170009091C42B9093ED1A4091C82B4093C42BBF
:100180009093C82B8F5F8093CB2B81110FC081E0A0
:10019000830F8093CA2B811109C081E0820F809365
:1001A000C92B811103C09F5F9093C82B8091C02BF6
:1001B0009091C12B9093EB1A8093EA1A2091C22B55
:1001C0003091C32B3093C12B2093C02B9093C32B22
:1001D0008093C22B8091B82B9091B92BA091BA2B10
:1001E000B091BB2B8093BC2B9093BD2BA093BE2BC7
:1001F000B093BF2B8091433190914431A091453110
:10020000B09146318093B82B9093B92BA093BA2B21
:10021000B093BB2BA1C3373089F02F5F2430C0F4DB
:1002200030E2239FC0011124FC01ED54FF4C318DBD
:100230003111F1CF2093ED1AEF010CC0209721F07E
:10024000428D3A8D341748F7EC01CD54DF4CE5CFA1
:100250002093ED1A209709F4BDC3D093B230C09318
:10026000B13083E08A8F888F1E8A84E08F8B1B8E4B
:100270008091C22B9091C32B9D838C838091C02B46
:100280009091C12B9F838E838091B82B9091B92B35
:10029000A091BA2BB091BB2B88839983AA83BB838F
:1002A00081E0898F8091F01A8C878091F11A8D8777
:1002B0008091F21A8E878091F31A8F8781E090E007
:1002C000998B888B8091C72B8B878091C62B8A87CF
:1002D0008091C52B89878091C42B888781E090E02D
:1002E0000E944E858091CC2B282F207F30E0213535
:1002F00031050CF445C082958F7090E00597880F0A
:10030000991F880F991F3091EC1A20E0E22FF0E03E
:10031000E817F9078CF5E455F44D30A5311105C007
:100320002093ED1A1092EC1A2BC0313011F42F5F8C
:10033000EDCF3230E1F441A54430C9F42093ED1AF9
:100340003093EC1A82A590E0982F882723A5822B62
:100350009093EB1A8093EA1A893DA4E09A0710F073
:1003600088ED94E09B8B8A8B9D8B8C8B09C041A57B
:10037000442311F0240FCACF2093ED1A3093EC1AC6
:1003800080E18093CD2B8091CD2B82608093CD2B0B
:1003900082E08093D42B84E08093D52B8093D62B5E
:1003A00088ED8093D72B8CE290E09093A52B8093DF
:1003B000A42B80E67EC2D093B230C093B1301092AD
:1003C000AC309091CD2B92FF03C0198E80E21AC2FF
:1003D0008091CC2B82958F70880F880F8093ED1AB7
:1003E000081B1109045111091093A52B0093A42B8C
:1003F0008F2D8F70823029F4892F8F73823139F4D9
:100400001FC0813021F4892F8F738230C9F0012BF6
:1004100019F4892F8370A1F02091C42B88852813AB
:100420003EC22091C52B8985281339C22091C62B45
:100430008A85281334C22091C72B8B8528132FC29D
:1004400094FF4AC0688979896115710509F444C02F
:10045000CE010C960E944F7C3091C82B8091A82B26
:1004600038133AC02091C92B8091A92B281334C08E
:100470009091CA2B8091AA2B98132EC08091CB2BE0
:100480004091AB2B841328C03C872D879E878F8794
:100490008B8D81111AC02E89888D9A8D891B922F80
:1004A000969596959695891B280F2E8B87FD81959D
:1004B0009F89392F36953695931B980F9F8B822FE6
:1004C000869586958695890F888F81E08093AC30DC
:1004D000888D8A8F198A188A498D842F8F7090E0B1
:1004E000FC013197E830F10508F074C2E057FF4F86
:1004F0000C94918D8091AC3080FF14C083E0898F83
:1005000080E48093AC30198A188A8091A42B909152
:10051000A52B009709F408C122E42093AC300E9477
:100520004E8502C18091CD2B8F73823009F052C26B
:1005300027CF8091AC3080FF70C08091CD2B8F731E
:10054000823109F06AC08091CC2B282F207F30E0C7
:10055000213531050CF445C082958F7090E00597E8
:10056000880F991F880F991F3091EC1A20E0E22F15
:10057000F0E0E817F9078CF5E455F44D30A531119A
:1005800005C02093ED1A1092EC1A2BC0313011F4F3
:100590002F5FEDCF3230E1F441A54430C9F4209310
:1005A000ED1A3093EC1A82A590E0982F882723A5A6
:1005B000822B9093EB1A8093EA1A893D24E09207EC
:1005C00010F088ED94E09B8B8A8B9D8B8C8B09C0FF
:1005D00041A5442311F0240FCACF2093ED1A309384
:1005E000EC1A83E0898F8091C42B88878091C52B7A
:1005F00089878091C62B8A878091C72B8B8781E062
:1006000090E00E944E8582E48093AC30198A188A6B
:100610001092A52B1092A42B87C080E28093AC305F
:100620000E946578E091B130F091B230118E7ACDB0
:100630008091CD2B80FF28C044FD26C088899989F0
:10064000892B09F0C7C18091A42B9091A52B01960D
:100650000E944E852091AC30822F80618093AC3017
:100660008091A42B9091A52B892B19F022612093C6
:10067000AC300E94657881E090E0998B888B88E0AF
:10068000898F1B8E81E10CC185FF1CC08091D22B0C
:1006900090E0982F88272091D32B822B2091AF3088
:1006A0003091B030280F391F3093B0302093AF30E5
:1006B0002091A42B3091A52B281B390B3093A52B0F
:1006C0002093A42B8091A42B9091A52B009749F007
:1006D00044FD07C02091AC3022602093AC300E94D2
:1006E0004E858091CE2B90E0982F88272091CF2B9C
:1006F000820F911D9093EB1A8093EA1A2C893D8901
:100700002817390710F0892B21F43093EB1A209326
:10071000EA1A8091EA1A9091EB1A9B8B8A8B80914E
:10072000AC30837009F456C11092483110924731B1
:100730000E9465788091AC3085FF07C010924831E7
:1007400010924731198E84E1ABC084FF0AC0109229
:1007500048311092473181E090E0998B888B84E09A
:100760008FCF209147313091483121153105E1F08B
:1007700080FF02C0198A188A88899989009781F4B4
:100780008A899B898217930720F49093483180933C
:1007900047318091473190914831998B888B04C0C3
:1007A00090934831809347311B8E8091A62B909176
:1007B000A72B9093B0308093AF30809147319091C8
:1007C0004831892B59F088899989009739F08896A2
:1007D0009093A52B8093A42B88E10BC08091AC3023
:1007E00081FFF8C088E290E09093A52B8093A42B22
:1007F00080E18093CD2B5CC08091AC3080FFEAC05B
:10080000198E80E18093AC300E946578E3C08091BE
:10081000A42B9091A52B009711F00E944E859091EA
:10082000CD2B8091AC3090FF0BC080FF06C087E0DD
:10083000898F1A8E198A188A19C086E0898F16C086
:1008400080FF1EC085E0898F198A188AC3C08091F5
:10085000A42B9091A52B009711F00E944E858091BA
:10086000CD2B80FF0DC087E0898F1A8E81E090E04C
:100870000E944E8580E18093AC300E9465780FC065
:100880008091A42B9091A52B892B49F4A3C0809132
:10089000AC3080FF9FC087E0898F1A8E9BC080E1BB
:1008A0008093CD2B88E290E09093A52B8093A42B8E
:1008B00080E58093CC2B88858093C82B8985809395
:1008C000C92B8A858093CA2B8B858093CB2B8C85F3
:1008D0008093C42B8D858093C52B8E858093C62BEA
:1008E0008F858093C72B86E08093B52B8C819D816B
:1008F0009093C12B8093C02B8E819F819093C32BAB
:100900008093C22B8091433190914431A091453125
:10091000B09146318093B82B9093B92BA093BA2B0A
:10092000B093BB2B88819981AA81BB818093BC2B1A
:100930009093BD2BA093BE2BB093BF2B898D84FFCA
:1009400005C01092CF2B1092CE2B06C084E080936E
:10095000CE2B88ED8093CF2B80E48093B42B8091B5
:10096000A42B9091A52B9093AE2B8093AF2B10923C
:10097000D32B1092D22B1092D12B1092D02B0E94FD
:10098000A17C809590959093D12B8093D02B85E47A
:100990008093AC2B1092AD2B1092B32B1092B22BF4
:1009A0008091F41A9091F51A01969093F51A80931C
:1009B000F41A9093B02B8093B12B1092B72B109216
:1009C000B62B0E94907C809590959093B72B809346
:1009D000B62B04C01092A52B1092A42B1092AC3011
:1009E000DF91CF911F910F91FF90EF90DF90CF900B
:1009F000BF90AF90089598278927982708950E945F
:100A0000978D0895FC018091A62B9091A72B2CEA3D
:100A100030E3281B390BAB01261737070CF4A9016B
:100A20001416150654F45093483140934731E81793
:100A3000F90719F0BF010C945293089580E8809350
:100A40006100109261000E94D8630E9438550E9494
:100A5000B6678091532990915429009729F0019706
:100A60009093542980935329C0905529D0905629AA
:100A7000E0905729F09058290E947266C616D70652
:100A8000E806F90611F30E94726660935529709387
:100A900056298093572990935829D7CF2091B13068
:100AA0003091B230BC01C90108960E944F7CE091A0
:100AB000B130F091B2308091A82B80878091A92B22
:100AC00081878091AA2B82878091AB2B83870895A1
:100AD0002F923F924F925F926F927F928F929F924E
:100AE000AF92BF92CF92DF92EF92FF920F931F933C
:100AF000CF93DF93CDB7DEB763970FB6F894DEBF21
:100B00000FBECDBF7C011B016A01FC01178216825A
:100B1000838181FF66C3BE016F5F7F4F4B01F70189
:100B20009381F10193FD859193FF81911F018823AA
:100B300009F453C3853239F493FD859193FF819174
:100B40001F01853239F4B70190E00E94D593560118
:100B50006501E5CF10E0512C20E02032A0F48B326B
:100B600069F030F4803259F0833269F420612CC08E
:100B70008D3239F0803339F4216026C02260246040
:100B800023C0286021C027FD27C030ED380F3A3040
:100B900078F426FF06C0FAE01F9F300D1124132FB2
:100BA00013C06AE0569E300D1124532E20620CC0F3
:100BB0008E3221F426FD11C3206406C08C3611F458
:100BC000206802C0883641F4F10193FD859193FFBE
:100BD00081911F018111C1CF9BEB980F933018F4C5
:100BE0002061805E06C09BE9980F933008F0AAC18F
:100BF0002F7E26FF16E02F73722E853621F4F22FFA
:100C0000F0647F2E08C0863621F4622F6068762E4D
:100C100002C01111115077FE07C01C3348F4442460
:100C20004394410E27E00BC0183030F4212F06C04A
:100C300027E04CE3442E03C027E017E0412C560187
:100C400074E0A70EB11CF6016081718182819381ED
:100C5000042DA4010E945A926C01098100FF02C078
:100C600003FF06C071FC07C072FC08C0612C08C0FD
:100C70003DE2632E05C02BE2622E02C090E2692E97
:100C8000802F8C7099F1662011F084E001C083E020
:100C9000851510F0512C0BC0581A73FC08C0B70111
:100CA00080E290E00E94D5935A94C9F7F3CF662072
:100CB00029F0B701862D90E00E94D59303FD03C073
:100CC0000DE911E102C009E911E1F72DF0717F2E64
:100CD000F8018491882309F476C271108052B7011B
:100CE00090E00E94D5930F5F1F4FF2CF77FE0FC0A9
:100CF0004C0C04FF04C08A81813309F44A94141413
:100D000074F5F8E0F41578F588E0482E2CC076FCF0
:100D10002AC0812F90E08C159D059CF06CEFC616C3
:100D20006FEFD60674F0772D7068772E0AC0E2E078
:100D3000F0E0EC0FFD1FE10FF11D8081803319F40D
:100D400011501111F4CF77FE0EC044244394410E8C
:100D5000812F90E0C816D9062CF41C1904C0442435
:100D6000439401C010E077FE07C01C141D043CF43E
:100D700096012F5F3F4F05C025E030E002C021E023
:100D800030E0662011F02F5F3F4F112331F0412FEB
:100D900050E04F5F5F4F240F351F452D50E0241763
:100DA000350714F4521A01C0512C872D897049F46B
:100DB000552039F0B70180E290E00E94D5935A9413
:100DC000F7CF662029F0B701862D90E00E94D593D9
:100DD00073FC09C0552039F0B70180E390E00E9410
:100DE000D5935A94F7CF77FE5FC09C2D8D2DD7FEFB
:100DF00002C090E080E0692E782E40E050E0C6010D
:100E0000841991099D878C87960126193709280D29
:100E1000391D812F90E0EE27FF27E81BF90BFF8794
:100E2000EE87FFEF6F167F0669F4B7018EE290E060
:100E30002B8B3A8B488B598B0E94D59359894889C3
:100E40003A892B89C614D70454F06C857D856615C4
:100E500077052CF4F901E40FF51F818101C080E3CF
:100E600071E0671A71084F5F5F4FEE85FF856E1660
:100E70007F066CF0B70190E02B8B3A8B488B598B37
:100E80000E94D5932B893A8948895989CACF6C1415
:100E90007D0439F49A81963318F4953311F404FFE4
:100EA00081E3B70190E04BC08A81813309F00F7E66
:100EB000B70190E00E94D593111105C074FE18C0CF
:100EC00085E490E017C0B7018EE290E00E94D593D0
:100ED00082E066246394680EF401E80FF11D8081BE
:100EE000B70190E00E94D593115041F3862DF1CFC8
:100EF00085E690E0B7010E94D593D7FC05C0C114E8
:100F0000D10439F404FF05C0D194C194D1088DE215
:100F100001C08BE2B70190E00E94D59380E36AE0C4
:100F2000C616D1042CF08F5FFAE0CF1AD108F7CFA4
:100F3000B70190E00E94D593B701C601C0960E9408
:100F4000D59341C1833631F0833779F0833509F089
:100F500058C021C0560172E0A70EB11CF601808175
:100F6000898301E010E0640114C05601F2E0AF0E85
:100F7000B11CF601C080D18026FF03C0612F70E054
:100F800002C06FEF7FEFC6012B8B0E9481938C0113
:100F90002B892F7715C05601F2E0AF0EB11CF60178
:100FA000C080D18026FF03C0612F70E002C06FEFC8
:100FB0007FEFC6012B8B0E9443938C012B89206805
:100FC000722E23FD1AC0852D90E008171907A8F48A
:100FD000B70180E290E00E94D5935A94F4CFF601D5
:100FE00077FC859177FE81916F01B70190E00E94B7
:100FF000D59351105A94015011090115110579F733
:10100000E2C0843611F0893651F5560127FF09C038
:10101000F4E0AF0EB11CF601608171818281938191
:101020000AC0F2E0AF0EB11CF60160817181882721
:1010300077FD8095982F022F0F7697FF08C0909527
:101040008095709561957F4F8F4F9F4F00682AE084
:1010500030E0A4010E940F95C82EC8183EC0022F90
:10106000853721F40F7E2AE030E01DC0097F8F36DE
:1010700091F018F4883559F0B0C0803719F08837EE
:1010800011F0ABC0006104FF09C0046007C024FF79
:1010900008C0066006C028E030E005C020E130E06E
:1010A00002C020E132E0560107FF09C0F4E0AF0EB4
:1010B000B11CF601608171818281938108C0F2E0E8
:1010C000AF0EB11CF6016081718180E090E0A40157
:1010D0000E940F95C82EC8180F7706FF0BC0202F4F
:1010E0002E7FC11650F404FF0AC002FD08C0202F55
:1010F0002E7E05C0DC2C202F03C0DC2C01C0D12E9D
:1011000024FF0DC0FE01EC0DF11D8081803311F430
:10111000297E09C022FF06C0D394D39404C0822F35
:10112000867809F0D39423FD13C020FF06C01C2D40
:10113000D51418F4150D1D19D52CD51468F4B70164
:1011400080E290E02B8B0E94D593D3942B89F5CF2E
:10115000D51410F45D1801C0512C24FF12C0B70142
:1011600080E390E02B8B0E94D5932B8922FF17C040
:1011700021FF03C088E590E002C088E790E0B70156
:101180000CC0822F867859F021FD02C080E201C098
:101190008BE227FD8DE2B70190E00E94D593C11646
:1011A00038F4B70180E390E00E94D5931150F7CF57
:1011B000CA94F401EC0DF11D8081B70190E00E940A
:1011C000D593C110F5CF552009F4C2CCB70180E208
:1011D00090E00E94D5935A94F6CFF70186819781CB
:1011E00002C08FEF9FEF63960FB6F894DEBF0FBE7D
:1011F000CDBFDF91CF911F910F91FF90EF90DF90C6
:10120000CF90BF90AF909F908F907F906F905F90A6
:101210004F903F902F9008955058BB27AA270ED08B
:101220004EC23FD230F044D220F031F49F3F11F44F
:101230001EF4FFC10EF4E095E7FBF5C1E92F50D293
:1012400080F3BA17620773078407950718F071F4E3
:101250009EF568C20EF4E0950B2EBA2FA02D0B015F
:10126000B90190010C01CA01A0011124FF27591BEB
:1012700099F0593F50F4503E68F11A16F040A22FF1
:10128000232F342F4427585FF3CF46953795279562
:10129000A795F0405395C9F77EF41F16BA0B620B61
:1012A000730B840BBAF09150A1F0FF0FBB1F661FA8
:1012B000771F881FC2F70EC0BA0F621F731F841FEB
:1012C00048F4879577956795B795F7959E3F08F011
:1012D000B3CF9395880F08F09927EE0F97958795D0
:1012E0000895DFD158F080E891E009F49EEFE0D155
:1012F00028F040E851E059F45EEF09C09AC112C2EB
:10130000E92FE078EDD168F3092E052AC1F32617FD
:1013100037074807590738F00E2E07F8E02569F01F
:10132000E025E0640AC0EF6307F8009407FADB01E8
:10133000B9019D01DC01CA01AD01EF9347D0BFD1D6
:101340000AD05F91552331F02BED3FE049E450FD89
:1013500049EC63CF0895DF93DD27B92FBF7740E8CD
:101360005FE31616170648075B0710F4D92FE5D17F
:101370009F938F937F936F934AD3E0E3F1E06CD117
:101380009ED12F913F914F915F919ED2DD2349F0E5
:101390009058A2EA2AED3FE049EC5FE3D0785D2760
:1013A0004DDFDF918CC11BD108F481E008950CD092
:1013B00086C17ED140F075D130F021F45F3F19F045
:1013C00032C15111B0C135C18BD198F39923C9F302
:1013D0005523B1F3951B550BBB27AA27621773073B
:1013E000840738F09F5F5F4F220F331F441FAA1FEF
:1013F000A9F333D00E2E3AF0E0E830D091505040AF
:10140000E695001CCAF729D0FE2F27D0660F771F5C
:10141000881FBB1F261737074807AB07B0E809F03E
:10142000BB0B802DBF01FF2793585F4F2AF09E3FD3
:10143000510568F0F8C077C15F3FECF3983EDCF3EC
:10144000869577956795B795F7959F5FC9F7880F4C
:10145000911D9695879597F90895E1E0660F771F9E
:10146000881FBB1F621773078407BA0720F0621B2F
:10147000730B840BBA0BEE1F88F7E095089519F4EF
:101480000EF0D1C04FC1D5C033D1C8F39638C0F7E4
:1014900007F80F92E8942BE33AEA48EB5FE716D29D
:1014A0000F920F920F924DB75EB70F92CED1EDE52E
:1014B000F1E0D2D04F915F91EF91FF91E595EE1F52
:1014C000FF1F49F0FE57E0684427EE0F441FFA95CE
:1014D000E1F74195550B3AD10F9007FE2EC10895C3
:1014E00097FB0EF4A9D03EC0E89409C097FB3EF4E8
:1014F00090958095709561957F4F8F4F9F4F992361
:10150000A9F0F92F96E9BB279395F69587957795DE
:101510006795B795F111F8CFFAF4BB0F11F460FF9E
:101520001BC06F5F7F4F8F4F9F4F16C0882311F0F6
:1015300096E911C0772321F09EE8872F762F05C00A
:10154000662371F096E8862F70E060E02AF09A95A5
:10155000660F771F881FDAF7880F9695879597F99A
:101560000895E894F92F96EBFF2381F012161306E5
:101570001406440B9395F69587957795679557953F
:101580004040FF23B9F71BC099270895882351F4E1
:101590009850D2F7872B762F652F542F432F322F59
:1015A00020E0B1F3121613061406440B88233AF018
:1015B0009A95440F551F661F771F881FCAF755233A
:1015C0004AF4440F551F11F460FF04C06F5F7F4F52
:1015D0008F4F9F4F880F9695879597F90895990F8C
:1015E0000008550FAA0BE0E8FEEF16161706E807ED
:1015F000F907C0F012161306E407F50798F0621B0E
:10160000730B840B950B39F40A2661F0232B242BE2
:10161000252B21F408950A2609F4A140A6958FEF01
:10162000811D811D089597F99F6780E870E060E053
:1016300008959FEF80EC0895909580957095609542
:1016400050954095309521953F4F4F4F5F4F6F4FCD
:101650007F4F8F4F9F4F0895DF93CF931F930F932B
:10166000FF92EF92DF927B018C01689405C0DA2E25
:10167000EF012AD1FE01E894A5912591359145917C
:101680005591AEF3EF01DADDFE019701A801DA947E
:1016900079F7DF90EF90FF900F911F91CF91DF913D
:1016A000089500240A9416161706180609060895C8
:1016B00000240A9412161306140605060895092E2E
:1016C0000394000C11F4882352F0BB0F40F4BF2B9D
:1016D00011F460FF04C06F5F7F4F8F4F9F4F0895DD
:1016E00057FD9058440F551F59F05F3F71F04795D3
:1016F000880F97FB991F61F09F3F79F087950895B8
:10170000121613061406551FF2CF4695F1DF08C0D6
:10171000161617061806991FF1CF869571056105F3
:1017200008940895E894BB2766277727CB0197F99B
:10173000089555DF08F48FEF08959B01AC0160E038
:1017400070E080E89FE333CE6ECF64C1D1DFE8F371
:101750009923D9F3940F511DBBF39150504094F04D
:1017600059F0882332F0660F771F881F9150504040
:10177000C1F79E3F510544F7880F911D96958795B7
:1017800097F908955F3FACF0983E9CF0BB27869593
:1017900077956795B79508F4B1609395C1F7BB0F3E
:1017A00058F711F460FFE8CF6F5F7F4F8F4F9F4F67
:1017B000E3CFB9CF0AD029ED3BE54EED5EE378C02B
:1017C0000EF028C136CF68942ECF92DFC8F399234C
:1017D000D1F3C6F3DF93CF931F930F93FF92C92FDB
:1017E000DD2788232AF02197660F771F881FDAF7F5
:1017F00020E030E040E85FEB9FE3883920F0803E56
:1018000030F021968F7709DDE5E8F1E003C005DDD2
:10181000E2EBF1E021DF8B01BE01EC01FB2E6F5703
:1018200071097595771F880B990B60DE28E132E707
:1018300041E35FE349D0AF2D9801AE01FF900F91D6
:101840001F91CF91DF91FADC3ACFFA01DC01AA0FA8
:10185000BB1F9B01AC01BF5728F422273327442725
:1018600050781FC0B75188F4AB2F002446953795A8
:101870002795011CA395D2F3002069F0220F331F96
:10188000441FB395DAF30DD0C7CC61307105A0E8E1
:101890008A07B94630F49B01AC0166277727882771
:1018A0009078309621F020833183428353830895CA
:1018B0000BD005CFF6DE28F0FBDE18F0952309F0FB
:1018C000B2CEB7CE11242FCF0BDFA0F3959FD1F36B
:1018D000950F50E0551F629FF001729FBB27F00DDE
:1018E000B11D639FAA27F00DB11DAA1F649F662733
:1018F000B00DA11D661F829F2227B00DA11D621F82
:10190000739FB00DA11D621F839FA00D611D221F3B
:10191000749F3327A00D611D231F849F600D211D1F
:10192000822F762F6A2F11249F5750408AF0E1F0C2
:1019300088234AF0EE0FFF1FBB1F661F771F881F0B
:1019400091505040A9F79E3F510570F06CCEEBCE00
:101950005F3FECF3983EDCF3869577956795B795F6
:10196000F795E7959F5FC1F7FE2B880F911D969520
:10197000879597F90895FA01EE0FFF1F309621051C
:10198000310599F16115710561F48038BFE39B075A
:1019900049F168949038810561F08038BFEF9B076A
:1019A00041F0992342F5FF3FE1053105210511F191
:1019B000E8940894E795D901AA2329F4AB2FBE2F08
:1019C000F85FD0F310C0FF5F70F4A695E0F7F73929
:1019D00050F019F0FF3A38F49F779F930CD00F9096
:1019E00007FC905808953EF024CE60E070E080E857
:1019F0009FE308954FE79F775F934F933F932F9314
:101A0000E4DE2F913F914F915F9152DF3DCD9B01DD
:101A1000AC014ECF9F3F31F0915020F487957795E0
:101A20006795B795880F911D9695879597F90895B5
:101A3000DB018F939F930E94BC8DBF91AF91A29FBA
:101A4000800D911DA39F900DB29F900D11240895BC
:101A5000AA1BBB1B51E107C0AA1FBB1FA617B707D4
:101A600010F0A61BB70B881F991F5A95A9F78095F0
:101A70009095BC01CD01089597FB072E16F40094B4
:101A800007D077FD09D00E94288D07FC05D03EF4D1
:101A9000909581959F4F0895709561957F4F08951A
:101AA000A1E21A2EAA1BBB1BFD010DC0AA1FBB1F62
:101AB000EE1FFF1FA217B307E407F50720F0A21BD4
:101AC000B30BE40BF50B661F771F881F991F1A9441
:101AD00069F760957095809590959B01AC01BD016B
:101AE000CF010895052E97FB1EF400940E94898D66
:101AF00057FD07D00E94508D07FC03D04EF40C9484
:101B0000898D50954095309521953F4F4F4F5F4FB0
:101B1000089590958095709561957F4F8F4F9F4F59
:101B20000895EE0FFF1F0590F491E02D09946927A9
:101B30009627692778278727782708950E94A68DFA
:101B4000332312F48A1B9B0B0C94B78DA29FB00118
:101B5000B39FC001A39F700D811D1124911DB29FE1
:101B6000700D811D1124911D08950E94A68DB7FF4F
:101B70000895821B930B08950E94A68DA59F900D3A
:101B8000B49F900DA49F800D911D11240895B7FF5F
:101B90000C94BC8D0E94BC8D821B930B0895DF9327
:101BA000CF931F930F939A9DF02D219FF00D8B9D46
:101BB000F00D8A9DE02DF10D039FF00D029FE00DC9
:101BC000F11D4E9DE00DF11D5E9DF00D4F9DF00D40
:101BD0007F936F93BF92AF925F934F93D5010E9413
:101BE000A68D8B01AC01D7010E94A68DEB01E80FF9
:101BF000F91FD6010E941F8E2F913F91D6010E949E
:101C0000A68DC60FD71FE81FF91FAF91BF910E9485
